:020000040800F2
:10000000A0C00024F13F00089DB20308DD3F0008B6
:10001000DD3F0008DD3F0008DD3F00080000000074
:100020000000000000000000000000004D4000083B
:10003000DD3F00080000000045420008B9C4000888
:10004000C1420008C1420008C1420008C142000884
:10005000C1420008C1420008C1420008C142000874
:10006000C1420008C1420008C1420008C142000864
:10007000C1420008C1420008C1420008C142000854
:10008000C1420008C1420008C1420008C142000844
:10009000C1420008C1420008C1420008C142000834
:1000A000C1420008C1420008C1420008C142000824
:1000B000C1420008C1420008C1420008C142000814
:1000C000C1420008C1420008C1420008C142000804
:1000D000C1420008C1420008C1420008C1420008F4
:1000E000C1420008C1420008C1420008C1420008E4
:1000F000C1420008C1420008C1420008C1420008D4
:10010000C1420008C1420008C1420008C1420008C3
:10011000C1420008C1420008C1420008C1420008B3
:10012000C1420008C1420008C1420008C1420008A3
:10013000C1420008C1420008C1420008C142000893
:10014000C1420008C1420008C1420008C142000883
:10015000C1420008C1420008C1420008C142000873
:10016000C1420008C1420008C1420008C142000863
:10017000C1420008C1420008C1420008C142000853
:10018000C1420008C1420008C1420008C142000843
:10019000C1420008C1420008C1420008C142000833
:1001A000C1420008C1420008C1420008C142000823
:1001B000C1420008C1420008C1420008C142000813
:0401C000C142000830
:1001C80081F0004102E000BF83F0004330B54FEA00
:1001D80041044FEA430594EA050F08BF90EA020F6D
:1001E8001FBF54EA000C55EA020C7FEA645C7FEA00
:1001F800655C00F0E2804FEA5454D4EB5555B8BF23
:100208006D420CDD2C4480EA020281EA030382EA93
:10021800000083EA010180EA020281EA0303362D25
:1002280088BF30BD11F0004F4FEA01314FF4801CF8
:100238004CEA113102D0404261EB410113F0004F0A
:100248004FEA03334CEA133302D0524263EB4303C1
:1002580094EA050F00F0A780A4F10104D5F1200E5F
:100268000DDB02FA0EFC22FA05F2801841F10001BA
:1002780003FA0EF2801843FA05F359410EE0A5F18E
:1002880020050EF1200E012A03FA0EFC28BF4CF0BF
:10029800020C43FA05F3C01851EBE37101F0004575
:1002A80007D54FF0000EDCF1000C7EEB00006EEB82
:1002B8000101B1F5801F1BD3B1F5001F0CD349080C
:1002C8005FEA30004FEA3C0C04F101044FEA445263
:1002D80012F5800F80F09A80BCF1004F08BF5FEAEA
:1002E800500C50F1000041EB045141EA050130BDCA
:1002F8005FEA4C0C404141EB0101013C28BFB1F5DC
:10030800801FE9D291F0000F04BF01460020B1FA26
:1003180081F308BF2033A3F10B03B3F120020CDAF9
:100328000C3208DD02F1140CC2F10C0201FA0CF0D7
:1003380021FA02F10CE002F11402D8BFC2F1200C3C
:1003480001FA02F120FA0CFCDCBF41EA0C019040F2
:10035800E41AA2BF01EB0451294330BD6FEA04043B
:100368001F3C1CDA0C340EDC04F11404C4F1200226
:1003780020FA04F001FA02F340EA030021FA04F338
:1003880045EA030130BDC4F10C04C4F1200220FA8F
:1003980002F001FA04F340EA0300294630BD21FACD
:1003A80004F0294630BD94F0000F83F4801306BF93
:1003B80081F480110134013D4EE77FEA645C18BF87
:1003C8007FEA655C29D094EA050F08BF90EA020F1E
:1003D80005D054EA000C04BF1946104630BD91EA16
:1003E800030F1EBF0021002030BD5FEA545C05D119
:1003F8004000494128BF41F0004130BD14F5800458
:100408003CBF01F5801130BD01F0004545F0FE41CB
:1004180041F470014FF0000030BD7FEA645C1ABF00
:10042800194610467FEA655C1CBF0B46024650EA37
:10043800013406BF52EA033591EA030F41F4002163
:1004480030BD00BF90F0000F04BF0021704730B5E9
:100458004FF4806404F132044FF000054FF00001BE
:1004680050E700BF90F0000F04BF0021704730B57F
:100478004FF4806404F1320410F0004548BF404254
:100488004FF000013EE700BF42004FEAE2014FEAA9
:1004980031014FEA02701FBF12F07F4393F07F4F84
:1004A80081F06051704732F07F4208BF704793F087
:1004B8007F4F04BF41F40021704730B54FF460749A
:1004C80001F0004521F000411CE700BF50EA01029D
:1004D80008BF704730B54FF000050AE050EA010246
:1004E80008BF704730B511F0004502D5404261EBB6
:1004F80041014FF4806404F132045FEA915C3FF4F7
:10050800D8AE4FF003025FEADC0C18BF03325FEA93
:10051800DC0C18BF033202EBDC02C2F1200300FA44
:1005280003FC20FA02F001FA03FE40EA0E0021FA69
:1005380002F11444BDE600BF70B54FF0FF0C4CF457
:10054800E06C1CEA11541DBF1CEA135594EA0C0F09
:1005580095EA0C0F00F0DEF82C4481EA030621EA44
:100568004C5123EA4C5350EA013518BF52EA03357F
:1005780041F4801143F4801338D0A0FB02CE4FF031
:100588000005E1FB02E506F00042E0FB03E54FF061
:100598000006E1FB03569CF0000F18BF4EF0010E59
:1005A800A4F1FF04B6F5007F64F5407404D25FEA55
:1005B8004E0E6D4146EB060642EAC62141EA555108
:1005C8004FEAC52040EA5E504FEACE2EB4F1FD0C4A
:1005D80088BFBCF5E06F1ED8BEF1004F08BF5FEAC8
:1005E800500E50F1000041EB045170BD06F000467A
:1005F80046EA010140EA020081EA0301B4EB5C0427
:10060800C2BFD4EB0C0541EA045170BD41F480111E
:100618004FF0000E013C00F3AB8014F1360FDEBF43
:10062800002001F0004170BDC4F10004203C35DA1F
:100638000C341BDC04F11404C4F1200500FA05F3A2
:1006480020FA04F001FA05F240EA020001F0004243
:1006580021F0004110EBD37021FA04F642EB0601B9
:100668005EEA430E08BF20EAD37070BDC4F10C04E3
:10067800C4F1200500FA04F320FA05F001FA04F2A7
:1006880040EA020001F0004110EBD37041F1000193
:100698005EEA430E08BF20EAD37070BDC4F120059E
:1006A80000FA05F24EEA020E20FA04F301FA05F206
:1006B80043EA020321FA04F001F0004121FA04F2AE
:1006C80020EA020000EBD3705EEA430E08BF20EA7E
:1006D800D37070BD94F0000F0FD101F000464000B8
:1006E80041EB010111F4801F08BF013CF7D041EA3A
:1006F800060195F0000F18BF704703F0004652003E
:1007080043EB030313F4801F08BF013DF7D043EA0E
:100718000603704794EA0C0F0CEA135518BF95EAC4
:100728000C0F0CD050EA410618BF52EA4306D1D14B
:1007380081EA030101F000414FF0000070BD50EA6A
:10074800410606BF1046194652EA430619D094EAF4
:100758000C0F02D150EA013613D195EA0C0F05D1DE
:1007680052EA03361CBF104619460AD181EA030132
:1007780001F0004141F0FE4141F470014FF00000EA
:1007880070BD41F0FE4141F4780170BD70B54FF085
:10079800FF0C4CF4E06C1CEA11541DBF1CEA135505
:1007A80094EA0C0F95EA0C0F00F0A7F8A4EB0504E7
:1007B80081EA030E52EA03354FEA013100F08880DE
:1007C8004FEA03334FF0805545EA131343EA1263A7
:1007D8004FEA022245EA111545EA10654FEA00265C
:1007E8000EF000419D4208BF964244F1FD0404F515
:1007F800407402D25B084FEA3202B61A65EB030571
:100808005B084FEA32024FF480104FF4002CB6EB2D
:10081800020E75EB030E22BFB61A754640EA0C00AD
:100828005B084FEA3202B6EB020E75EB030E22BFED
:10083800B61A754640EA5C005B084FEA3202B6EB2E
:10084800020E75EB030E22BFB61A754640EA9C00ED
:100858005B084FEA3202B6EB020E75EB030E22BFBD
:10086800B61A754640EADC0055EA060E18D04FEA7B
:10087800051545EA16754FEA06164FEAC30343EA1B
:1008880052734FEAC2025FEA1C1CC0D111F4801FE8
:100898000BD141EA00014FF000004FF0004CB6E7E1
:1008A80011F4801F04BF01430020B4F1FD0C88BF80
:1008B800BCF5E06F3FF6AFAEB5EB030C04BFB6EB8B
:1008C800020C5FEA500C50F1000041EB045170BD7E
:1008D8000EF0004E4EEA113114EB5C04C2BFD4EBAB
:1008E8000C0541EA045170BD41F480114FF0000E2F
:1008F800013C90E645EA060E8DE60CEA135594EAAB
:100908000C0F08BF95EA0C0F3FF43BAF94EA0C0FAD
:100918000AD150EA01347FF434AF95EA0C0F7FF422
:1009280025AF104619462CE795EA0C0F06D152EA76
:1009380003353FF4FDAE1046194622E750EA41065A
:1009480018BF52EA43067FF4C5AE50EA41047FF46B
:100958000DAF52EA43057FF4EBAE12E74FF0FF3CD0
:1009680006E000BF4FF0010C02E000BF4FF0010CA1
:100978004DF804CD4FEA410C7FEA6C5C4FEA430C1A
:1009880018BF7FEA6C5C1BD001B050EA410C0CBF69
:1009980052EA430C91EA030F02BF90EA020F0020CB
:1009A800704710F1000F91EA030F58BF994208BF32
:1009B80090422CBFD8176FEAE37040F001007047EF
:1009C8004FEA410C7FEA6C5C02D150EA013C07D146
:1009D8004FEA430C7FEA6C5CD6D152EA033CD3D091
:1009E8005DF8040B704700BF8446104662468C468B
:1009F8001946634600E000BF01B5FFF7B7FF0028BE
:100A080048BF10F1000F01BD4DF808EDFFF7F4FFE6
:100A18000CBF012000205DF808FB00BF4DF808ED71
:100A2800FFF7EAFF34BF012000205DF808FB00BF94
:100A38004DF808EDFFF7E0FF94BF012000205DF8B6
:100A480008FB00BF4DF808EDFFF7CEFF94BF01206B
:100A580000205DF808FB00BF4DF808EDFFF7C4FF64
:100A680034BF012000205DF808FB00BF4FEA4102B7
:100A780012F5001215D211D56FF47873B3EB6252E8
:100A880012D94FEAC12343F0004343EA505311F00F
:100A9800004F23FA02F018BF404270474FF00000A1
:100AA800704750EA013005D111F0004008BF6FF0DF
:100AB800004070474FF00000704700BF4FEA410206
:100AC800B2F1E04324BFB3F5001CDCF1FE5C0DD9A4
:100AD80001F0004C4FEAC0024CEA5070B2F1004FEE
:100AE80040EB830008BF20F00100704711F0804FF1
:100AF80021D113F13872BCBF01F00040704741F4B6
:100B080080114FEA5252C2F11802C2F1200C10FAB9
:100B18000CF320FA02F018BF40F001004FEAC1239D
:100B28004FEAD32303FA0CFC40EA0C0023FA02F341
:100B38004FEA4303CCE77FEA625307D150EA013317
:100B48001EBF4FF0FE4040F44000704701F00040E7
:100B580040F0FE4040F40000704700BF80F00040C5
:100B680002E000BF81F0004142001FBF5FEA41037D
:100B780092EA030F7FEA226C7FEA236C6AD04FEA7D
:100B88001262D2EB1363C1BFD218414048404140C2
:100B9800B8BF5B42192B88BF704710F0004F40F474
:100BA800000020F07F4018BF404211F0004F41F490
:100BB800000121F07F4118BF494292EA030F3FD05C
:100BC800A2F1010241FA03FC10EB0C00C3F120036F
:100BD80001FA03F100F0004302D5494260EB4000FE
:100BE800B0F5000F13D3B0F1807F06D340084FEA69
:100BF800310102F10102FE2A51D2B1F1004F40EB5E
:100C0800C25008BF20F0010040EA030070474900C5
:100C180040EB0000013A28BFB0F5000FEDD2B0FA62
:100C280080FCACF1080CB2EB0C0200FA0CF0AABF85
:100C380000EBC25052421843BCBFD0401843704723
:100C480092F0000F81F4000106BF80F40000013229
:100C5800013BB5E74FEA41037FEA226C18BF7FEA00
:100C6800236C21D092EA030F04D092F0000F08BF42
:100C78000846704790EA010F1CBF0020704712F029
:100C88007F4F04D1400028BF40F00040704712F168
:100C980000723CBF00F50000704700F0004343F0CD
:100CA800FE4040F4000070477FEA226216BF084603
:100CB8007FEA23630146420206BF5FEA412390EAC6
:100CC800010F40F4800070474FF0000304E000BFBC
:100CD80010F0004348BF40425FEA000C08BF70476D
:100CE80043F0964301464FF000001CE050EA010231
:100CF80008BF70474FF000030AE000BF50EA010246
:100D080008BF704711F0004302D5404261EB410132
:100D18005FEA010C02BF84460146002043F0B64357
:100D280008BFA3F18053A3F50003BCFA8CF2083A7C
:100D3800A3EBC25310DB01FA02FC634400FA02FC85
:100D4800C2F12002BCF1004F20FA02F243EB02008C
:100D580008BF20F00100704702F1200201FA02FCEE
:100D6800C2F1200250EA4C0021FA02F243EB0200E1
:100D780008BF20EADC7070474FF0FF0C1CEAD05225
:100D88001EBF1CEAD15392EA0C0F93EA0C0F6FD0E6
:100D98001A4480EA010C400218BF5FEA41211ED0C4
:100DA8004FF0006343EA501043EA5111A0FB0131B0
:100DB8000CF00040B1F5000F3EBF490041EAD37185
:100DC8005B0040EA010062F17F02FD2A1DD8B3F101
:100DD800004F40EBC25008BF20F00100704790F070
:100DE800000F0CF0004C08BF49024CEA502040EAC2
:100DF80051207F3AC2BFD2F1FF0340EAC250704788
:100E080040F400004FF00003013A5DDC12F1190FC5
:100E1800DCBF00F000407047C2F10002410021FA37
:100E280002F1C2F1200200FA02FC5FEA310040F14F
:100E3800000053EA4C0308BF20EADC70704792F0C8
:100E4800000F00F0004C02BF400010F4000F013A00
:100E5800F9D040EA0C0093F0000F01F0004C02BFFB
:100E6800490011F4000F013BF9D041EA0C018FE76A
:100E78000CEAD15392EA0C0F18BF93EA0C0F0AD070
:100E880030F0004C18BF31F0004CD8D180EA010096
:100E980000F00040704790F0000F17BF90F0004F2F
:100EA800084691F0000F91F0004F14D092EA0C0F11
:100EB80001D142020FD193EA0C0F03D14B0218BFA4
:100EC800084608D180EA010000F0004040F0FE40EA
:100ED80040F40000704740F0FE4040F44000704786
:100EE8004FF0FF0C1CEAD0521EBF1CEAD15392EA05
:100EF8000C0F93EA0C0F69D0A2EB030280EA010CF5
:100F080049024FEA402037D04FF0805343EA11118D
:100F180043EA10130CF000408B4238BF5B0042F1EB
:100F28007D024FF4000C8B4224BF5B1A40EA0C0090
:100F3800B3EB510F24BFA3EB510340EA5C00B3EBC2
:100F4800910F24BFA3EB910340EA9C00B3EBD10FB0
:100F580024BFA3EBD10340EADC001B0118BF5FEA02
:100F68001C1CE0D1FD2A3FF650AF8B4240EBC2502B
:100F780008BF20F0010070470CF0004C4CEA5020EC
:100F88007F32C2BFD2F1FF0340EAC250704740F43B
:100F980000004FF00003013A37E792F0000F00F02D
:100FA800004C02BF400010F4000F013AF9D040EAAB
:100FB8000C0093F0000F01F0004C02BF490011F43F
:100FC800000F013BF9D041EA0C0195E70CEAD15337
:100FD80092EA0C0F08D142027FF47DAF93EA0C0F1E
:100FE8007FF470AF084676E793EA0C0F04D14B0202
:100FF8003FF44CAF08466EE730F0004C18BF31F0B4
:10100800004CCAD130F000427FF45CAF31F00043AD
:101018007FF43CAF5FE700BF4FF0FF3C06E000BF46
:101028004FF0010C02E000BF4FF0010C4DF804CD69
:101038004FEA40024FEA41037FEA226C18BF7FEA79
:10104800236C11D001B052EA530C18BF90EA010F7B
:1010580058BFB2EB030088BFC81738BF6FEAE1700A
:1010680018BF40F0010070477FEA226C02D15FEAA6
:10107800402C05D17FEA236CE4D15FEA412CE1D012
:101088005DF8040B704700BF844608466146FFE7D9
:101098000FB5FFF7C9FF002848BF10F1000F0FBDBB
:1010A8004DF808EDFFF7F4FF0CBF012000205DF8B4
:1010B80008FB00BF4DF808EDFFF7EAFF34BF012039
:1010C80000205DF808FB00BF4DF808EDFFF7E0FFD2
:1010D80094BF012000205DF808FB00BF4DF808ED23
:1010E800FFF7D2FF94BF012000205DF808FB00BF86
:1010F8004DF808EDFFF7C8FF34BF012000205DF868
:1011080008FB00BF4FEA40024FEA41037FEA226C26
:1011180002D15FEA402C08D17FEA236C02D15FEA52
:10112800412C02D14FF0000070474FF0010070478A
:101138004FEA4002B2F1FE4F0FD34FF09E03B3EBDC
:1011480012620DD94FEA002343F0004310F0004F1C
:1011580023FA02F018BF404270474FF00000704772
:1011680012F1610F01D1420205D110F0004008BF11
:101178006FF0004070474FF00000704742000ED2F9
:10118800B2F1FE4F0BD34FF09E03B3EB126209D4BA
:101198004FEA002343F0004323FA02F070474FF070
:1011A8000000704712F1610F01D1420202D14FF0E5
:1011B800FF3070474FF00000704700BF7BB972B92D
:1011C8000029BEBF00204FF0004106E008BF0028FC
:1011D8001CBF6FF000414FF0FF3000F077B8ADF161
:1011E800080C6DE904CE002909DB002B1ADB00F09E
:1011F800A9F8DDF804E0DDE9022304B070474042B5
:1012080061EB4101002B1BDB00F09CF8DDF804E0EA
:10121800DDE9022304B0404261EB4101524263EB35
:1012280043037047524263EB430300F08BF8DDF849
:1012380004E0DDE9022304B0404261EB410170475C
:10124800524263EB430300F07DF8DDF804E0DDE98A
:10125800022304B0524263EB4303704753B94AB9BF
:10126800002908BF00281CBF4FF0FF314FF0FF30A6
:1012780000F02CB8ADF1080C6DE904CE00F062F86E
:10128800DDF804E0DDE9022304B07047D0B5FFF7CC
:10129800FBF80C4B002206460F46FFF74DF900F00D
:1012A80017F80446FFF7CEF8074B0022FFF744F97A
:1012B80002460B4630463946FEF786FF00F008F82E
:1012C8002146D0BD0000F03D0000F041704700BF4E
:1012D8004A0011D212F5001211D20DD56FF47873AD
:1012E800B3EB62520ED44FEAC12343F0004343EA02
:1012F800505323FA02F070474FF00000704750EA4D
:10130800013002D14FF0FF3070474FF000007047B6
:1013180010F8012B11F8013B012A28BF9A42F7D097
:10132800D01A7047034611F8012B03F8012B002A45
:10133800F9D17047034613F8012B002AFBD1181A7C
:10134800013870472DE9F0478C468E46089E1546B1
:1013580004461946002B40F0D080724547D9B2FAAE
:1013680082F74FB1C7F120030EFA07FC20FA03F306
:10137800BD4043EA0C0CBC404FEA154EA8B2BCFB7A
:10138800FEF8230C0EFB18CC08FB00F943EA0C43CB
:10139800994528D9EB1808F1FF3204D2994502D9AA
:1013A800A8F102022B44A3EB0903A4B2B3FBFEFC91
:1013B8000EFB1C330CFB00F044EA0344A04214D992
:1013C8002C190CF1FF3304D2A04202D9ACF102036C
:1013D8002C44241A43EA02401EB1FC400023346026
:1013E8007360BDE8F0874246DDE76346F1E7002A0F
:1013F80079D0B2FA82F3002B3FD01946C1F120030D
:1014080002FA01F52EFA03F20EFA01FE20FA03F3AE
:1014180043EA0E034FEA154E00FA01F4B2FBFEFC54
:10142800AFB20EFB1C201A0C0CFB07F842EA004274
:1014380090455AD9AA180CF1FF3004D2904502D928
:10144800ACF102002A44A2EB08029BB2B2FBFEFCFC
:101458000EFB1C220CFB07F743EA02439F4246D9C6
:10146800EB180CF1FF3204D29F4202D9ACF1020210
:101478002B44DB1B42EA004202E0AEEB02030122EE
:101488004FEA154EAFB2B3FBFEFC200C0EFB1C332B
:101498000CFB07F840EA034398452AD9EB180CF1EE
:1014A800FF3004D2984502D9ACF102002B44A3EBDB
:1014B8000803A4B2B3FBFEFC0EFB1C330CFB07F7BE
:1014C80044EA0344A74216D92C190CF1FF3304D27D
:1014D800A74202D9ACF102032C44E41B43EA0040C2
:1014E8000F46114678E71F2188E76046ABE762465A
:1014F800BFE76046DBE76346EFE7734506D916B9F1
:10150800002108466DE7C6E9000EF9E7B3FA83F74C
:1015180087B9734501D3824207D8841A6EEB030357
:1015280001209C461EB900215BE73846FAE7C6E968
:10153800004CF8E7C7F1200CBB4022FA0CF51D431C
:1015480020FA0CF12EFA0CF30EFA07FE41EA0E010E
:101558004FEA154900FA07F4B3FBF9F81FFA85FEBC
:1015680009FB18300B0C08FB0EFA43EA00439A45B6
:1015780002FA07F240D9EB1808F1FF3004D29A4575
:1015880002D9A8F102002B44A3EB0A0389B2B3FBEA
:10159800F9F809FB183308FB0EFE41EA03418E45B2
:1015A8002CD9691808F1FF3304D28E4502D9A8F165
:1015B8000203294443EA0040A0FB0298A1EB0E0174
:1015C8004145CE46434602D306D14C4504D2B9EB39
:1015D800020E68EB05030138002EA4D0B4EB0E020E
:1015E80061EB030101FA0CFC22FA07F34CEA03034E
:1015F800F940C6E9003196E74046C5E74346D9E7D2
:101608002DE9F04390F8A53085B004460D4623B97E
:101618004FF07E50FFF7A6FA0546D4F884202E4BEB
:101628009A4212D12846FEF72FFF29A3D3E90023B7
:10163800FFF712FA011E04F1840018BF012113F00C
:1016480065F80120C4F8985005E0B4F89C30B3F56B
:10165800807F03D1002005B0BDE8F08304F1500974
:1016680048462DF04DFE0028F4D01C492846FFF7C7
:1016780083FB94F89C60FFF781FD94F88080C3B2E7
:10168800276E206DB8F1000F0DD08DF80D300223B4
:1016980001220021009303AB8DF80C60B84748463F
:1016A8004BF068F8CDE78DF80B60012641468DF8C0
:1016B8000C3032460DF10B030096B847009603AB89
:1016C800276E42463146206DE8E700BFAFF3008041
:1016D800AE47E17A14AEEF3F70AE050800007F43D5
:1016E8002DE9F04F044685B0084690466160062112
:1016F8001D469DF838709DF83CB017F04BFCA06073
:10170800067C16F0010602D07D481BF015FD9DF8F9
:10171800403005FB08F00DF1080A277384F82A30D9
:101728007D309DF8443084F828307E2390FBF3F018
:10173800C0010430C4E90485606245F0EEFE06226B
:101748007049A661C4E9070620464EF05AF90222FC
:1017580051462046ADF808804EF053F90222514612
:101768002046ADF808504EF04CF9F623032269469E
:101778002046ADF800308DF802604EF042F97B1E2D
:10178800DBB2082B05D840F25515DD4015F00105F0
:1017980001D15D48B9E7052F09D0072F06D0032FDF
:1017A80073D1012384F82930002502E02E4684F8FD
:1017B8002960002646F34F10C0EB0020FEF752FECA
:1017C8000022524BFEF702FD0022514BFEF7DEFFCE
:1017D800FFF74CF95FFA80F8C6F38200C0EB0020EF
:1017E800FEF740FE00224B4BFEF7F0FC00224A4B6E
:1017F800FEF7CCFFFFF73AF9C7B206F00300C0EBDB
:101808000020FEF72FFE0022404BFEF7DFFC0022EF
:101818003F4BFEF7BBFFFFF729F9C0B2002D5ED0A2
:101828008DF808008DF809808DF80A7001360322BA
:10183800514620464EF0E5F8802EBBD1BBF1000F93
:101848001AD0364D01A920462A88AB78ADF8042075
:1018580003228B704EF0D5F80B22314920464EF00A
:10186800D0F8D5F80300EB790522029051462046BE
:101878008AF804304EF0C5F820464EF0B0F8A0695A
:101888004EF0D1F805B0BDE8F08F092F84F8296033
:101898008AD135460FF25809D9E9008916A7D7E940
:1018A80000672846FF35FEF7DDFD42464B46FEF74A
:1018B8008DFC32463B46FEF769FFFFF7D7F8032257
:1018C800C0B251468DF808008DF809008DF80A005D
:1018D80020464EF096F8B5F5FF4FE2D1AEE78DF809
:1018E80008808DF809708DF80A009FE7AFF3008033
:1018F8000000000000C04F400000000000C05F4032
:10190800CB560608853F0608285106080000F83F10
:101918000000084000000C4000001C409326050809
:101928008C3F06080000000030F000422DE9F84F17
:101938000146034604D1BDE8F84F012037F0E8BF5F
:10194800002803DABDE8F84F37F0EABFB0F1FF4FDF
:1019580003DBFFF709F9BDE8F88FB0F5000F35DABA
:101968004FF09841FFF708FA6FF018020346C3F3E7
:101978001604DE15764B234403F400007F3E80F006
:101988007E5016444FF07E51204306EBD356FFF7A6
:10199800E9F8704B04F10F0213400546002B3ED1C5
:1019A8000021FFF77DFB98B1002E00F0C88030467B
:1019B800FFF78EF968490546FFF7DEF967490446DF
:1019C8002846FFF7D9F901462046C2E70022CEE7AC
:1019D8005DA1D1E90001FFF771F82946FFF7CCF9BD
:1019E80001464FF07C50FFF7BDF8294604462846CB
:1019F800FFF7C2F901462046FFF7BEF904460EB9C3
:101A080021466FE03046FFF763F953490746FFF771
:101A1800B3F9524906463846FFF7AEF972E04FF07F
:101A28008041FFF7A1F801462846FFF759FA814699
:101A38003046FFF74DF9494680464846FFF79CF97E
:101A480001468246FFF798F94549DFF818B107467D
:101A5800FFF792F94449FFF787F83946FFF78CF901
:101A68004249FFF781F83946FFF786F94049FFF701
:101A78007BF85146FFF780F93E4982463846FFF722
:101A88007BF93D49FFF770F83946FFF775F93B498F
:101A9800FFF76AF83946FFF76FF901465046FFF736
:101AA80063F8C4F55713A34403F5227343EA0B0301
:101AB800002B074630DD4FF07C512846FFF75CF9D4
:101AC8002946FFF759F9014604463846FFF74CF80E
:101AD8004946FFF751F9074646B901462046FFF740
:101AE80041F801462846FFF73DF834E71A494046D1
:101AF800FFF742F9194906464046FFF73DF93946CE
:101B0800FFF732F801462046FFF72CF82946FFF781
:101B180029F801463046E6E701462846FFF722F84D
:101B28004946FFF729F90446002E3FF469AF0A49F0
:101B38004046FFF721F90949064640466CE7002070
:101B480009E700BFAFF30080555555555555D53FAA
:101B580020FB4A00F0FF7F008071313FD1F7173733
:101B68009788173E305CCFFF25333A3E2549923E91
:101B7800ABAA2A3F4FD01C3E298E633ECDCCCC3E2B
:101B88002DE9F04F31F0004387B081460E460746F5
:101B98000C460DD180F480077F0017F5000F40F246
:101BA800528331464846FEF7DFFF07B0BDE8F08FA5
:101BB80020F00048B8F1FF4F014602D8B3F1FF4FBB
:101BC80008D9B7F17E5FECD184F48004640014F581
:101BD800000FE4E7002823DAB3F1974F80F0388349
:101BE800B3F17E5F36D3DA15C2F1960243FA02F5F5
:101BF80005FA02F29A4225D105F00105C5F1020560
:101C0800B3F17E5F27D1002C7EDA00214846FFF72A
:101C180047FAC8B1F80F07B0BDE8F04F37F078BE03
:101C2800B3F1FF4F0ED1B8F17E5F00F00C8304D9F9
:101C3800002C80F20B830020B7E7002CFBDA06F1BA
:101C48000040B2E70025DBE749464FF07E50FFF73A
:101C580047F9AAE70025B4F1804F424640F0FE82DA
:101C6800B8F1BF4F20D2B8F1D05F04D949464846F1
:101C7800FFF782F899E729F00040B8F1000F40D04B
:101C8800F90F01390391294324D0B3F19A4F40F257
:101C9800D780654B984539D8002C3CDA002007B02E
:101CA800BDE8F04F37F02CBE27F0404CBCF17E5F0A
:101CB80029F000401AD1002C04DA01464FF07E507A
:101CC800FFF70EF9002FBFF670AFA8F17E5858EA5B
:101CD800050805D1484607B0BDE8F04F37F020BEEB
:101CE800012D7FF462AF00F100405EE7B8F1000F0C
:101CF800C6D1002C05DA17B16B1E59425941084666
:101D080089E7012D7FF451AF48464EE7474B984588
:101D180007D9002CC2DC002007B0BDE8F04F50F016
:101D2800DFB84FF07E51FEF71DFF41490746FFF728
:101D380023F8404981463846FFF71EF8804638A107
:101D4800D1E90001FEF7BAFE4FF07A5182463846D3
:101D5800FFF712F801465046FEF704FF3946FFF731
:101D68000BF801464FF07C50FEF7FCFE39468246E0
:101D78003846FFF701F801465046FEF7FDFF2E49A9
:101D8800FEF7FAFF01464046FEF7ECFE01468046A4
:101D98004846FEF7E9FE20F47F6727F00F0749461B
:101DA8003846FEF7DFFE01464046FEF7DBFE039BA2
:101DB800013D6FF30B041D438046214630460CBF9E
:101DC8001E4D4FF07E55FEF7CDFE3946FEF7D4FF87
:101DD800314681464046FEF7CFFF01464846FEF7AA
:101DE800C3FE214606463846FEF7C6FF01460746AB
:101DF8003046FEF7B9FE00280446804620F000432E
:101E080040F34481B3F1864F40F22D8100212846EA
:101E1800FFF750F9003818BF012040E7AFF3008002
:101E2800E13D55555555D53FF3FF7F3F0700803FAE
:101E380000AAB83F70A5EC363BAAB83F000080BFA7
:101E480017F0FF4F40F00B814FF09741FEF794FFDA
:101E58006FF017010246D3157F3B0B449649029356
:101E6800C2F316028A4242F07E5308DD93498A4241
:101E780040F3F780029A01320292A3F5000300278B
:101E88008F4A049352F827B0184659469A46FEF7E7
:101E980069FE514681465846FEF766FE01464FF0F8
:101EA8007E50FFF71DF8014605904846FEF764FF8F
:101EB8000190019B83496FF30B039846049B01EA49
:101EC800630343F0005303F5800303EB4753414694
:101ED80018460493FEF750FF01464846FEF742FEB7
:101EE800049B814659461846FEF73CFE014650467B
:101EF800FEF738FE4146FEF73FFF01464846FEF72B
:101F080031FE059A1146FEF737FF019983460846C8
:101F1800FEF732FF6C498146FEF72EFF6B49FEF74C
:101F280023FE4946FEF728FF6949FEF71DFE49468C
:101F3800FEF722FF6749FEF717FE4946FEF71CFF2A
:101F48006549FEF711FE4946FEF716FF6349FEF79D
:101F58000BFE494682464846FEF70EFF01465046AC
:101F6800FEF70AFF414681460198FEF7FDFD5946F6
:101F7800FEF702FF4946FEF7F7FD41468246404616
:101F8800FEF7FAFE56490490FEF7EEFD5146FEF7BD
:101F9800EBFD20F47F6929F00F0941464846FEF71A
:101FA800EBFE4F4980464846FEF7DCFD0499FEF7F4
:101FB800D9FD01465046FEF7D5FD0199FEF7DCFE36
:101FC800494682465846FEF7D7FE01465046FEF778
:101FD800CBFD834601464046FEF7C6FD20F47F69E7
:101FE80029F00F093F494846FEF7C6FE414682469A
:101FF8004846FEF7B7FD01465846FEF7B3FD3A4995
:10200800FEF7BAFE394980464846FEF7B5FE014656
:102018004046FEF7A9FD364B53F82710FEF7A4FDFE
:1020280080460298FEF754FE324B53F827B081469B
:1020380041465046FEF798FD5946FEF795FD49463C
:10204800FEF792FD20F47F6727F00F0749463846D0
:10205800FEF788FD5946FEF785FD5146A1E60021A9
:10206800F9E601270CE74BD123493046FEF77CFD02
:10207800394681462046FEF775FD01464846FFF77A
:1020880037F800287FF4C2AE86233EE01B4A93420D
:1020980007D900212846FFF70DF8003818BF01209E
:1020A8003AE62DD13946FEF75DFD3146FFF716F8C1
:1020B8000028E9D0EDE700BF71C41C00D6B35D006D
:1020C800B0D2050800F0FFDF42F1533E55326C3EB6
:1020D80005A38B3EABAAAA3EB76DDB3E9A99193F82
:1020E800000040400040763F4F38763FC623F6B8A0
:1020F800A0D20508A8D205083CAA38330000164328
:10210800B3F17C5F40F29B80DB157E3B4FF400040B
:102118001C414444C4F3C75357497F3B19412140EC
:10212800C4F31604C3F1170344F400041C41B8F1C6
:10213800000F3846B8BF6442FEF714FD0746314623
:102148003846FEF711FD20F47F6929F00F094B4945
:102158004846FEF711FE394680464846FEF702FD1E
:1021680001463046FEF7FEFC4549FEF705FE4549A7
:1021780006464846FEF700FE01463046FEF7F4FCE8
:10218800074601464046FEF7EFFC41460646FEF785
:10219800E9FC01463846FEF7E5FC31468046304604
:1021A800FEF7EAFD38490746FEF7E6FD3749FEF730
:1021B800D9FC3946FEF7E0FD3549FEF7D5FC39462E
:1021C800FEF7DAFD3349FEF7CDFC3946FEF7D4FDBC
:1021D8003149FEF7C9FC3946FEF7CEFD01463046C7
:1021E800FEF7C0FC074601463046FEF7C5FD4FF036
:1021F800804181463846FEF7B5FC01464846FEF761
:102208006FFE414607463046FEF7B6FD4146FEF7EB
:10221800ABFC01463846FEF7A5FC3146FEF7A2FCAA
:1022280001464FF07E50FEF79DFC00EBC453B3F51A
:10223800000F06DA214637F005FB294618E5002489
:102248007DE71846F9E74FF07E50AEE43046ACE43F
:10225800B3F1FF4F3FF4E7AC42460225B4F17C5F8F
:102268007FF422AD002FFFF61FAD484607B0BDE84A
:10227800F04F4FF0D6BD00BF000080FF0072313F25
:102288001872313F8CBEBF354CBB31330EEADD3599
:1022980055B38A38610B363BABAA2A3E2DE9F84F75
:1022A8000B1F884602F00701D408A3EB000903F0CE
:1022B80007030B3100AF4FEAD90629F007090B4491
:1022C8000546814404EBD3048368B9F802B09C4204
:1022D80028BF1C461BF0010B16D1EA4688B06A4697
:1022E8004A4BCDE90538032342F8103F4FF4C25159
:1022F8005B46474800F0C4FFD5468BF31188BFF30F
:102308006F8F0423184602DF3146284637F0C1FF95
:10231800304435F83030C01A864217D0EA4688B0C3
:102328006A463C4BCDE90538032342F8103F0023A9
:102338004FF4C251364800F0A3FF0023D54683F37B
:102348001188BFF36F8F0423184602DF31462846F1
:1023580037F09FFF8442824622D026D23444284652
:10236800224638F03BF8B9F802302146284643F0B7
:102378000103A9F8023037F08CFF261805EBC603D5
:102388005B88DB0708D43146284637F0CBFF324656
:102398002146284638F00BF82146284637F07EFFBC
:1023A80001221046BD46BDE8F88F06EB000805EB94
:1023B800C802528812F0010225D14146284637F05A
:1023C80068FF50448442ECD82846A4EB0A0A37F048
:1023D800A9FF4146284637F05CFF824507D23219EB
:1023E800284637F0FBFF2846114637F057FF42468C
:1023F8003146284637F0DBFFB9F8023043F00103D5
:10240800A9F80230CCE70022CBE700BFA0DC050822
:10241800C8250508C4DC05082DE9F84F8A4600AF31
:10242800002974D004680E1F361BF50826F007062D
:1024380004EB0608B8F802B01BF0010B16D1E94608
:1024480088B06A46334BCDE90531032342F8103F83
:102458004FF4C2515B46304800F012FFCD468BF373
:102468001188BFF36F8F0423184602DF29462046E0
:1024780037F00FFF284434F83030C01A854217D09F
:10248800E94688B06A46254BCDE9053A032342F868
:10249800103F00234FF4C2511F4800F0F1FE002303
:1024A800CD4683F31188BFF36F8F0423184602DFEC
:1024B800B8F802302946204623F00103A8F8023074
:1024C80037F0E7FE05EB000804EBC8035B88DA0782
:1024D80008D44146204637F025FF42462946204683
:1024E80037F065FFA65BAE1B04EBC6035B88DB0712
:1024F80009D43146204637F015FF2A46354631467D
:10250800204637F054FF2946204637F0C7FEBD461F
:10251800BDE8F88FEDDC0508C8250508C4DC05080A
:10252800024808B538F0EEF8002008BD1ADD0508A5
:102538002DE9F04F91B0840705460E46009302F04E
:102548000403DDF868A00293C2F3C203039203F107
:102558000103059340F09D81041D002849D101F035
:102568000706341DC6F10806009B00274FF0040833
:102578005A1E4FF0FF33B946BB46019343460497B2
:102588000DB1009921600598002800F3D680904885
:102598000099814203D38F488142C0F0CE800399CD
:1025A800601B11F0020C40F0D680B9F10F0F00F259
:1025B800CF80002D00F0D68009F14001C0F38700DC
:1025C8000DEB010E01990EF8200C0EF8101CBCF151
:1025D800000F00F0C38060F07F0001370EF8200C78
:1025E80009F10109C5F1080104344FF6DA7E0691B4
:1025F8008CE00729B8D86FF01B0011B0BDE8F08F48
:102608007A285BD84B280FD8472857D829282ED89E
:10261800252850D052D8202818BF23280CBF4FF0A7
:10262800010B4FF0000B71E04C382E2846D8DFE83C
:1026380000F06D45454545454545454545454845B1
:1026480045454545454545564548485656566D48BD
:102658006A456D4518481845457F7C4845454845B5
:102668007C0000204FF0000B4FF0040835E02A38BA
:102678000121C0B201FA00F010EA0E0F46D110F0A5
:10268800625C2CD110EA010B40D06046013C444406
:10269800B4FBF8F408FB04F425B1A3EB050CA4443F
:1026A800B445A8D8002870D00599013905915AF881
:1026B800041B009164E70199013901914FF0000B67
:1026C80024E012F8010C6C2834D112F8023C0020E6
:1026D8006C2B8346C8D14FF008084346D6E70AF169
:1026E800070A07342AF0070A24F00704FAE802BCAC
:1026F80035B106982044B0423FF67DAFC4E900BC2E
:1027080008344FF0000B4FF00808434612F8010F49
:10271800002853D0BBF1000F7FF472AF2528F5D104
:10272800019B4FF0010B013301934FF00408ECE7D4
:10273800584697E700208346A8E7039988077FF55E
:1027480051AF601B4FF0010CB0F5007FFFF42DAFC7
:102758006FF0150051E74FF0000CF5E704980130D1
:1027680004903DE7BCF1000F01D0013638E702982C
:10277800023600287FF434AF0098CDE90632FEF720
:10278800D9FD0644DDE906322AE7042B08D10AF10F
:10279800040015B1DAF80010216004348246B5E768
:1027A8000AF1070323F0070303F1080A1DB1D3E96F
:1027B8000001C4E9000108340823A7E7631BB3F547
:1027C800806FC5D245B9A6F10804E01815E700BF27
:1027D8000C1F05088C6B06089B08029A28602B7052
:1027E8009DF81030AAB1EB70AF702FB108A8002285
:1027F800C5F1010C91450ED1C5F101030DF1200879
:102808004FF0000A0DF1300B0193D14512D1601B36
:10281800F3E66B70E8E710F8013B190608D50CEBF6
:10282800040E03F07F03B6453FF6E5AE04F8013B1E
:102838000132DFE71FB198F90020002A17DB029B5D
:10284800D3B11AF80B2004F8012B0022019B1819A8
:102858001044B0423FF6CFAE98F80000009904F853
:10286800010B204603924FF0F9F9039A14440AF138
:10287800010A08F10108C8E798F8002055F8223045
:102888000093029B009845F82230FEF753FD421C46
:10289800DCE76FF00D00B0E62DE9F04F97B0054684
:1028A8008A4600AFC7E90A3249B903784678807882
:1028B80000EB83002844564524D8A0EB050AD7F836
:1028C800803095F8028003F00103D7F88040FB615F
:1028D800B8F1000F0CBF002404F00104EB787B6210
:1028E8001BB1D7F880309A0715D4A4B9FB6A1BB17D
:1028F800BA6A514628469847564630465C37BD4620
:10290800BDE8F08F441C0AF1010A2046FEF712FDCB
:1029180001302044CFE7D7F88030C3F3C0033B62CF
:102928002B78BB619B003B616B687B61BB6905EBE6
:10293800830BFB6A002B77D15646D844BCB11C46A2
:102948001BF8013B55F82300FEF7F4FCD7F8843058
:10295800013043B1D7F88830A34282BFD7F884301A
:1029680023F814000134C3450644E9D1D846D7F802
:1029780080304FF0000913F0050F0CBF4FF0020B29
:102988004FF0010B7B6A9945B7D298F8013008F1EE
:10299800020855F823A0AD4B9A45C0F04B81AC4BCB
:1029A8003A6A9A452CBF002301230AB318F8021C7F
:1029B8007869FB6237F087FEFB6AC8B1EA468AB0DD
:1029C8006A46A44B05937B69CDE906314FF4007341
:1029D800ADF82030A04B42F8103F00234FF41251BD
:1029E8009E48023E00F04CFCD54609F10109C9E7B2
:1029F80023B1FB6933B9A6EB0B06F6E7D7F88030AD
:102A08009B07F2D55046FEF795FCD7F884304BB1BA
:102A1800D7F888309C423FBF431CD7F8842022F85F
:102A2800143001340644E0E7002C69D1B8F1000FF6
:102A38006CD0D7F8803058076BD5C14607F14800ED
:102A4800424659464FF00AF90BEB08030022FB6097
:102A58000233796A8A425ED3D7F8802095F801B0AC
:102A68009207F96904EB0B0354BF4FEA590200229D
:102A7800DBB2002940F0A680D7F8801011F0040FCF
:102A880014BF494600216B702846A970EA7039695D
:102A9800BA6AFB6A9847061EFFF62FAFBB6949461C
:102AA800BA6A07F148002B707B6A85F801B0EB70B1
:102AB80085F80280FB6A9847B0F10009C0F2B68039
:102AC8003B697A6A786A03EB4201FB68BA6A414457
:102AD80003EB4000FB6AAAEB010198470028C0F20B
:102AE800A780B1444FF0000B07F1380A09EB000644
:102AF800A34569D30021BA6AFB6A08469847FCE6F1
:102B0800444607F138004FF0000999E74446C146AA
:102B18009AE7A14698E713F8016CDFF830C155F839
:102B2800260013F8021C6045C0F08A80DFF820C137
:102B38006045386A2CBF4FF0000B4FF0010B38B1DD
:102B48007869C7E9013237F0BEFDD7E90132F0B93B
:102B5800BBF1000F1ED0F96949B1611C04F12800CE
:102B680007F13004041904F8206CCCB20FE0D7F850
:102B7800801049070BD509F1280007F1300C09F13D
:102B8800010100EB0C0909F8106C5FFA81F90132B8
:102B980002335EE7D7F880008007DED409F1280CFD
:102BA80007F1300E09F1010009F10209F4445FFA56
:102BB80089F90CF8101C07F1580151FA80F000F857
:102BC800106CE4E700215EE71BF80A3055F8239003
:102BD80087F83730D7F884302BB3D7F888309B453F
:102BE80021D2D7F8843033F81B80BA6A012107F163
:102BF8003700FB6A984700281ADB0644B8F1000F33
:102C080006D14846FEF796FB00F101081FFA88F83E
:102C1800BA6A41464846FB6A9847002808DB0644DA
:102C28000BF1010B64E74FF00008DEE74E4664E65F
:102C3800064662E63B6A002B3FF4E0AE0023B5E6A9
:102C4800386A0028A6D04FF0000B79E70C1F05085A
:102C58008C6B060848DD05080400000120250508DE
:102C6800014B1860704700BF80010024044608B576
:102C7800EFF31183102383F31288BFF36F8F01F0F2
:102C880061FB01F0C9FB3BF03CFA204601F0C8F9B2
:102C9800024837F037FD38F01AFBFCE7FCDD050881
:102CA800054B00205A6822F002025A605A6822F046
:102CB80001025A60704700BF0010005C08B5416807
:102CC80005480C3183681B681BB1984700EAE0701F
:102CD80008BD6FF05700F9E74C2005080A2810B521
:102CE80002D90024204610BD044B53F8204020464A
:102CF8003CF084FD0028F5D1F3E700BF80270508E4
:102D080008B501F06FFB01F0EFFA0C4B0C4A1A60A2
:102D18000C4AD36823F03F0343F00403D3600A4B03
:102D28001A6841F20303B3EB124F06D1074AD2F8EF
:102D3800083143F00103C2F8083108BDF80800243F
:102D48000090D003004802580010005C0080005139
:102D58002DE9F047044607464FF00109DFF84C809B
:102D680094FAA4F5B5FA85F509FA05F32E0108EBEE
:102D780005156FEA030A24EA03042B7B63B158F8AC
:102D880006301B696BB946440222284607EA0A073F
:102D98007368196838F06BF8002CE1D13846BDE843
:102DA800F087284698470028F6D1ECE778260508EA
:102DB80010B5002288B00E490E483DF0A2F9002255
:102DC800002300240C490D480094CDE906230E2366
:102DD8004FF44072CDE90334CDE90144084B0DF0BE
:102DE800F9FB084905483CF09DFF204608B010BD96
:102DF800112E0008282800240048002480230024DD
:102E080031310008F0DE050801480DF0E9B800BFCF
:102E1800281200242DE9F047804620480F4637F055
:102E2800FEFF0646002832D000252846BDE8F08778
:102E3800237B83B12368DB680BB12046984763681E
:102E480083F8069023681B69CBB963680222204681
:102E5800196838F00CF8013610345445E8D3B8F145
:102E6800000FE2D0002DDFD02846FFF771FF05469E
:102E7800002FF7D0002164203DF057F8F2E72046F4
:102E880098470028E1D009FA06F31D43E3E7044C0C
:102E98000546DFF810A04FF00109DEE75835002499
:102EA8007826050888260508014B53F82000704746
:102EB800EC27050808B5034608462BB1044A1360F9
:102EC80000F050FC002008BD6FF01500FBE700BFC4
:102ED8008401002410B5044C237813B903480DF07D
:102EE8007FF80123237010BD064400242812002413
:102EF80010B504460B4837F092FF5CB10A4BBFF39C
:102F08005B8F53E8001F013943E80012002AF8D10B
:102F1800BFF35B8F05480EF03BF90548BDE810404C
:102F28000DF05EB8503500245435002428280024BC
:102F380028120024064B0022BFF35B8F53E8000FD2
:102F480043E800210029F9D1BFF35B8F704700BF28
:102F58005035002470B5FFF7EDFF084C0546084EC4
:102F6800B44200D370BD63685B792BB123685B689A
:102F780013B12946204698471034F1E7782605080A
:102F88008826050810B5044C0449204637F0C6FCCD
:102F9800034B1C6010BD00BF40110024D827050852
:102FA8004835002400230D4A4FF47A710C4810B5B7
:102FB80013700C4A13600C4A1360FFF77BFFFFF78E
:102FC800E1FF0A4B0A4918468B4200D310BD1A1A72
:102FD8005C681033121101322271F5E707440024AE
:102FE80041AE0308503500245435002478260508DE
:102FF80088260508014600220023014837F0AFBCA7
:1030080040110024014837F046BD00BF401100249C
:10301800024B0146186837F099BD00BF48350024B7
:10302800014837F0CEBD00BF40110024274B70B5D2
:103038001B78002B47D0FFF7E5FF044600283FD157
:10304800234B244D1B68002B12DD3DF012F80A2299
:103058000023FEF703F9D5E90032C01A40F2E9333C
:1030680061EB0201984271F1000101D3FFF772FF91
:10307800D5E9003213F57A7342F10002C5E900324E
:103088000CB3BDE87040FFF7CBBF6B685B7923B129
:103098002B68214628461B6898471035B542F4D35B
:1030A8002046FFF7B5FF0C4BBFF35B8F53E8001FBB
:1030B800013943E80012002AF8D1BFF35B8FBFE75C
:1030C800064D074EEAE7002070BD00BF0644002405
:1030D800503500242028002454350024782605087B
:1030E8008826050870B50D4D297861B90C4C01206A
:1030F8000C4EFFF78FFEB44206D3FFF797FF002868
:10310800FBD101232B7070BD63685B791BB1236809
:1031180020469B6898471034EDE700BF0744002419
:10312800782605088826050800212DE9F843084671
:10313800FFF770FE044648B34FF4FA784FF00009E1
:103148001B4B01F0CBF81B4A1B58136033B11A4BC9
:103158001B68092B02DD19480CF042FF0025184FA7
:1031680044B12046FFF7F4FD044618B94FF0FF3884
:103178004FF0FF39FFF75AFF064628B9B5B90F488F
:1031880042464B460CF068FF3546E9E74FF0FF38FA
:103198004FF0FF39D4E72B689B691BB10022284602
:1031A800114698471035BD42F5D3E8E7054DFAE7D3
:1031B800080000004C35002454350024281200244F
:1031C800882605087826050813B5184837F027FE1D
:1031D800174B1B7873B1EFF31184102383F3128814
:1031E800BFF36F8FFFF722FF84F31188BFF36F8F50
:1031F80002B010BD0F4B1B68002BF9D050B900224C
:1032080000230D48CDE9002342F2107200230DF08F
:1032180097FFEDE70928EBD107480DF0B9FF0748FC
:1032280002B0BDE810400CF0DBBE00BF54350024EE
:10323800074400244C3500242828002428120024A0
:10324800064B10B504461B6898472146A060044801
:1032580037F002FCBDE81040FFF7B6BF8401002438
:1032680040110024044A054B9B1AB1EBD30F34BF1D
:1032780052F83100002070471825050878260508FF
:103288002DE9F04F8FB0C1F34A260D46904604AFA2
:103298000C0DB8607B60002E61D04FF000090A2346
:1032A8004FF0040B07F1140AFE604A46C7F8249051
:1032B8004046C7E90799009307F11C03CDF808B009
:1032C800CDF804A0F968FFF7E7FAB0F5006F0346F8
:1032D8001CD36C468AB0D8F8041004AB24481A46AC
:1032E800C3E9050140F2FF71D9614FF400711984F7
:1032F800204B42F8103F4FF412514B461E48FFF73F
:10330800BFFFA5462C37BD46BDE8F08FC0F30A06BF
:1033180004F117003B60184466F3532520F00700BA
:103328008008FFF767FE044680B13B6800F1100192
:10333800124A4046F961C7E908390A23009307F1A0
:103348001C03CDE901ABF968FFF7A6FA66F353252C
:103358007B68B96820462A4637F0A9FDD2E704F110
:10336800170020F007008008FFF744FE0446EDE749
:1033780001DF0508040000018025050889AE03085F
:103388002DE9F04F87B00546884614469946DDE991
:10339800127ADDE9106BBFB110213B465A46002076
:1033A800CDF800A0CDF814A0FFF7C2F8B0F5006F73
:1033B80001460BD340F2FF73184A0221184807B0A0
:1033C800BDE8F04F37F0CCBD3946384604F0070366
:1033D80005F00704E40044EA831444EA402444EA7C
:1033E800065406F117000391084420F007008008EE
:1033F800FFF700FE054640B13FB13B465A460399E8
:103408001030CDF800A0FFF793F84B46224641460E
:10341800284607B0BDE8F04F37F049BD40DF050842
:1034280080250508406820B1034BC01A40F3CF003F
:1034380070474FF0FF307047182505080EB403B5E4
:1034480003AB0146054853F8042B019301F07AF9C0
:1034580002B05DF804EB03B0704700BFCBAF0308C0
:10346800CA0605D48B064CBF02490349FFF7E6BFDD
:10347800704700BF020C06088E0506082DE9F04FBC
:103488008BB0994604460D46179B9DF858800793C4
:103498001A9F0692DDE918A30593B8F1000F00F012
:1034A800BF80844B07F0020B13F80830089307F429
:1034B8008073099337F0D9FC024600287DD07E49F5
:1034C8002046FFF7BBFF0646BBF1000F08D017F0F8
:1034D800440F74D12A4679492046FFF7AFFF0644C6
:1034E80007F0010353B1764B2046764953F828205C
:1034F800754B002A08BF1A46FFF7A0FF07F4807330
:10350800002B07F0080318BF4FF00009002B00F04C
:1035180082806E4B20466E4953F82820FFF78EFFB5
:103528000546069B2BB11A466A492046FFF786FFD7
:103538000544B9F1000F0DD0089B002B6ED06649E9
:10354800664BB8F1040F18BF19464A462046FFF7E4
:1035580075FF054435446248079B1BB12246614903
:1035680037F080F8059B002B00F09080DDF8149070
:10357800002639462046B9F1100F28BF4FF0100930
:10358800FFF76EFFB54252DC002633461AF80320D7
:1035980020465549FFF752FF0136102E4DD07107CE
:1035A80003D152492046FFF749FF4E453346EDD334
:1035B8004F492046FFF742FFEEE7064684E74D4BAA
:1035C800186800288BD04C4B4FF47A7B4FF03C0C9A
:1035D8001B68B5FBF3F5B5FBF0F100FB11554FF493
:1035E80061630BFB05F5B1FBF3F2B5FBF0FE03FBE2
:1035F800121100FB1E55B1FBFCF30BFB05F50CFB90
:103608001311B5FBF0F5009120463C49CDE901E5E1
:10361800FFF714FF63E707F0080582E72F4994E7EF
:10362800B9F1010F45460CBF2D48354894E72F499D
:1036380020460136FFF702FFA4E70026314920465D
:10364800FFF7FCFE33461AF8032020462E49A2F164
:1036580020035F2B28BF2E22FFF7F0FE0136102E25
:103668000DD0720703D121492046FFF7E7FEB14587
:103678003346E8D81D492046FFF7E0FEEEE7059BF4
:10368800CA44B3EB090305937FF470AFB8F1000F98
:103698000AD0FB0704D50C4A20460A49FFF7CEFE9C
:1036A80039462046FFF7DCFE20460BB0BDE8F04F58
:1036B80037F07ABCE83F060886DF05088ADF050888
:1036C800FC270508DF0B060878DF05081028050821
:1036D800AFDF0508B5DF05087DDF050881DF0508D0
:1036E800CBAF03084D470008B9DF0508C33D0608FE
:1036F800C13D0608603500245C35002493DF0508C9
:1037080001B00308BFDF0508190C060842F20F7361
:10371800114A8B4273B5044628BF0B46056805213C
:10372800684634F045FC636806460B2228465B6809
:103738000A4937F02BFC63683246694628465B68BD
:1037480037F024FC63681B2205495B68284637F07C
:103758001DFC02B070BD00BFD4F10508DC3F0608AF
:10376800C03F060800210123064A904206D8064AAF
:1037780001B901231360054B186070474008012107
:103788005B00F2E740420F005C35002460350024FE
:10379800F8B50D4604464618054FB44201D12846EF
:1037A800F8BD14F8011BBB6801485B689847F4E74B
:1037B8007C220508014B0360032070475828050840
:1037C8000B4B2DE9F3421B6805460E460024094FB2
:1037D8004FF014090193019BA34202DC02B0BDE83B
:1037E800F0823868314609FB04000134A847F2E743
:1037F8008828050890010024104B70B51C680D46F8
:10380800B4B10F4B196800238B4202DB6FF0010043
:1038180070BD224612F8146B864202D0013314465A
:10382800F2E7E0683BF0EAFF28B100202C60EFE700
:103838006FF00C00ECE76FF01200E9E7900100244C
:103848008828050810B588B043680C460293836839
:10385800C068CDE903320A68002306490593CDE91B
:10386800062301AA39F086FD079808B9059B23604D
:1038780008B010BD9FB103082DE9F8430646FDF7CF
:1038880059FD0546EFF31188102383F31288BFF31F
:103898006F8F114B1C68D3F804909C4208BF00241A
:1038A80034B988F31188BFF36F8F2046BDE8F883D9
:1038B800A7683846FDF73EFDA84206D12A46394694
:1038C80030464EF017FA0028EBD04C4501D024685A
:1038D800E6E70024E5E700BF940100242DE9F04164
:1038E8000E461546FFF7C8FF044628B3C3681BB346
:1038F8005F690FB3062E07D0072E20D02A4631461F
:103908003B46BDE8F0411847838A3BB92A46314611
:10391800B84750B9A38A0133A38206E04FF6FF7275
:10392800934204D00133A3820020BDE8F081124AFB
:103938000121124837F00BFB6FF01500F5E745B190
:103948002A7832B10022314682822A465B6998473A
:10395800EAE7A38A012B08D12A4607212046B8475F
:103968000028E2D1A38A013BD6E70BB1013BDAE795
:10397800034A0221DDE700BF22E0050830250508DB
:1039880044E0050810B5044608B1806838B9104A03
:103998001048012137F0DBFA6FF0150010BDFFF772
:1039A8006BFF08B10C4AF3E7A082EFF311811023F3
:1039B80083F31288BFF36F8F084B5A68C4E900324B
:1039C80014605C6081F31188BFF36F8FE6E700BF76
:1039D80062E00508302505087BE00508940100240D
:1039E80080B505460E46174698460DF00DF9DFF8E6
:1039F8002090034600F072FC0446424649F8003025
:103A080039463046A84754F8090000F001FC00BFC9
:103A18000800000003480021034A08B5121A37F0CD
:103A280031FC08BD40140024004800240748084A17
:103A38000849121A08B537F027FC0748074A084909
:103A4800121ABDE8084037F01FBC00BF0000002470
:103A58000C1400248C6B06080000002400000024CD
:103A68008C6B06082DE9F047064600AF0C46002986
:103A780036D0E9468AB0A3686D46D1E900122148DC
:103A88004FF0050AE846CDE90501CDE9072348F8D6
:103A980010AF002342464FF421511B48FFF7F0FBBB
:103AA800CD466369AD46D4E903121848C5F810A09D
:103AB800C5E90501C5E90723002342464FF4215112
:103AC8001148FFF7DDFBCD46E369114A01210E4895
:103AD80037F046FAA3690F4A01210B4837F040FA3C
:103AE800012E07D1EFF305830B4A103B31460648F8
:103AF80037F036FA214630460BF0C6FEBD46BDE823
:103B0800F08700BFAAE00508C0250508D9E0050828
:103B180008E1050817E1050845E1050830BFFFF78A
:103B2800FDBF00BF2DE9F0410B4E0546DFF82C80A4
:103B3800324606EB0807CC1B094920464EF08EF8A2
:103B4800A019083C424600214EF0AFF807F10800E2
:103B5800C5F89040BDE8F0810000000008000000B2
:103B68008826050810B5204C2049214837F099FBD4
:103B7800A36A990136D51E481E4937F092FB1E20CC
:103B8800A36ADA0104D51A481B4937F08AFB1F20BB
:103B9800154CA36A1B0304D51548184937F081FB57
:103BA8002120A36A590304D51148154937F079FB38
:103BB80022200D4CA36A9A0304D50D48114937F009
:103BC80070FB2320A36ADB0304D509480E4937F0AC
:103BD80068FB2420044A936A6FEA03436FEA13439D
:103BE800936210BD1D20CBE700ED00E058E1050809
:103BF800C025050870E1050883E105089DE1050871
:103C0800BBE10508E0E10508FAE1050870B50646DC
:103C18000D46284C2849294837F043FBA36AD904A4
:103C28003CD52648264937F03CFB1720A36A1A05DD
:103C380004D52248234937F034FB18201D4CA36AC9
:103C48009B0512D51D48204937F02BFBA36BA26AB0
:103C5800100409D51D4A0121184837F081F91EB111
:103C6800A36A23F40043A3621920124CA36A5905DE
:103C780004D51248164937F014FB1A20A36ADA054E
:103C88000ED50E48134937F00CFB1B20094A936ADE
:103C980043F47F43936200232B7070BD1620C5E761
:103CA800A36A9B04F2D505480B4937F0FAFA1C20A1
:103CB800ECE700BF00ED00E025E20508C025050897
:103CC8003BE205084CE205085FE2050878E20508D2
:103CD8008DE20508A8E20508C0E205082DE9F843C9
:103CE800804689461746354D3549364837F0D9FA62
:103CF800AB6ADE0627D511243349324837F0D1FAAA
:103D0800AB6A1D0704D5122430492E4837F0C9FA8A
:103D18002A4DAB6A980718D52D492A4837F0C1FAB9
:103D28006E6BAB6A190646D52A4A334601212548E7
:103D380037F016F9B9F1000F03D0AB6A23F080030E
:103D4800AB62132403E01024DAE76FF015061B4D6D
:103D5800AB6ADA0704D514241F491A4837F0A1FAC8
:103D6800AB6A9B0604D515241C49164837F099FA06
:103D7800124B9A6AD50602D49A6A90070AD55B68EC
:103D8800190507D54146304600F0F4F910B180F323
:103D980009880224094B9A6A920603D55A6A22F4C2
:103DA80000525A629A6A204642F0FF029A62002341
:103DB8003B70BDE8F8836FF01506C2E700ED00E040
:103DC800EFE20508C025050805E305084CE20508EB
:103DD80038E3050850E3050866E30508C0E205086E
:103DE8002DE9F041684B8AB004460025D3F80480D9
:103DF80000AFC8F3080685F31188BFF36F8F02F090
:103E08007F43B3F17F4F07D102F00C03082B12D187
:103E18005E495F4837F045FA00252C460023FB71C0
:103E2800F31E092B00F29080DFE803F00A868982EE
:103E38008E8E8E8E8E8C10074CBF0C460125EDE7BA
:103E48005449534837F02DFA4F4E0023FB71F36A5B
:103E58009A0705D550494E4837F023FA00232DE03C
:103E6800F36A002B01DA4D49F5E7F36A5B00F5D5F3
:103E78004B49474837F015FA7369A26943F48073D0
:103E88007361BFF34F8FBFF36F8F32F8023C7269D3
:103E980022F480727261BFF34F8FBFF36F8F03F408
:103EA8007F42B2F55F4F2CD1DBB2022B29D12368B8
:103EB8003C4A0121364837F053F82368FA79E2B9C9
:103EC80007F1080604F1200C2068083454F8041C93
:103ED8003246644503C21646F6D17A6A002D50D0A0
:103EE800C2F3080121B96FEA52226FEA42227A62CC
:103EF80007F108011846FFF7B5FD2837BD46BDE8AC
:103F0800F081214B9A6AD2B22AB1FA1D01212046CA
:103F1800FFF7E4FE0EE09A6A12F47F4F04D0F91D11
:103F28000120FFF773FE05E09B6AB3F5803F95D348
:103F3800FFF718FE0346C1E7FA1D0021E7E7F91D60
:103F48000020EEE7184986E718F4F87F174AE84694
:103F58008AB0174B08BF13466A461649103ECDE98A
:103F680005134FF400730796ADF82030124B42F852
:103F7800103F00234FF411510548FFF781F9C5465A
:103F88006CE76FF30802B2E700ED00E0B3E3050861
:103F9800C0250508DEE30508F5E3050816E405086D
:103FA80024E4050843E405085FE4050885E30508FB
:103FB8009AE3050883E4050804000001044B5A69E4
:103FC80042F010025A615A6922F008025A61704799
:103FD80000ED00E0EFF30880EFF3098101B57246C8
:103FE800FFF7FEFE01BD00BF0B4880F3088836F0DE
:103FF80003FF102080F3118808484FF4046140182B
:1040080080F30988EFF314800221084380F31488B1
:10401800BFF36F8F00F078F8A0C000240058002488
:10402800BFF34F8F0549064BCA6802F4E062134399
:10403800CB60BFF34F8F00BFFDE700BF00ED00E08E
:104048000400FA051EF0040F0CBFEFF30880EFF32D
:104058000980816911F8021C0229FFD001B5724656
:1040680037F014F901BD00BF09010028C9B206DB09
:1040780000F1604000F5614080F80013704700F0DF
:104088000F00014B1954704714ED00E000B20028EE
:1040980007DB0123410900F01F00024A834042F870
:1040A8002130704700E100E000B200280CDB430932
:1040B800012200F01F0005492033824041F82320E7
:1040C800BFF34F8FBFF36F8F704700BF00E100E071
:1040D8004209054B00F01F0053F82220012303FA80
:1040E80000F01040704700BF00E100E0044B054AB3
:1040F80023F07F039360BFF34F8FBFF36F8F704739
:104108000000000800ED00E008B5FFF7EFFF0C4ADB
:10411800D2F8883023F47003C2F88830EFF31483A0
:1041280023F0040383F31488BFF36F8FFFF772FC47
:10413800FFF77CFC00F0B4F837F0D6F80BF0C6FCBB
:1041480000ED00E042F8203C203A009B084953600B
:10415800019B21F001019360029B9161D3604FF0B4
:104168008073D36100230265C0F89430704700BFA4
:10417800E93900080A4A0346906878B113F1160F26
:10418800D0F8800005D0A0F14002934205D38342C5
:1041980003D2814228BF002070470020704700BF2B
:1041A8009439002415460D4A0E4608B50C4B90600C
:1041B800D0F890201A6000F04FF92C4686F3098851
:1041C8000020044B98472046002100220023024C7F
:1041D80020470000C9B20308E939000894390024CF
:1041E80090350024014B10221A61704700ED00E061
:1041F800054B5A699B689A4204D0044A536843F0B5
:1042080080535360704700BF9439002400ED00E0EC
:10421800084B9B6883420BD1EFF3058343B1064BF0
:104228005A6842F080525A605A6A22F400425A622E
:104238003BF07DBD9439002400ED00E015498A6803
:104248004FF030001044EFF3098C80E8F01F102085
:1042580080F31288BFF36F8F0F4F4FF000664A69E3
:104268008A603E60D2F890000C4C2060D2F894002E
:104278000023C2F8943080F3118804B5104600F08A
:10428800EBF8BDE8044002F1300090E8F01F8CF331
:10429800098870479439002404ED00E09035002423
:1042A800002304481021C2180133612B82F800133F
:1042B800F9D1704700E100E008B5EFF30583064A3D
:1042C800103B02EBC30152F8330049688847BDE848
:1042D8000840FFF78DBF00BF000E002401480068AA
:1042E8007047000090350024154A70B5536913F4DF
:1042F800803323D1C2F88430BFF34F8FD2F8803097
:1043080043F6E074C3F3C900C3F34E335B0103EA19
:104318000406014646EA81750139C2F86052F9D2AD
:10432800203B13F1200FF2D1BFF34F8F536943F4B1
:1043380080335361BFF34F8FBFF36F8F70BD00BFE2
:1043480000ED00E07FB51A4A5369DB032ED5002340
:10435800C2F88430BFF34F8F536923F4803353611D
:10436800BFF34F8F01ABC2F87032BFF34F8FBFF36B
:104378006F8FD2F8803043F6E074C3F3C90001931D
:10438800C3F34E335B0103EA0406014646EA81752E
:104398000139C2F87452F9D2203B13F1200FF2D13F
:1043A800CDE90211BFF34F8FBFF36F8F04B070BD1B
:1043B80000ED00E0002910DD00F01F030B44BFF3FF
:1043C8004F8F07490344C1F8680220301A1A002A9F
:1043D800F9DCBFF34F8FBFF36F8F0020704700BF2A
:1043E80000ED00E00B4B5A6912F4003211D1BFF313
:1043F8004F8FBFF36F8FC3F85022BFF34F8FBFF3B8
:104408006F8F5A6942F400325A61BFF34F8FBFF37E
:104418006F8F704700ED00E0BFF34F8FBFF36F8FD2
:10442800064B5A6922F400325A610022C3F850221E
:10443800BFF34F8FBFF36F8F704700BF00ED00E0F1
:10444800024B0121024A034800F08CB80000042402
:10445800000000248C280508D0F880304021054A47
:10446800403B10461360044BC2E90113012100F0E0
:1044780083B800BF9435002400000B1508B5034627
:104488001048D0F89020C2F30722013A934207D986
:104498000D4801210D4A36F063FD6FF0150008BD87
:1044A800C0F898300A6822F01F021A4342F010023E
:1044B800C0F89C208A6842F00102C0F8A020184683
:1044C800EDE700BF00ED00E0A82505089AE405081F
:1044D800F0B50E4685B01F4604460025B5420DDAF4
:1044E800606810B397B1431E18420AD0104A2B4691
:1044F8000121104836F034FD6FF01502104605B062
:10450800F0BD1F28F2D921680B42EFD1236801A919
:10451800019336F0EAFEA3680343D0B20393FFF792
:10452800ADFF10F1160FE7D0421C01350C34D5E76A
:10453800C0E40508A8250508044B0522C3F8942003
:10454800BFF34F8FBFF36F8F704700BF00ED00E0E0
:10455800BFF35F8F024B0022C3F89420704700BF5F
:1045680000ED00E010B5034C01232278FFF7B0FFFF
:10457800207010BD094400240B4A08B500231278A6
:10458800FFF7A6FF10F1160F07D0084A0021D2F84E
:104598009030C3F30723984200DB08BDC2F89800A7
:1045A8000130C2F8A010F2E70944002400ED00E051
:1045B8005E485F492DE9F043D0F8903085B00C682B
:1045C800C3F307239C4200F2AE80FFF7C1FF49689E
:1045D8000022944201F10C011AD1564F68464FF05F
:1045E8000008554D3C70FFF7E5F8544C8146544E91
:1045F800C14520D13B7800204C49D1F89020C2F326
:1046080007229342C0F289800020FFF795FF50E00F
:10461800C0F8982051F80C3C23F01F0313430132D3
:1046280043F01003C0F89C3051F8043C43F00103F8
:10463800C0F8A030CDE700984FEA081C00EB08113D
:10464800CB682340B3F5000F49D00BD8B3F5001F52
:1046580032D0B3F5800F37D0B3F5801F14D008F1EE
:104668000108C5E7B3F1007F42D0B3F1805F48D0BD
:10467800B3F1807FF3D150F80C30886836F035FEFE
:104688004A6840F0887009E050F80C30886836F0C5
:104698002CFE40F088504A6840F43020039001A96D
:1046A8003878CDE90123FFF7E9FE002831DA6FF009
:1046B800150005B0BDE8F08350F80C30886836F076
:1046C80014FE4A683043E9E750F80C30886836F041
:1046D8000CFE40F000704A6840F40030DEE750F805
:1046E8000C30886836F001FE4A6840F08270D5E7E1
:1046F80050F80C30886836F0F8FD4A6840F480209D
:10470800CCE750F80C30886836F0EFFD4A6828434B
:10471800C4E73B7801333B70A1E7C1F89830013317
:10472800C1F8A00069E74FF0FF30C2E700ED00E0F4
:10473800AC27050809440024000002110000F0FF1E
:1047480000000811F0B587B007460E461446002150
:10475800102268461D464DF0A8FA02232A46214633
:104768008DF802306846044BCDE90476019333F0A6
:1047780023FD07B0F0BD00BF19B3030808B5024B0D
:104788001B689847002008BDA0350024034B044A45
:104798001860937843F0020393707047A0350024A3
:1047A8009C01002408B5054835F0ACFF002383F3CD
:1047B8001188BFF36F8F0423184602DFE6E405086B
:1047C8000649074821F00701C1F1105208B502F562
:1047D800802235F006FF002008BD00BF9FDD0024C1
:1047E800A43500244FF0FF324FF0FF3301480BF09F
:1047F80003BB00BFAC01002401480BF06FBB00BF36
:10480800AC01002438B50546FFF7ECFF082108483D
:104818002A4635F03CFE044628B925B1054B0C2242
:10482800FFF75CFD1A50FFF7E7FF204638BD00BFD1
:10483800A43500240C00000038B504460D46FFF7E7
:10484800D1FF082221462B46074835F092FE044640
:1048580028B925B1054B0C22FFF740FD1A50FFF788
:10486800CBFF204638BD00BFA43500240C00000053
:1048780010B50446FFF7B6FF03482146FDF7CCFD07
:10488800BDE81040FFF7B8BFA435002470B54169F2
:104898000446867A0A4D59B1437ADB0706D42C239D
:1048A80003FB06535B6A1B689B6898470023636198
:1048B8002C20214600FB0650BDE870403BF08EB925
:1048C8007C1200242C22024B02FB0030704700BFF0
:1048D8007C120024827A2C21054B01FB02339A6A50
:1048E8001B7F801A1B3323F00303B0FBF3F07047E0
:1048F8007C12002438B52C24827A064B04FB023340
:104908005B6AD3E901240C601568FFF7E3FF04FB39
:10491800005038BD7C1200242DE9F04385B00546CF
:1049280090461C46684603913BF0A5FBDDE900670D
:10493800EFF31189102383F31288BFF36F8F6B8B0A
:10494800002B41D02A8B9A4225D9002200232846E1
:104958000BF014FB0446F0B189F31188BFF36F8F95
:10496800039B002B41D032463B4668463BF0A8FBF0
:10497800A27A2C21254B204601FB023303A95B6A4E
:104988001B681D68DDE90023A847606170BB2046ED
:10499800FFF77CFF24E0698B4B1E6B8389F311883A
:1049A800BFF36F8F2B7F2A8B1B33AC6A521A23F00D
:1049B800030302FB0344154B154AEB1A9B105343A0
:1049C800A3722B7FE372CBE789F31188BFF36F8F54
:1049D8002346424628460BF0D1FA04460028BFD1A8
:1049E8000024204605B0BDE8F0836361012300255B
:1049F800E27A04F1180023812946039B65606382EB
:104A08004DF053F963692582E360EAE77C120024DC
:104A1800A38B2EBAF8B50024114D2C2600B9F8BD89
:104A280000F108024768BFF35B8F52E8003F591E48
:104A380042E8001CBCF1000FF7D1DBB2BFF35B8F7B
:104A4800012BECD1837AC46006FB035344601B6AD4
:104A580013B198473846E1E7FFF718FFFAE700BFB8
:104A68007C120024F7B506460D461446124F384608
:104A78003AF0C4FEE0B1BB68AAB2314638461B68BA
:104A88009847002802DB002003B0F0BD002CFBD1C2
:104A9800AC42F8D22F1B042F28BF042707F0D8FDFB
:104AA80001A901903A4630194DF0D8F83C44EFE797
:104AB8006FF01200E8E700BF4422050838B5044645
:104AC8000CF07EF8204636F0A3FCA069C8B194F833
:104AD8006C30DB070DD56FF07705154A02211548B4
:104AE80036F094FC201D36F09AFC0CF07DF8284630
:104AF80038BD3AF083FE38B90F4A01210D4836F027
:104B080085FC6FF01205EDE7204601F04BF80546ED
:104B18000028E7D10146242204F128004DF0C5F809
:104B280094F86C3043F0010384F86C30DAE700BF86
:104B380006E505084826050830E5050870B5044669
:104B48000CF03EF8204636F063FC94F86C30DA0737
:104B58000DD44FF0FF35254A0221254836F056FC82
:104B6800201D36F05CFC0CF03FF8284670BDC3F3FE
:104B780040019B0707D51F4A02211D486FF07705A2
:104B880036F044FCECE7A06937F0AAFE0646A069B7
:104B980037F036FF054628B1174A0121144836F088
:104BA80035FCDDE7A36F4BB13146204636F0CEFD2C
:104BB8000546A0B1A06937F04FFFD1E7A06937F0EB
:104BC800C7FEA0670028EFD10C4A012108486FF002
:104BD8000B0536F01BFCA06937F03EFFC0E794F8E0
:104BE8006C3043F0020384F86C30B9E753E50508EC
:104BF8004826050879E505089FE50508BBE5050889
:104C080038B590F86C3004469B0708D46FF07705E8
:104C1800134A0221134836F0F9FB284638BD36F00E
:104C2800F7FB0021204601F057F920B10E4A012177
:104C38000C4836F0EBFBA06937F00EFF054620B1B3
:104C48000A4A0121074836F0E1FB94F86C30201D30
:104C580023F0020384F86C3036F0E1FBDDE700BF97
:104C6800D7E5050848260508FEE505081CE60508F9
:104C780038B580210446806937F08DFE054678B145
:104C88000146204601F076FB044638B1064801216A
:104C9800064A36F05CF92846FFF7BCFE204638BDC8
:104CA8006FF00B04FAE700BF282605084CE6050854
:104CB80038B50446806F36F05FFB054636F040FB9A
:104CC8002046294601F056FB044638B10448012124
:104CD800044A36F03CF92846FFF79CFE204638BDCA
:104CE800282605086FE605082DE9F04F994685B096
:104CF80007468846154636F094FB0446B9F1000F7E
:104D080010D0384636F092FB012808D0334B6FF0AC
:104D18008502FFF7E3FA1A5005B0BDE8F08FB4FA40
:104D280084F46409013521463846EAB236F027FD95
:104D3800064630B92A4A2B4601212A4836F010F98E
:104D4800E4E74568B9F1000F09D0286801AB696844
:104D580003C32A7A01AD1A7007238DF8053008F1CC
:104D68000C09484636F095FC2A782946824228BF25
:104D78000246484636F01FFBD6F80CA0BAF1000FE1
:104D880009D1B8F81010FB8D9942C5D9C91A4846FF
:104D980036F02CFBC0E7DAF8040083681B6B13B904
:104DA800DAF800A0EAE7214698470028F8D0051F5E
:104DB80055F804BFBBF1000FF2D09BF80060002E3D
:104DC800EED0484636F065FCB042594634BF82B250
:104DD8003246484636F0EFFAEAE700BF0C0000001A
:104DE8008EE60508282605082DE9F04190F82830B8
:104DF80004460F4600F1280603F01F03012B2FD0AD
:104E0800022B18D08BB394F82910204636F055FBA6
:104E1800024678B330461E4D36F043FC002834D1A4
:104E280013693BB33A463146204698470346FFF795
:104E380055FA2B5024E0818DC9B201F099F9054645
:104E48000028E0D0304636F02CFC024668688368BB
:104E5800CAB99B6873B13A463146BDE8F041184774
:104E6800818DC9B236F0DFFCE9E790F8291036F0F9
:104E7800F3FCE4E7064B6FF08502FFF72FFA1A50B0
:104E88000020BDE8F081DB68E4E7D368C9E700BF2C
:104E98000C0000002DE9F04F0B7E95B004460D463E
:104EA80033F0800816460AD06FF00408A74A01219B
:104EB800A74836F04CF8404615B0BDE8F08F82B1EF
:104EC8000846FFF7A7FD6B7EDF0704D49E07F2D5DF
:104ED8002B7E002BEFD1204615B0BDE8F04FFFF731
:104EE800E7BE4A7E00F12809900705D5802B09D135
:104EF8002846FFF78FFDDEE7910700F05784002B67
:104F080040F05484D20734D52B8A082B0DD1EA6897
:104F1800294600201368A3625368C9F8043036F0A4
:104F280032FA054640B18B4A00E08B4A0121884895
:104F380036F00DF800F012BC484636F0B2FBE28DB0
:104F480070B9B2B12946A06937F011FD01460028B1
:104F580000F06784204615B0BDE8F04F01F00ABAAA
:104F68003AB11146204636F05BFD0546002800F0B0
:104F7800588494F828800023FFF7B0F9774F18F089
:104F8800600FC351C8F3411307D0032B40F0D681FB
:104F98006FF08503FFF7A2F938E0484636F081FB49
:104FA80094F82930002840F06981013B0A2BEFD89A
:104FB80001A252F823F000BF71510008994F000870
:104FC800F9510008994F0008ED4F0008994F000863
:104FD800994F0008994F000869500008994F000838
:104FE800DB500008618D7F29D2D8A38D002BCFD14B
:104FF800E38D002BCCD118F01F0FC9D194F83030B5
:10500800022B05D14FF0FF33FFF768F93B5084E0DE
:10501800A069036993F880301B070DD5C9B236F033
:1050280079FB804658B1638D4D4A0121484835F0D7
:1050380097FF002D74D13EE7012384F8393094F8A6
:105048003030012B0AD1638D43B984F83030FFF733
:1050580045F93B58002B00F09C805EE00123F4E703
:10506800204636F0DEF9628D0146FF2A90D8E38D9E
:10507800002B8DD194F82830D80689D194F8303097
:10508800002BBFD02AB1D2B2204636F09EFB0028B2
:10509800B8D0618D94F838308B42D8D0C9B2204648
:1050A80000F01AFF638D804630B12E4A012100902E
:1050B800274835F05FFFBCE7002B4FF0050120467D
:1050C80014BF0222012284F830201A4636F0ECFC84
:1050D800BDE708F01F08B8F1010F7FF459AFE38D61
:1050E800002B7FF455AF628DFF2A3FF651AFA18D9B
:1050F800FF293FF64DAF94F83030022B82D1D2B25F
:105108002046C9B236F011FC10F1020F804640F07B
:105118001A81FFF7E3F847F8008065B14FF00008FF
:105128002846FFF777FCB8F1000F7FF4C4AEFFF70D
:10513800D5F83B586BB3484636F0B3FA0346A06936
:10514800002B00F07183802177E300BFB4E60508E7
:1051580028260508ECE60508D5E605080C00000039
:105168000EE7050830E70508E38D002B7FF410AF44
:1051780094F83030002B3FF445AF012BA18D02D1BC
:1051880000297FF43FAF18F01F080CD0B8F1020FC8
:1051980016D0E38D002B40F0D4822046FFF768FD3F
:1051A8000028C8D197E600297FF42CAF638D012B26
:1051B800EFD194F86C3061F3C30384F86C30E8E7FE
:1051C800B4F82AA0BAF1000FE3D15FFA81F82046BB
:1051D800414601F037F90346FFF780F83B500133A9
:1051E80000F0338352464146204636F060FA2EE7F7
:1051F800E38D002B7FF4CCAE628DA38D022A5FFA7B
:1052080083FA11D108F01F085AEA08087FF4C0AEE3
:105218000122190AA06936F05AFA00287FF4B8AEBC
:10522800012384F8393012E794F8301000293FF44C
:10523800E9AE012902D1002B7FF4E4AE18F01F0873
:1052480012D0B8F1020FA4D1002AA2D151462046AB
:1052580001F0D6F80346FFF741F83B50013300F060
:10526800F48201225146BFE7002B7FF4CBAE012A1E
:105278008FD194F86C3043F008039EE70A2B3FF671
:1052880087AE01A252F823F0BD520008994F0008DA
:10529800994F0008994F0008994F0008994F000846
:1052A80037530008994F0008C3560008994F000863
:1052B800F1560008E38D022B7FF46AAE94F8303083
:1052C800002B3FF49FAE012BA18D02D100297FF462
:1052D80099AE18F01F0811D0B8F1020F1CD04FF08A
:1052E800000805F10C0A504636F0D3F9E38D9842D0
:1052F80018D26FF00B03FEF7F1FF87E600297FF461
:1053080081AE94F86C304FEA9308C3F3001308F0A9
:10531800020848EA0308E4E7C9B2204636F0A4FBCD
:105328008046DEE74146504636F056F88FE6628DF5
:1053380018F01F0F4FEA1223D2B209D0294620468F
:10534800FFF752FD8046B8F1000F7FF472AE7EE69B
:10535800013B0E2B3FF61CAE01A151F823F000BF14
:10536800A5530008E1530008F1530008994F0008BD
:10537800994F000849550008ED530008994F000857
:10538800994F0008994F0008994F0008994F000855
:10539800994F0008994F0008DD55000805F10C08E1
:1053A800B4F82EA0404636F074F98346204636F00D
:1053B80038F820B101287FF4EBAD616F00E0216F70
:1053C800002900F03E82DA450A7828BFDA465245BD
:1053D80028BF524640462FE0002329462046FFF7C3
:1053E80083FC34E60123F8E70321204636F0A5F8CC
:1053F800824600283FF4CCAD36F046F9B4F82EB01A
:105408009AF81520D8B99AF814808DF831208DF8BB
:105418003080DAF8103005F10C0A1B885046ADF8D8
:10542800323036F036F9D8450CA928BFD846804521
:10543800424628BF0246504635F0BDFF07E6DAF877
:10544800081000238DF81D20C64A8DF81C300A402C
:10545800C5498A4263D1102108A805F0C5FDB0F1FD
:10546800000842DB0CAAB8F1100F08A94FF000039E
:10547800104628BF4FF01008DFF8F0E2984502F117
:1054880002023CD84FEA8808034608F102085FFA8E
:1054980088F88DF81C8005F10C0A0493504636F004
:1054A800F8F8D84507A928BFD846804528BF8046C0
:1054B8005046B8F1020FC34628BF4FF0020BA8EBC5
:1054C8000B085A4635F077FF4FEA58030393049BBD
:1054D8009B4603EB58025A4528D118F0010F3FF4B8
:1054E800B6AD039A995C5046FBE018F1580F7FF46B
:1054F8004FAD9F4A01219F4835F029FD48E511F835
:1055080001CB01334FEA1C1A0CF00F0C1EF80AA04D
:105518001EF80CC002F802AC02F801CCAEE79AF80B
:105528001480DAF810308DF81C80B4E71BF8011BE2
:105538005046CDE9042335F04FFFDDE90423CAE7DF
:10554800204635F06EFFD4E91C83002808BF984632
:1055580000232046CDF83230CDF836300A238DF8B6
:10556800303006238DF8313035F060FF012805D042
:105578006FF08503FEF7B2FE3B5068E5B8F1000F07
:1055880000F05F81B8F80230ADF8323098F8043096
:105598008DF8343098F805308DF8353098F80630A5
:1055A8008DF8363098F807308DF8373098F8113084
:1055B80005F10C0840468DF8383036F06AF8E28D6F
:1055C8009DF830300CA99A4228BF1A46824228BF5B
:1055D8000246FFE6204635F024FF18B10128C7D15E
:1055E800636F00E0236F002B00F02B815B88B3F51D
:1055F800007FBDD9604B04F14C0B0C9300238DF850
:105608003430E36C9B4508BF0023BDF8322093B1CA
:10561800597D0F2908D1197D0A44ADF832209DF82B
:10562800342001328DF83420226D934201D01B685A
:10563800EBE7BDF8322005F10C0A0392504636F02C
:1056480028F8B4F82E80039A0CA9904528BF9046F4
:10565800804528BF804650464246052A28BF052275
:10566800039235F0A8FE039AB8EB02083FF4EFACBA
:10567800E36C5B453FF4EBAC002B3FF4E8AC5A7DA0
:105688000F2A14D11A7D504619694245039328BF41
:10569800424635F090FE039B1A7D424594BFA8EB25
:1056A8000208A8EB0808B8F1000F3FF4D0AC226D4F
:1056B8009A423FF4CCAC1B68DEE794F83030002BFC
:1056C8003FF4A0ACE38D012B7FF462AC05F10C082C
:1056D800404635F0DEFF00283FF40BAE94F8381052
:1056E800404635F071FEB2E408F01F08B8F1010F2A
:1056F8007FF488AC204636F056F800283FF482AC98
:10570800B4F82C80B8F1FF0F3FF642AC43681B7920
:105718004345FFF43DAC5FFA88F30F2B3FF638ACF6
:10572800E38D012B7FF434AC05F10C0A504635F0BB
:10573800B0FF00283FF4DDAD04EB080393F83A10FE
:10574800D1E6484635F0ADFF18B92846FFF762F9AB
:1057580023E52946204600F00DFE78B12846FFF7DC
:1057680059F9E8E400FF020000030200ED3F0608D3
:1057780053E7050828260508050F0500A0690369F1
:1057880093F8801011F004017FF4A5AB37F003F90A
:10579800054600283FF4CFAC0146204600F0EAFD5C
:1057A80000283FF498AB2B4AFFF7C0BB52077FF5A0
:1057B800C2AC002B3FF49CAB2846FFF72BF994F8BA
:1057C8003930002B3FF477AB94F82930052B0CD1F6
:1057D800618DA069C9B235F09DFF064628B1638D79
:1057E8001D4A01211D4835F0BBFB94F82930032BD5
:1057F80011D1638D022B0ED1A18D0022A0690D0A53
:10580800294635F064FF064628B1154A2B46012182
:10581800124835F0A5FB0023B04684F83930FFF76D
:105828004ABB6FF00B0686E4E38D002B3FF48BAC8C
:1058380016F10C0118BF0121C90136F0AFFFFFF7BF
:105848004ABB6FF01508FFF7F4BB4FF0FF38FFF7BE
:10585800F0BB00BF75E705080EE705082826050810
:1058680099E705080B78062B10B414D10369D3F80F
:105878009C20EFF31184102383F31288BFF36F8FFA
:1058880000204B681860506A58B9C2E9083384F39D
:105898001188BFF36F8F00220023034810BC3AF031
:1058A800ABB803605362F2E7F811002430B589B051
:1058B8000022002300241E491E480094CDE9062337
:1058C8006FF007034FF48062CDE90334CDE901445A
:1058D800194B0AF07FFE194916483AF023FA184B7B
:1058E80018498B4207D3184B002018498B4210D314
:1058F800002009B030BD03F11402BFF35B8F52E8FA
:10590800000F42E80045002DF9D11833BFF35B8F33
:10591800E7E703F11402BFF35B8F52E8004F42E858
:105928000005002DF9D11833BFF35B8FDEE700BF08
:10593800404B002460280024B1590008230B0608B6
:105948007C130024C4130024C41300240C14002462
:1059580038B50D4635F027FF30B9114A01211148F5
:10596800BDE8384035F0F3BAC46804B938BD2B78BF
:10597800032B05D0052B0ED0022B08D02468F4E7A2
:10598800606883685B69002BF8D09847F6E7606821
:1059980083689B69F7E760688368DB69F3E700BFA2
:1059A800C0E70508382605082DE9F04385B04FF013
:1059B800100800AF4FF0FF334FF0FF32391D734826
:1059C8000AF0B6F9FB681B69D3F89C40236A93B1C7
:1059D800EFF3118288F31288BFF36F8F256A2DB118
:1059E800616A2B688D42236208BF636282F3118863
:1059F800BFF36F8FC5B93B79062BDBD0072BD9D8FE
:105A080001A252F823F000BF8D5A0008815A0008FD
:105A1800B55A0008935A0008EB5A0008D75A0008EC
:105A2800BD590008855B00082B7E2946D5F81E2045
:105A380020465E061DD1FFF72DFA06460028C5D080
:105A4800E9468AB02B7E6A465149CDE907350523D8
:105A5800CDE9051042F8103F00234FF421514D487D
:105A6800FDF70EFC324607212046CD4636F01CF8DD
:105A7800ACE735F0E8FEE0E700220121204636F0E9
:105A880013F897E700221146F8E794F86C3043F0D2
:105A9800040384F86C3094F83030022B03D1391D9C
:105AA8002046FFF755FF00220321E7E794F86C3002
:105AB80023F0040384F86C3094F83030022B03D1BF
:105AC800391D2046FFF744FF00220221D6E794F84B
:105AD8003030022B7FF46EAF391D2046FFF738FFB8
:105AE80068E794F86C30A66923F0040384F86C30F6
:105AF800D6F808903369BFF35B8FD3F8A030BFF3B3
:105B08005B8F9A071ED5D9F83C3030469847D9F8AC
:105B180024300021304698470546D9F840303046B1
:105B2800984795B11C4A01211A4835F010FA00220D
:105B38000421204635F0B8FF002D3FF43BAF2A463C
:105B480007219BE74FF0FF35ECE72946204600F098
:105B5800C3F9054608B1114AE5E7A06936F03AFFEE
:105B6800831E84F830505842584194F86C3023F022
:105B7800680343EA401384F86C30D8E7084A0121E7
:105B8800044835F0E4F9BA68062177E7F8110024EB
:105B9800EFE705083826050819E8050847E8050865
:105BA80073E8050838B5024605460C49806936F0A1
:105BB80077FF044630B10A4A01210A4835F0C7F98F
:105BC800204638BD85F83800284600F043F90446D9
:105BD8000028F5D0A86936F096FFF1E76D5800085F
:105BE80083E8050838260508F8B501231D460C6822
:105BF800002C35D063F07F02D6B202F07F0210325B
:105C080024FA02F7FF0716D5046824FA02F7FF07FB
:105C180008D4334613480121134A35F0A1F96FF02F
:105C28001500F8BD05FA02F224EA020404600C68C3
:105C380024EA02040C60DC40E6070ED5026822FA6A
:105C480003F4E40700D4E5E705FA03F422EA0402C2
:105C580002600A6822EA04020A600133102BC6D1E6
:105C68000020DEE760260508AAE805082DE9F04FC0
:105C7800002691B05368D4680A900891069202935E
:105C88000E96039674B9039B029A093316719BB258
:105C980093701B0AD370069BDC68002C40F0C6800A
:105CA800A346ADE060684FF0000A8368CDF83CA0D9
:105CB8001B6B002B00F0AB8008999847002800F078
:105CC800A680A0F104093546C4E903AA59F8043F9F
:105CD8000BB11A789AB9B54240F29680E3680F9AE8
:105CE8001343E360606883689B6A002B00F091802F
:105CF80098478346002800F08F80534A7CE05A7802
:105D08000B2A08BF9D70D9F800305A78042A10D1A0
:105D1800E2680F990A43E260DA78002A5BD101222F
:105D28009D702369AA4001351343EDB22361CDF874
:105D38003CA0D9F800707B78052BC7D10A9B6FF07F
:105D4800120B4FF001089B69099379793A790E9BF8
:105D580042EA01225FFA88F10493ADF8362097F9F8
:105D68000220002AB3BF41F080014FFA88F342466F
:105D78004BB2B7BF21F08002079310320793049B00
:105D880023FA02F0C0072DD40F9B23FA02F20593E1
:105D9800D30727D4BB79FA78099800930DF1360315
:105DA8000B9136F071FC0B998346D8B9079BB970F3
:105DB800002B4FF001030498B8BF21F08001BDF813
:105DC8003620B8BF1031BA808B4005991843194363
:105DD800CDE90E017AE76A1E0FA90EA89A70FFF79F
:105DE80003FFA4E708F10108B8F1100FADD1BBF12A
:105DF800000F3FF46BAF154A0121154835F0A7F89D
:105E0800584611B0BDE8F08F6FF0150BF3E7354633
:105E180068E76FF0850B70E760682E46089935F0E3
:105E2800E2FC039B2468034403932BE7E36804F133
:105E38000C010EA8A360FFF7D7FE08B924682CE769
:105E48006FF0150BDCE700BFEBE80508C7E80508AD
:105E58006026050870B583690546026F1B6993F8CB
:105E68008030C3F34113022B0CD0032B0CD0012B31
:105E78000CBF10230823D371EE6D3EB96E6DBEB909
:105E8800344611E02023F6E74023F4E732460121A7
:105E98002846FFF7EBFE044640B173685B790B4A6E
:105EA80001210B4835F05CF8204670BD3668E4E700
:105EB800324600212846FFF7D9FE044618B1736818
:105EC8005B79044AECE73668D9E700BF0FE90508B3
:105ED8006026050832E905082DE9F04105460E4619
:105EE80035F09FFA804695F8383033B3284635F0B8
:105EF8005AFC0746F0B10146284635F0C4FC10228A
:105F08000446002105F13A004BF0CFFE002385F846
:105F18003830FF683FB984B119491A4835F022FC76
:105F28002046BDE8F081786883685B6A03B19847CA
:105F38003F68EFE76FF03C04EEE71EB985F838607C
:105F48000024EDE732464146284635F018FC07465E
:105F580090B10246284635F0C0FC04460028DFD13F
:105F680085F83860FC68002CEAD0606883681B6A92
:105F780003B198472468F6E76FF03C04D0E700BF08
:105F8800FEE50508202605082DE9F04105460F46DF
:105F98001446D2F8048035F0E9FB95F86C30D9073F
:105FA8000BD56FF00F074649464835F0DBFB281D37
:105FB80035F0E3FB3846BDE8F081012F0AD12846C9
:105FC80035F034FA30B940493E486FF0850735F06E
:105FD800C9FBECE798F807309A0607D5AB691B6947
:105FE80093F880309B0701D43849EDE71FB1012FA2
:105FF80006D03749E8E7EB6D2BBB05F1540603E003
:106008006B6DABB905F15C06336800220BBBD5E9B3
:106018001C23002F08BF134662685B7C03F1010351
:10602800DBB25371D5E91C1208BF0A46537422E04B
:106038009C4206D1274923486FF0150735F092FB9B
:10604800B5E71B68DDE79C4201D12349F3E71B68EC
:10605800D2E79C4221D12368CAB97268336094425E
:1060680000D173600023236063685B791B4A0221B7
:10607800144834F075FFA168B9B1284635F077FAAD
:10608800074668B116490F4835F06CFB8FE7136077
:1060980073689C4208BF7260E4E71A461B68B5E75C
:1060A800A06835F0F1FA88F80600002323607368C9
:1060B8001BB9C6E90044002779E71C607460FAE759
:1060C80083E9050820260508A5E905085FE905080C
:1060D800C3E90508E3E9050800EA05081DEA05081B
:1060E8003AEA0508F8B5054600AF29B301290BD1EE
:1060F800184C194E2BE0636828461968FBF708F915
:10610800B8B11834B442F6D36C4688B06A46134B1B
:10611800CDE905354FF40073ADF81C30104B42F84B
:10612800103F00234FF4E2510E48FDF7A9F8A546A9
:1061380000242046BD46F8BD0B4C0C4EE2E76368D0
:1061480028461968FBF7E4F80028F2D01834B4425E
:10615800F5D3D9E7C41300240C14002471EA050808
:1061680003000001302605087C130024C413002412
:1061780001F07F0311F0800F70B518BF10330125AF
:1061880004469D4090F83030022B06D00C4A01217D
:106198000C4834F0DCFE002070BD90F8386035F013
:1061A80040F901462046324635F0E9FA0028F2D097
:1061B800C0680028EFD083681D42EDD10068F8E779
:1061C8008FEA0508302605082DE9F84305460846F4
:1061D800114616461F46FFF785FF044600284AD099
:1061E800284635F0F9FA95F86C30DA0702D5234AD3
:1061F80001210CE0D4F8048004F11409BFF35B8F8B
:106208006369BFF35B8FDB070CD51D4A02216FF072
:106218000F041C4834F09BFE281D09F05FFE204641
:10622800BDE8F883D8F804301BB1AB4201D0164A58
:10623800DEE73A463146284635F0A1FAC0B10023D8
:10624800236003698BB9C0E90344BFF35B8F59E846
:10625800003F43F0010349E80032002AF7D1BFF3B9
:106268005B8F0024C8F80450D6E71C600461ECE793
:106278006FF03C04D0E76FF01204D0E783E905081B
:10628800B4EA050830260508D6EA05082DE9F04FD6
:1062980083B00E468146904600AF4C687B6097F805
:1062A80030303B6035F0BDF8A36801461B6B33B94D
:1062B8006FF0150420460C37BD46BDE8F08F204628
:1062C80098470028F4D0051F002406F10C0A55F859
:1062D800041F09B10B782BB9002C14BF00246FF0F0
:1062E8003C04E7E74B78042B0ED1002C3CD18B788B
:1062F8007A689342EBD1CB783A689342E7D10B792D
:10630800002BD7D00124E2E7052BE0D1002CDED00A
:10631800B8F1010F91F802B009D0B8F1020FF1D12C
:1063280052465946D9F8180035F064FB04E0524645
:10633800D9F8180035F043FB04460028E2D06D4632
:106348008AB0F3686A4609490990CDE907B306237C
:10635800CDE9051842F8103F00234FF44151044895
:10636800FCF78EFFAD46A5E70024A3E716EB05086A
:10637800582605082DE9F0410B7E0C4605465906BE
:1063880037D16BB335F08DF840B11B4801211B4A5A
:1063980034F0DDFD4FF0FF30BDE8F0812846D5F838
:1063A8007080268AEF8D35F03CF8F8B1421E5342D2
:1063B80053419B01228A9AB1BE423246E98D28BFD9
:1063C8003A4691420CD9B2FBF3F103FB11223AB9D8
:1063D80094F91830002BBEBF637E43F00803637640
:1063E8002146A869BDE8F04136F034BA98F807307C
:1063F800E0E76FF01500CFE75026050852EB0508D7
:1064080070B5064680690C4636F0C8F9054638B1BD
:106418000A4A234602210A4834F0A2FD284670BDE4
:1064280014F0800F4FF00102736B1CBF24F080043E
:106438001034A2401A437263F0E700BF66EB050808
:106448005026050870B5054680690E4636F0D1F924
:10645800044638B1064A33460221064834F080FD26
:10646800204670BD314605F1340035F09AFAF7E759
:106478007DEB05085026050870B50646EFF3118137
:10648800102383F31288BFF36F8F1B4D2A6881F3A3
:106498001188BFF36F8F526892F86C20D20705D429
:1064A8000A220023BDE8704009F0E0BFEFF3118233
:1064B80083F31288BFF36F8F2C682CB16968236847
:1064C8008C422B6008BF6B6082F31188BFF36F8F1B
:1064D80044B1606804F10801C36998472146074838
:1064E80039F027FA2B6833B1304600220023BDE883
:1064F800704009F087BF70BDB035002484110024B6
:1065080030B585B0054600231548CDE900120022B4
:1065180003A909F073FB0246E8B9039BDDE9000112
:106528005D60083383E80300EFF31180102383F3E1
:106538001288BFF36F8F039B1A600A4A516861B9CA
:10654800C2E9003380F31188BFF36F8F0022002364
:10655800054809F057FF05B030BD0B605360F1E7FF
:1065680084110024B03500240000002438B54B788D
:106578000469202B4568206908D0222B19D0124BBA
:106588006FF08502FDF7AAFE1A5010E0CB88072BA2
:10659800F5D1D3681A6842609A8802819B79837220
:1065A80035F0A7FA22460821284635F08BFA002054
:1065B80038BD4B880921C3F34002838103F00103EE
:1065C800027622464376EFE70C00000008B5134632
:1065D8004A78212A14D133B90C4B6FF00B02FDF71E
:1065E8007DFE1A500AE0CA88016903F10C00072AE7
:1065F800096928BF0722043134F0DDFE002008BDF8
:10660800024B6FF08502FDF769FEEAE70C00000017
:1066180073B5102504698DF80710EFF3118685F31B
:106628001288BFF36F8F01220DF10701E06B34F080
:106638002FFB86F31188BFF36F8F012816D039F02E
:106648006BFBD8B1114B0122BFF35B8F53E8001FDE
:10665800002903D143E800200028F7D1BFF35B8F5E
:1066680004D10B4A02210B4834F071FC0A220023A2
:1066780004F1480009F0C6FE02B070BDA37E002BED
:10668800E0D000210A2039F050FCC6E7B8350024D4
:10669800A7EB05081826050838B5056900240E4932
:1066A800EB6B05F14800C3E90144DC606B6BC3E99F
:1066B8000144DC6039F024FB05F17800074939F022
:1066C800F3FA074905F1240039F0EEFA284635F0C7
:1066D80010FA204638BD00BFF56700082569000894
:1066E800F96900082DE9F341036906460D46D0F81B
:1066F80004801C690F7E002A32D00B8A7132384818
:1067080007BF0221374A0121374A00933B4634F03C
:1067180031FC2F7E304635F063FA874204D10421DC
:1067280004F1880035F0CCFA2F7E304635F066FA51
:10673800874204D1052104F1880035F0C1FA2F7E83
:10674800304635F03FFA874203D104F18C0009F056
:10675800A9FC2946404602B0BDE8F04135F081B9B0
:1067680035F03EFAB84214D12A8AE968606B34F0F1
:106778008FFA28B1E3691BB104F1240009F0D2FDB6
:1067880004F18800042135F09BFA04F1780009F03F
:10679800C9FD2F7E304635F031FA874215D1E369BD
:1067A8001BB104F1240009F0BDFD052104F18800A6
:1067B80035F086FAE36B5A89DB889A4205D00022C5
:1067C800002304F1480009F01DFE2F7E304635F005
:1067D800F9F98742BDD104F18C0009F001FCB8E752
:1067E80018260508C6EB0508EAEB05082DE9F04769
:1067F80050F8483C00F14006074600215B683046E7
:10680800D3F8009035F0D5F900285AD00121304648
:1068180035F0CFF98046002853D1BFF35B8F56E897
:10682800003F43F0200246E800210029F7D19B06EB
:10683800BFF35B8F45D4484635F0E0F900220546A2
:106848000023214834F081FD044650B93046052123
:1068580035F036FA38460A220023BDE8F04709F039
:10686800D1BD82460576428A5AF80C1F57F80C0C9F
:1068780034F02EFA05460146504634F096FD5DB1D7
:10688800D9F8040035F013FAB5FBF0F303FB105503
:10689800B5FA85F84FEA58182146484607F82D8C6E
:1068A80035F0C7F868B10121084A094834F04FFBB0
:1068B8002046FEF7AFF830460521BDE8F04735F031
:1068C800FFB9BDE8F08700BF7C1200240BEC050877
:1068D8001826050838B5034640681B695D68AC682A
:1068E800A37A84F8223094F82D3084F8233069682C
:1068F80049B1237C3BB934F03AFE30B1054A012155
:10690800054834F024FB002038BD686834F0BCFE2C
:106918002074F8E71DEC05081826050870B550F82E
:10692800782C00F1100403460021526820461568AF
:1069380035F03FF9002851D00121204635F039F9CA
:1069480000284BD153F8442C6868938891891669BC
:106958005B1A9BB2F61A35F0AAF9B0423ED8BFF3DB
:106968005B8F54E8003F43F0100244E800210029FF
:10697800F7D1DB06BFF35B8F06D5194A0221194808
:10698800BDE8704034F0E3BA284635F029F9002212
:1069980006460023144834F0D8FC0446F0B10676C5
:1069A800686835F084F9638A984203D2686835F0DC
:1069B8007EF983B221462846638235F03AF868B1F9
:1069C800284635F00DF9034606480121074A34F0F8
:1069D800C7FA2046BDE87040FEF71CB870BD00BF7E
:1069E80047EC0508182605087C12002467EC050802
:1069F80038B550F8083C044633B92C4A01212C48D4
:106A0800BDE8384034F0A3BA50F8243C00F16405DE
:106A180002215B681A68002383828383284635F045
:106A2800C8F8B8B1106954E902319847637D1BB1C1
:106A380004F1540009F076FC0521284635F0B9F830
:106A480098B9637F6BB10022002304F1240009F098
:106A5800D9FC0AE00321284635F0ABF80028E1D13B
:106A6800E4E714F8093C002BEDD10221284635F063
:106A7800A0F838B12369DA885B899A4202D02046A7
:106A880009F050FC0321284635F093F860B1A2695B
:106A98009388918912695B1A9BB29A4204D0204666
:106AA800BDE8384009F03EBC38BD00BF8CEC050895
:106AB80018260508D3B50026002704460648CDE960
:106AC800006734F046FC20B1230604765CBF00233F
:106AD800038202B0D0BD00BFA81200242DE9F04304
:106AE80083B000231D4C4FF00108056902AF1C4E0E
:106AF80005F1240928602B7785F82030B442234615
:106B080001D3002019E095F820201034CAB16C4652
:106B180088B01B6802AA1349C2E905134FF4007331
:106B28009383114B42F8103F104800234FF4E25171
:106B3800FCF7A6FB6FF00B00A5460437BD46BDE881
:106B4800F08385F82080484654F8043C009354F8B4
:106B5800101C54E9032335F083FBCFE7987F060820
:106B6800A87F0608EEEC0508030000016826050862
:106B78001FB5CDE9010103924FF0FF324FF0FF330B
:106B880001A9034838F038FF002005B05DF804FB80
:106B9800C811002413B54B781446FE2B15D14B8829
:106BA8009BB9CB888BB1036993F820300BB1013BBB
:106BB800DBB201220DF1070104F10C008DF807305A
:106BC80034F0F9FB002002B010BD034B6FF08502D2
:106BD800FDF784FB1A50F5E70C0000001FB50023F1
:106BE8000190CDE902334FF0FF324FF0FF3301A996
:106BF800024838F001FF05B05DF804FBC811002415
:106C080008B54B78FF2B07D14B882BB9CB881BB91C
:106C1800FFF7E4FF002008BD034B6FF08502FDF786
:106C28005DFB1A50F6E700BF0C0000002DE9F041AB
:106C380017460E460446006835F096F931463A463E
:106C48008046FFF737FFD4F87B3005460146DB1B4B
:106C58002068C4F87B3034F0ECFE88B10B4A434618
:106C680001210B4834F07CF93146204635F02AFAE8
:106C78002846FDF7CFFE2046BDE8F04135F0DEB9E5
:106C8800A37F0133A377BDE8F08100BF67EC050857
:106C9800682605082DE9F84F0446006835F079F9AB
:106CA8004FF030090746E37F012B1ED82368D3F83D
:106CB80010B0D3F804A09BF8616009FB06B624362F
:106CC800304635F0F3FA314602468046504635F0F4
:106CD80076F99BF81F30054633B1A8EB0002314620
:106CE800504635F06CF905460DB9BDE8F88F2046D9
:106CF80035F022F92A46014606463846FFF7DAFEFD
:106D080005460146206834F094FE80B10A4A3B46A5
:106D180001210A4834F024F92846FDF77BFE314664
:106D2800204635F0CFF9BDE8F84F35F087B9E37F55
:106D38000133E377B7E700BF67EC05086826050865
:106D48002DE9F04FBE4F89B04FF0FF324FF0FF33BF
:106D580005A9BC4808F0ECFF059E069D3469002D86
:106D680040F0998004F12406257794F820309D425C
:106D7800C0F28B8004F11803BFF35B8F53E8002F38
:106D880022F0020243E800210029F7D1BFF35B8F0C
:106D9800BFF35B8F53E8001F21F0040143E80012A2
:106DA800002AF7D1BFF35B8FBFF35B8FA369BFF3F3
:106DB8005B8FDB07C8D5237F022B00F08F81032B65
:106DC80000F0888153BBDDF814A0DAF81050EB7F8F
:106DD80023BB504635F0DDF88146284635F0ACF83F
:106DE8004FF40072014606464846FFF763FE8046A8
:106DF8000146504634F01DFE002800F06781924A93
:106E08004B460121914834F0ABF84046FDF702FEAD
:106E18003146284635F056F935F010F9A37F002B96
:106E280092D1237F012B40F07E81302394F861506A
:106E380004F1630694F8621003FB054530462435D7
:106E480000F060FA314602462369284600F078FAD5
:106E58000646C4F88400284635F01EFA81462846BE
:106E680035F01FFA8046284635F020FAE26D3044A6
:106E7800002A40F03C81002840F03481284635F053
:106E88003CFA003818BF01202DE130460135303674
:106E980035F0F9F969E7DDF81C80D6F804A095F813
:106EA8001890B8F1000F22D02B8A18F1710F67489B
:106EB80008BF0221009318BF01214B460CBF644A4A
:106EC800644A34F057F895F81880304635F061F880
:106ED800804540F0EF80E37F013BE3776969204616
:106EE80035F0F0F82946504634F0BBFD5CE73046F3
:106EF80035F04FF8484540F09580237FD5F80C8051
:106F0800B5F810B0002B49D1BBF11F0F42D1D8F80A
:106F18000030BB423ED1414604F1540308F11C0243
:106F280051F8040B914243F8040BF9D10A881A80EE
:106F38008A7842219A705523E26D84F8733053237E
:106F4800C4F87B2084F8743084F87630A36D84F814
:106F58007510C4F877300023C4F8803094F8603096
:106F68009A060FD194F8612094F820309A4209D2F9
:106F780094F86230013B0F2B04D8012384F87F304A
:106F88002377A0E7206834F0FAFF022384F87F30E3
:106F98000423F5E7204635F051F894E7032B92D106
:106FA800302394F8619003FB0949D4F880305B449E
:106FB80009F12409C4F88030BBF1000F16D0484607
:106FC80035F074F990B141465A46484635F080F993
:106FD800804628B9204A5B4602211C4833F0C0FF8E
:106FE800D4F87B30A3EB0803C4F87B30D4F88020B6
:106FF800E36D9A420DD2484635F058F900287FF4DF
:1070080062AFD4F88020E36D9A4202D2206834F04F
:10701800CCFF484635F071F9003818BF012084F8D4
:107028007F00B5E795F81890304634F09DFF81450C
:107038007FF449AF237F052B10D184F81C8042E7E9
:1070480055534243C811002467EC05086826050813
:10705800C6EB0508EAEB050805ED0508022B7FF4E9
:1070680032AF2A8A4FF03009D4F8803094F8618022
:107078001344C4F8803023681969D3F804B091F830
:10708800613009FB031124310846039135F00EF9EC
:1070980003990246584634F092FF00287FF413AF54
:1070A800D4F87B3013B1206834F069FF09FB08403D
:1070B8002430AFE795F81880304634F055FF804506
:1070C80002BFA37F03F1FF33A37707E7EB7F013309
:1070D800EB77A3E62046FFF7DDFD9FE6204635F077
:1070E80001F89BE6022084F87F0004231AE094F953
:1070F800601040B90029206802DA34F040FFBDE68C
:1071080034F053FFBAE6002914DA904202D8B9F1F4
:10711800000F06D1206834F032FF022384F87F3054
:10712800E3E702232377237F022B0ED1204634F096
:10713800D9FF09E6904202D8B8F1000F03D12068C0
:1071480034F033FFE9E70323ECE7032B03D12046B0
:10715800FFF7A0FDF8E5042B7FF4F6ADA37F2BB174
:107168001D4A01211D4833F0F2FEEDE5206834F098
:10717800FBFE8046204634F0DFFE04F1730305462B
:10718800024604F17F0153F8040B8B4242F8040BCA
:10719800F9D11B782946404613700D22FFF78AFC67
:1071A80006460146206834F044FC78B10C4A434650
:1071B80001210A4833F0D4FE3046FDF72BFC29465E
:1071C800204634F07FFF34F039FFBDE5A37F01335B
:1071D800A37705232377B7E52BED0508682605086F
:1071E80067EC0508802938B50D46144621D0832957
:1071F8000DD019BB80230320117153718323937120
:107208000023E070043065702370A37038BD02233A
:10721800137101235371002393710A23D371082238
:107228004168A0184AF078FD064B0E201B8823827F
:10723800E6E7044B02201B889380E1E76FF08500A6
:10724800E4E700BFC23D06082DE9F041876906461C
:10725800D0F82480BA4228BF3A46B2FBF8F4C26993
:107268002346006833F0F7FF0546C0B9B7FBF8F7C7
:10727800A7420BD1002205213068FCF72FFB28B16B
:1072880001250A4A01210A4833F061FEF3692344C3
:10729800F3613DB1074B0020B362BDE8F0810024E3
:1072A8000125E7E7706A6043F7E700BF4CED050882
:1072B800682605080203000C81420B4607B509D36E
:1072C8000D4A02210D4833F04BFE6FF0150003B054
:1072D8005DF804FB6AB101391144814201D28B4245
:1072E80007D90221009305481346054A33F042FEA8
:1072F800EBE70020EBE700BF63ED0508682605080B
:107308007AED05080C290346084616D11B78252B6B
:1073180012D009D8122B10D8084A42FA03F313F0F6
:10732800010F08BF0620704703F0FD02282A03D08A
:107338005A2B08BF0A2070470A207047F6FFFBFF48
:107348002DE9F041984690F82C3086B0062A23F0B3
:107358000C0304460F4680F82C304FF0000383617D
:10736800C0E904330B7840F010810BBB4B795B0705
:1073780024D490F82C309F070DD402234FF4685280
:107388001946002584F8283084F829106285284693
:1073980006B0BDE8F08134F0E4FE0028EDD100230A
:1073A80019461A46EDE70223052145F20232E8E7BD
:1073B800032B36D14E7916F0040604D0022305219A
:1073C8004FF41052DDE790F82C308DF8076043F049
:1073D80004038DF808608DF8096080F82C3070235C
:1073E8000D7901A9ADF8043090F82930122D8DF8E7
:1073F8000A6003F00F0328BF122503968DF80630A4
:107408000A232A46ADF812608DF80B30438D4046AA
:10741800ADF814605BBAADF810304AF01FFCA662F4
:10742800B5E71B2B00F0898009D8122B1AD01A2B2C
:1074380061D0B64A0121B64833F092FDBEE71E2B53
:10744800F7D14B795E07B9D40B7913F0030300F039
:107458009780012BA3D190F82C3043F0010380F8DA
:107468002C309CE74B795E07A8D490F82C3043F079
:10747800040380F82C304A7812F002061FD1D50791
:107488008B7822D5B1F80350424619466DBAFFF7FA
:10749800A9FEADB285420BDAB7F803506DBAADB2AA
:1074A80000231A4684F8283084F8296062856EE73C
:1074B8004246B9782046FFF795FE051EF0DA02230A
:1074C80005264FF410520025ECE72BB1914A022112
:1074D8008F4833F045FDF2E7B1F80350414634F0E8
:1074E80076FE6DBAADB2232DD6D941462046242565
:1074F80034F06DFED4E74D7915F004057FF45EAFE6
:1075080090F82C3043F0040380F82C308B783F2B14
:107518000ED1CE78002ED2D10D79032301A9404691
:10752800042D019328BF04252A464AF097FBB7E7A4
:10753800022305264FF41052B4E74B7959073FF55B
:107548003DAF3B791A090CD19A070AD5DB0715D448
:1075580094F82C3003F00303032B3FF424AF0023EB
:1075680005E094F82C209707C2F34003F0D594F86F
:107578002C2063F3410284F82C2010E70123F6E75E
:1075880090F82C2063F30002F5E70A2A7FF451AF44
:107598002A2B1BD8222B7FF64CAFA3F12302072AF4
:1075A8003FF647AF01A151F822F000BF2B76000843
:1075B8003B740008AD7600083B7400083B74000873
:1075C800217700083B740008797700085A2B7FF46C
:1075D80030AF4D7A15F004057FF4F0AE90F82C30FA
:1075E80043F0040380F82C308B783F2B40F0E38085
:1075F800CE78002E40F0DF804FF4C0634046CDE9DE
:107608000136B1F8075001A96DBAADB2082D28BFEF
:1076180008252A464AF022FB3246334684F82820B9
:1076280053E07B7A13F004037FF4C8AE90F82C2063
:1076380001AEADF8043042F00402B370082380F8BC
:107648002C208DF8073034F08CFD00283146404658
:10765800ABBF236A4FF0FF3302220322A8BF1BBA35
:107668008DF80C200293636A1BBAC3F307228DF8C6
:107678000D30C3F307438DF80E208DF80F3094F8C2
:107688002C3043F0040384F82C30B7F807506DBA57
:10769800ADB20C2D28BF0C252A464AF0DFFA00238C
:1076A800A36274E67E7A16F004067FF487AE90F83B
:1076B8002C3043F004039D0780F82C3009D40226AF
:1076C8004FF46853002584F8286084F8296063859E
:1076D8005DE634F046FD0028F1D1236AA3B1013BF1
:1076E8001ABA1B0622F07F4294F82C001343616AF1
:1076F800082540F0040009BA84F82C00C8F80030C6
:107708000023C8F80410DEE71A46EDE7C1ED0508C6
:1077180068260508A4ED05087B7A58073FF54EAEA4
:1077280094F82C30D7F8026043F00403B7F80750F8
:10773800990784F82C307FF520AE204634F011FDEF
:1077480000287FF41AAE6DBA36BA206AADB2314657
:107758002A46FFF7B1FD20B1022305214FF4045258
:107768000FE6174B2361636AE6616B43A36116E674
:107778007B7A5A073FF522AE90F82C30D7F8026092
:1077880043F00803B7F8075080F82C309B077FF5C3
:10779800F4AD34F0E6FC00287FF4EFAD6DBA36BAEC
:1077A800206AADB231462A46FFF786FD0028D3D1BC
:1077B800044B6361D7E7022205264FF410532DE7E7
:1077C8003BC203085172000807B5084A92E8030053
:1077D800CDE9000106488268126822B169469047DF
:1077E80003B05DF804FB6FF05700F9E78826050839
:1077F8004C20050800F01F0201215F2801FA02F25F
:1078080008B5034605D90C480C4A33F0A9FB0020FB
:1078180008BD1F284FF0B04106D8D1F888309A43E8
:107828000CBF01200020F3E73F2802D8D1F8983098
:10783800F5E7D1F8A830F2E740250508DCED0508A2
:1078480000F01F0201215F2801FA02F208B5034681
:1078580006D90B480B4A33F083FB6FF0150008BDBF
:107868001F284FF0B04103D8C1F888200020F6E760
:107878003F2802D8C1F89820F8E7C1F8A820F5E712
:1078880040250508DCED0508044B03EB4000002308
:10789800013320F8022B8B42FADB7047A00C00243E
:1078A8002DE9F041054600260F4F4FF00108F4B2CC
:1078B8006B78A34201D8BDE8F0812B781C442046A0
:1078C800FFF798FF68B12046FFF7BAFF57F8343042
:1078D8003BB107EBC40204F01F04516808FA04F036
:1078E80098470136E3E700BFBC350024034680B162
:1078F800B0FA80F2C2F11F02D2B2074931F9120080
:107908004FF0B042D2F880100B43C2F88030FCF739
:10791800BDBBFF22F1E700BFA00C002430B5B0B119
:10792800B0FA80F3C3F11F03DBB20B4850F83340C1
:107938008C4204D100EBC3056D68954205D044B96B
:1079480040F8331000EBC3004260002030BDFF2335
:10795800EBE76FF00F00F9E7BC35002460B1B0FA2F
:1079680080F3C3F11F03DBB2044A002142F833104D
:1079780002EBC30251607047FF23F5E7BC350024D2
:1079880000F003020F23043292009340094A43EAAD
:10799800900000F00303023352F82320030C02EA9C
:1079A800104293FAA3F008B1B0FA80F022FA00F07E
:1079B800704700BF00040058F8B5036900AF0C46D3
:1079C80003F1A005BFF35B8FD3F8A030BFF35B8F43
:1079D800C3F38003994218D1184A6E46184B88B0F1
:1079E800002918BF13466A461649CDE905134FF416
:1079F8000073ADF81C30144B42F8103F00234FF4CD
:107A0800E4511248FBF73CFCB546BFF35B8F5CB111
:107A180055E8003F43F0040345E80032002AF7D157
:107A2800BFF35B8FBD46F8BD55E8003F23F0040364
:107A380045E80032002AF3D0F6E700BF1CEE05083F
:107A480024EE05082BEE05080300000108260508AA
:107A58002DE9F0470546894690461F46D0F808A00C
:107A680034F04BFD0446D0B1067FF3070AD590F8F1
:107A7800203018480121184A33F072FA6FF0770065
:107A8800BDE8F0873B464246494634F0EEFC48B92B
:107A980094F82030114A01210E4833F061FA6FF052
:107AA8001200EDE79DF8203026F0060684F82180C4
:107AB80021466784284684F824302677DAF8183077
:107AC8009847B0FA80F3227F5B0963F300022277BC
:107AD800D6E700BF082605083DEE050857EE05085D
:107AE80070B50546866834F008FD0446D8B1037FB2
:107AF800DB0709D490F820300C4801210C4A33F0F8
:107B08002FFA6FF0770070BD0146F3692846984751
:107B180038B1237F03F00103227F63F30002227749
:107B2800F1E70346F8E76FF01200ECE708260508CE
:107B380079EE05082DE9F341D0F808801746054687
:107B48000E46D8F83C3098470022002339460B48A7
:107B5800FCF7E2FE044670B9094A3B460121094890
:107B6800009633F007FA2846D8F840309847204660
:107B780002B0BDE8F0810676F5E700BFD412002414
:107B880094EE05080826050813B503690C4691F814
:107B98002010D3F8A40036F04EFF94F8203048B1F6
:107BA800094A01210090094833F0E4F96FF0040014
:107BB80002B010BD5B0601D10020F9E7237F43F036
:107BC80002032377F8E700BFC2EE05081026050870
:107BD800F8B591F9203091F82060002B01DB0020E6
:107BE800F8BD7306FBD047684C8CB7F84830C4F32F
:107BF8000A040069A34295BF033303349B08A30812
:107C0800D0F8A440402BD4F8E80498BF5B009D004E
:107C180092B9A8424FF0000224BF401BC4F8E80400
:107C2800204691F8201001F07F0136F099FF0028D6
:107C3800D5D06FF00400D3E7BA68121AAA4207D267
:107C48000A4832460A4934F0CAFF6FF00B00C7E70A
:107C58009AB206F07F01204636F082FF0028E8D16C
:107C6800D4F8E8342B44C4F8E834B8E710260508FB
:107C7800F0EE0508F7B54668074603697468D3F857
:107C8800A450640028469834A1B2A40036F087FFB7
:107C98001022C5F8E84400212846012436F060FF88
:107CA800D5F8E8344033C5F8E83473689C420ED3FD
:107CB800284636F0CAFD054680B16FF00404024636
:107CC8001549164834F08BFF204603B0F0BDE1B2E9
:107CD80000222846013436F043FFE6E70246014613
:107CE800009040233846FFF7B3FE044628B12A46E1
:107CF8000B490A4834F073FFE6E702460090402338
:107D080080213846FFF7A4FE044608B18022EFE739
:107D18003069FCF7BBF9D7E713EF0508102605080B
:107D280028EF050838B503690446D3F8A45043681A
:107D38001869FCF7B9F900212046FFF7D1FE38B1E0
:107D48000C490D4834F050FF6FF00404204638BD4C
:107D580020468021FFF7C4FE04460028F0D12846BB
:107D680036F093FD02460028F0D00449024834F06A
:107D780036FFE9E742EF05081026050865EF050814
:107D880038B503690546D3F8A440204636F0E2FE2C
:107D9800024630B10D490E4834F021FF6FF004005F
:107DA80038BD0021142038F0C0F8204636F0D5FE42
:107DB80004460028F2D101462846FFF7FDFD224679
:107DC8000221284634F0D3FB2046E9E779EF05087D
:107DD8001026050870B5036904464568D3F8A40061
:107DE80036F01EFD024618B11A491B4834F0F7FE5A
:107DF8006668F069D8B1436898470446B8B117492E
:107E08000246154834F0EBFE002C19DB00F012FC9A
:107E1800024618B11249104834F0E1FE2869FCF70F
:107E280057F910B12869FCF73FF9002070BD0D48DB
:107E3800716983685B6843B90B49074834F0D4FE1D
:107E48000A49054834F0D0FEE0E798470028DDD01D
:107E5800F2E700BF99EF050810260508AFEF0508FF
:107E680002F005084C200508CDEF0508E9EF0508E4
:107E78002DE9F341036906464768D3F8A45000F09A
:107E8800ADFB044640B13B4902463B4834F0A7FEEF
:107E9800204602B0BDE8F0817668384896F84A3046
:107EA800D0F80880012B13D97169D8F81830083137
:107EB80053B93349304834F097FE32492E4834F0EC
:107EC80093FE6FF00404E3E7224698470028F0D1B8
:107ED800D8F8003071690BB92B49EBE72748984768
:107EE80004460028F8D196F84A30012B14D9716954
:107EF800D8F80C3008310BB92449DBE701AA1F4830
:107F080098470028F8D1019A214B9A4204D0214978
:107F1800194834F064FED0E7F06950B10368984717
:107F2800064630B11C490246134834F058FE002E6C
:107F3800C3DB40F2E4420021284649F0B6FE3B6824
:107F480028462B607B682B7140232B723B6B6B722E
:107F58007B6BEB7136F0F6FB024620B10F49064801
:107F680034F03DFEADE7284636F08FFC00288FD070
:107F7800A7E700BF20F00508102605084C200508D3
:107F88003DF00508D7F005085FF005087AF0050808
:107F9800006CDC029EF00508BAF00508EFF0050851
:107FA8002DE9F04FD0F810908BB006464568D9F807
:107FB800A48000274FF0280A4FF0400B6B68BB42A3
:107FC80056D800274FF0280A4FF0400B6B68BB4289
:107FD80000F2858099F8803023F06A0343F06A0341
:107FE80089F880306B6B2BB999F8803043F0010326
:107FF80089F8803008F5B86108F5B260C8F8E4641B
:108008000823042208F59E6837F0E3FCD5E910122E
:108018004FF0000A4FF0000B6FF007030120002714
:108028000096CDE90330CDE906AB524B4046CDE989
:10803800017708F0CFFA3168404637F073FEEB68F5
:10804800984709AA3946A86935F0AFFD041E07DB31
:10805800099B3A461979186835F0B9FD041E6BDAA0
:10806800A31C69D044492246444834F0B8FD30E0A6
:10807800EB6B0AFB07F117F0800F07F07F000B444A
:108088009A7E83F820700CBF42F0400242F0200232
:108098009A769A7E50B942F001029A76EB6B5FB1FC
:1080A800EB6BB5F848200B441A8307E022F00E0268
:1080B80042F00E029A76F3E7A3F818B0EB6B30465D
:1080C800194434F02CFA044638B12D492B4834F0C1
:1080D8008BFD20460BB0BDE8F08F01376EE7AB6B28
:1080E8000AFB07F167F07F027C060B4483F8202027
:1080F8009A7E42F020029A760BD1D2B242F0010267
:108108009A76AB6B67B1AB6BB5F848200B441A8312
:1081180008E09A7E22F00E0242F00E029A76F2E70A
:10812800A3F818B0AB6B3046194434F0F8F904469C
:108138000028CAD1013749E7A86A08B90024C8E766
:10814800283537F05BFB30B90E496FF015040B4842
:1081580034F04AFDBDE74FF4B011284634F0FEFC78
:108168000028EBD008496FF00404044834F03CFDC3
:10817800AFE700BF5D8200081FF10508102605085B
:1081880003F105083DF1050859F1050873B5D0F864
:10819800A46008460C46154634F0B8F918BB94F8A4
:1081A8002030298A802BEA680B4602D1402928BF53
:1081B8004023D018C91AE8603046298294F8201064
:1081C80036F01FFC58B194F82030084A012100907D
:1081D800074832F0CFFE6FF0040002B070BD0121F5
:1081E800204634F097F90020F7E700BF76F105083C
:1081F8001026050813B591F820300C46D0F8A400D5
:10820800DBB9537EDB071ED4538AC0F8EC34538A9B
:10821800402B28BF4023D26894F8201036F0CCFBBE
:1082280068B194F82030094A01210090084832F0DA
:10823800A1FE6FF0040002B010BD538AEBE70121E4
:10824800204634F067F90020F5E700BFA7F10508DC
:10825800102605082DE9F34703690746D3F8A460FB
:108268004FF0FF334FF0FF3201A906F5B26007F077
:108278005FFD9DF80430012B60D0022B07D0002B46
:10828800EED106F29C41384634F0A4F9E8E79DF8AF
:108298000590D6F8E48449F0800A4046514634F007
:1082A8002CF90546002134F035F9284634F052F906
:1082B80004460028D4D019F07F0F19D1038ABBB126
:1082C800402BC2684FF08001304628BF40231D462E
:1082D80036F097FB024620B13F49404834F07FFC16
:1082E800BEE7238A5B1B2382E3682B44E360B7E77E
:1082F800204634F033F9814660B1204634F032F933
:10830800E26800235146304636F07BFB02460028DF
:10831800A6D0E1E7284634F019F94A460146404616
:1083280034F031F9284634F015F90246002897D080
:108338002946D8F81000FFF729FF91E79DF8059026
:10834800D6F8E4844946BDF806A0404634F0D5F88E
:10835800054634F0FFF8044648B921494A461F4803
:1083680034F03DFC2146284634F0D4F878E75146ED
:108378000C3033F01AF8B9F1000F17D1BAF1400FE9
:1083880014D1228AD6F8EC349A420FD2E068638A74
:1083980061699B1A0244411A30465B1A95F820100D
:1083A800402B28BF402336F007FB59E7284634F016
:1083B800CDF800220146404634F0E5F8284634F06E
:1083C800C9F8024628B12946D8F81000FFF712FF6D
:1083D80046E70146C7E700BFD7F10508102605089C
:1083E80000F20508F7B591F82150012203690C46FF
:1083F80005F00305D3F8A4706B1E022B88BF002577
:10840800FFF7E6FB064698B9628C2B4694F82010D5
:108418003846C2F30A0236F071FA48B194F82030AF
:108428006FF004060090044A0121044832F0A2FDCE
:10843800304603B0F0BD00BF19F205081026050844
:1084480013B503690C46D3F8A40036F044FA40B1DA
:10845800054A234600900121044832F08BFD6FF055
:10846800040002B010BD00BF42F20508102605083E
:1084780037B5036905460C4691F82010D3F8A400D7
:1084880036F071FA024630B92146284603B0BDE8F5
:108498003040FFF79DBB94F82030054A0121009039
:1084A800044832F067FD6FF0040003B030BD00BF30
:1084B80070F205081026050873B5036905460C46D1
:1084C80091F82010D3F8A40036F0ECFA58B194F8DB
:1084D8002030174A01210090164832F04BFD6FF00A
:1084E800040002B070BD237F60F341032046237768
:1084F80034F030F8064608B90020F2E7204634F098
:1085080005F894F92030002B07DA0028F4D1324618
:1085180021462869FFF73AFEEEE70028ECD13246FB
:108528002146286902B0BDE87040FFF763BE00BF6E
:108538009AF205081026050837B50D46044636F0A8
:1085480058FA01238DF805508DF80430ADF806006F
:108558000022002301A904F5B26037F04DFA18B1E2
:108568000249034834F040FB03B030BDCAF20508A5
:1085780010260508002307B5ADF8063002238DF84C
:1085880005108DF804300022002301A900F5B2601F
:1085980037F032FA18B10349034834F025FB03B029
:1085A8005DF804FBCAF2050810260508002307B584
:1085B80001930022002301A900F5B26037F01CFAEC
:1085C800002803DA0349044834F00EFB03B05DF8D1
:1085D80004FB00BFCAF205081026050838B54FF09D
:1085E800FF324FF0FF33104807F036FD0546C8B993
:1085F8000E4A1368591C11608BB90D4CE36843F09F
:108608008073E360E36823F00073E360E3685B0171
:1086180005D400214FF47A7037F087FCF6E702485A
:1086280007F0DEFC284638BD581200240C39002417
:108638000048025810B54FF0FF324FF0FF330A4898
:1086480007F00AFD044660B9084A1368013B136045
:1086580023B9074AD36823F08073D360024807F030
:10866800BFFC204610BD00BF581200240C3900245E
:1086780000480258044A81680020D2F8603123EA91
:108688000103C2F86031704700440258074A82B0BB
:1086980083680020D2F860111943C2F86011D2F83B
:1086A800602113400193019B02B0704700440258B7
:1086B800324B10B518680B88C3F30B03132B31D852
:1086C80013B96FF0850045E0013B122BF9D801A4DE
:1086D80054F823F073870008CB860008CB8600087F
:1086E8002987000863870008CB860008CB86000826
:1086F800738700086787000873870008CB8600081F
:10870800CB860008CB8600086B8700086B870008BB
:108718006F870008CB86000851870008518700083A
:10872800174811E0D42B0FD003F62873C3F30B03BB
:108738001C2BC6D8012404FA03F3124C23420AD195
:1087480040F211142342BCD010600B68B3F5805F6F
:108758000DD2002010BD4008F6E70B48F4E70B489F
:10876800F2E70B48F0E70B48EEE70B48ECE7C3F3FA
:1087780013330133B0FBF3F01060EAE7F808002484
:1087880000366E0100101111006CDC0200B4C40444
:10879800804A5D05405489000076B010904B13B5AF
:1087A800D3F83C2142F00402C3F83C21D3F83C2121
:1087B80002F004020192019A1A6822F480221A60D7
:1087C8001A6842F480321A601A689403FCD51A6851
:1087D80042F480521A60824A13689804FCD5002338
:1087E8000093804B9A6942F440429A619A6902F474
:1087F80040420092009A9A699104FCD5784B1A6914
:108808001A6902F03802182A16D11A68520706D4D3
:108818001A6842F001021A601A685407FCD5704BB6
:108828001A6922F007021A611A6912F0380FFBD18F
:108838009A6922F00F029A61694B1A6822F08072D5
:108848001A601A6822F080621A601A6822F0805250
:108858001A609A6A22F0030242F002029A629A6A45
:1088680022F47C7242F0C0029A62DA6A22F00C02A8
:10887800DA62DA6A42F00202DA621A6B6FF308020D
:1088880042F48B7242F001021A63DA6A22F00102A2
:10889800DA621A6B22F47E4242F400721A63DA6AD0
:1088A80042F48032DA621A6B22F4FE0242F4C022E9
:1088B8001A63DA6A42F40032DA621A6B22F0FE4274
:1088C80042F080721A63DA6A42F48022DA621A6825
:1088D80042F080721A601A689001FCD59A6A404C7E
:1088E80022F07C7242F400029A62DA6A22F4406250
:1088F80042F48062DA62DA6A22F40072DA621A6C8E
:108908006FF3080242F03B021A64DA6A22F48072BA
:10891800DA621A6C22F47E4242F400721A64DA6A4D
:1089280042F48002DA621A6C22F4FE0242F48032C7
:108938001A64DA6A42F40002DA621A6C22F0FE4221
:1089480042F098521A64DA6A42F08072DA621A685F
:1089580042F080521A6023689900FCD5224806F03C
:10896800A5FEA3691E4A23F47063A361A36923F0DB
:108978000F03A361E36923F0700343F04003E3614D
:10898800E36923F4E06343F48063E361A36923F0BC
:10899800700343F04003A361236A23F0700343F09C
:1089A80040032362236923F0070343F00303236191
:1089B800136903F03803182BFAD10A4B9A6942F469
:1089C80040429A619A699204FCD5054A00201369CD
:1089D80023F400431361054B034A1A6002B010BD2B
:1089E80000440258004802580076B010F8080024E5
:1089F800132808D8054BC34013F0010F0CBF6FF0C4
:108A08008500002070476FF08500704732C70D0061
:108A180008B5074836F0F2FE38B10648FBF7B6FE4F
:108A28000448FAF71DF9002008BD6FF01200FBE7B3
:108A38007C220508418A00080A2838B50446074DF3
:108A480004D1AB680D2128465B689847AB68E1B252
:108A580002485B689847204638BD00BF7C2205085D
:108A6800034610B4DA880C46006802F0400219790F
:108A7800224383689C6934B1054BA44610BC13405B
:108A880002F0B07260476FF0570010BC704700BF2B
:108A98004000000603460A46F0B41979DB880068EE
:108AA80013430A4A012506699A4305FA01F5346811
:108AB80008BF83F44023876823F48012DB074CBF88
:108AC8002C43AC4334603B68F0BC184701001000ED
:108AD800034637B5D0F8D00070B193F8D440056993
:108AE800836801A95B689847031E08D010DA0A4A10
:108AF80002210A4834F0ABF9012003B030BD2A68DE
:108B0800019B53400122A2401340003B18BF0123A0
:108B1800181E18BF0120F0E716F30508E825050818
:108B280008B5836E034A0121034834F090F96FF0C9
:108B3800040008BD34F30508E8250508F8B50369FD
:108B48000D4616464FF0FF321C694FF0FF33271DC4
:108B58003434384634F090F9AA192946204605F0ED
:108B6800E1FB034658B16FF00404084A01210848A4
:108B780034F06DF9384607F033FA2046F8BD204640
:108B880036F04CF80428FAD10024F3E762F305081C
:108B9800E825050810B501210446D0F8E40034F0B2
:108BA80088F9034630B1862804D0064A02210648CF
:108BB80034F04DF904F1D8004FF4B011BDE810407D
:108BC800FFF768BF7EF30508E825050838B50446B1
:108BD800343035F0FEFF05460D48D4F8E0108368C0
:108BE8005B6803B198472DB12046FFF799FF6FF0F6
:108BF800040038BDD4F8D03013B1204634F044F91D
:108C0800204634F065F901230020C4F8B030F0E7BD
:108C18004C20050870B505690446D5F8E80036F01B
:108C2800EDFDE8B12E46204656F8043B9847012250
:108C38003046114636F0E0FF0122002105F11C0004
:108C480036F0DAFF05F1B400094937F02DF8284667
:108C580034F03EF907480461BDE87040FAF792BE67
:108C6800054A0121054832F072F96FF0120070BD13
:108C7800E5CE0308F0050024A6F30508E825050855
:108C8800F7B503691D69D5F8D800A8B105F1D8046E
:108C980036F0B4FD20B96FF00404204603B0F0BDEF
:108CA8004FF4D0112046FFF7F5FE0028F3D14FF41A
:108CB800FA70002137F039F90021D5F8E40034F0D2
:108CC800F8F8041E03DA284634F002F9E5E7D5F887
:108CD800D000B0B336F092FD68B395F8D4300122D5
:108CE8004F4905F1C40702FA03F3D5F8D000C5E9E6
:108CF80032138368DB690BB339469847044600286A
:108D0800E1D105F1D0064FF480313046FFF7C2FEBD
:108D1800044650B94FF0E8613046FFF7A1FE04461B
:108D280078B100213046FFF7B5FE3946D5F8D000B6
:108D380034F0A4F8C7E76FF01204C4E76FF05704E3
:108D4800C1E72846FFF7C4FE60B902236FF012049A
:108D5800C5F8B030D5F8D030002BB4D0284634F060
:108D680093F8B0E72F4C0127D5F8E010A668C5F8AE
:108D7800B0700831B36963B92B4A6FF0040401215C
:108D88002A4832F0E4F82A4A0121284832F0DFF86C
:108D9800E0E70022204698470028EDD1D5F8E010FA
:108DA800F36808310BB9234AE7E701AA2046984738
:108DB8000028F8D1019B204A934207D01F4A394620
:108DC8001A486FF0850434F042F8DCE73368D5F8C8
:108DD800E01073B12046984704460028D3D1D5E95E
:108DE8003A018368DB683BB19847044638B1144AB6
:108DF800CAE76FF05704C6E76FF05704F7E705F1C5
:108E0800340035F01FFF40B1AB6E0E4A0121074810
:108E18006FF0040434F01BF89CE7C5F8B0003CE799
:108E28005BCE03084C200508C5F30508E8250508AE
:108E38002DF40508E9F30508006CDC020FF40508B9
:108E480043F405085EF405082DE9F84399460369DB
:108E58000D4616461C694FF0FF324FF0FF33271DB1
:108E680004F13408384634F007F84B4632462946B0
:108E7800404605F095F9034668B904F11C004FF027
:108E8800FF324FF0FF3333F0F7FFD4F8B0407CB136
:108E98000A4A234600E00A4A6FF0040401210948FF
:108EA80033F0D5FF384607F09BF82046BDE8F88335
:108EB800404635F0B3FE0428FAD1F3E7A2F40508DA
:108EC8008AF40508E82505082DE9F8439946036959
:108ED8000D4616461C694FF0FF324FF0FF33271D31
:108EE80004F13408384633F0C7FF4B46324629466A
:108EF800404605F0B7F9034668B904F11C004FF085
:108F0800FF324FF0FF3333F0B7FFD4F8B0407CB1F5
:108F18000A4A234600E00A4A6FF00404012109487E
:108F280033F095FF384607F05BF82046BDE8F88334
:108F3800404635F073FE0428FAD1F3E7CCF405086F
:108F4800B3F40508E82505082DE9F8431C46D0F8D0
:108F580004809B88D8F800500B440669089FAB42F0
:108F6800D6F8B80005D8E388D8F804C01344634598
:108F780007D91948194934F083F86FF01500BDE88E
:108F8800F88396F8AA3005FB02114FF0000901FB9F
:108F98000305E2881FFA89F39A4201D80020EEE718
:108FA800A388294696F8AA2038465A4348F056FE20
:108FB800A18896F8AA305943384609F10109FBF708
:108FC800F9F996F8AA30D8F8002002FB035522894F
:108FD80003FB0277DDE700BF38250508FCF4050828
:108FE8002DE9F843099F1D460646894690469DF897
:108FF800203004693FB92248224934F041F86FF023
:109008001500BDE8F883D4F8EC2032B11C481E499D
:1090180034F036F86FF00F00F3E733B91B491848FE
:1090280034F02EF86FF05700EBE715F0040101D08B
:109038001749F4E7AB0702D5204604F047F80123A7
:109048003B6084F8FC30C4E93B69C4E93D853B6872
:10905800C4F800312368196C21B1196C226B914254
:1090680008D2196CC4F804115B6C9BB2994203D8FE
:109078000020C6E70021F5E7204604F027F8F7E7C7
:109088003825050824F5050857F505088DF5050860
:10909800D0F5050898B5406800AF046B036924B99A
:1090A80023B96FF05700BD4698BD33B10121103088
:1090B80033F07EFF0028F6DB14B3204636F09EFB23
:1090C8000346B0B921686C4688B06A460D48CDE9B8
:1090D80005014FF40071ADF81C100B4942F8101F40
:1090E8000A484FF4E251FAF7CBF86FF01200A546A0
:1090F800D9E7A3685B68002BD3D020469847D2E70E
:109108002046D0E70FF605080300000138250508BA
:10911800F7B5456807460669AB6873B14FF4D011D7
:1091280005F1080033F029FF041E06DA34493548F2
:1091380033F0A6FF204603B0F0BD2B694BB14FF4C6
:10914800B01105F1100033F018FF041E01DA2E49A2
:10915800EDE701AA0021A86A34F027FD041E07DB09
:10916800019B00221979186834F031FD041E01DAD8
:109178002649DCE72648A96983681B6823B1984714
:10918800041E04DA2349D2E76FF05704FAE7D5E959
:1091980008018368DB6803B198471023A6F8A83054
:1091A800022386F8AA300122002106F1BC0036F01D
:1091B80023FD012206F1D400114636F01DFDEB6AAD
:1091C80038469847144A3046136823F00D03136055
:1091D80034F09FFF04460028ACD1024606F138015E
:1091E800304634F0F4FF04460028A3D13268D2F8A0
:1091F800043123F00103C2F80431084B186499E7DD
:109208002BF60508382505085FF6050896F60508C3
:109218004C200508B0F60508004000520010005028
:1092280098B5406800AF046B036924B923B96FF09F
:109238005700BD4698BD33B10021103033F0B8FE59
:109248000028F6DB14B3204636F0D8FA0346B0B946
:1092580021686C4688B06A460D48CDE905014FF48F
:109268000071ADF81C100B4942F8101F0A484FF462
:10927800E251FAF705F86FF01200A546D9E7A3689E
:109288001B68002BD3D020469847D2E72046D0E76A
:109298000FF6050803000001382505082DE9F843F5
:1092A800D0F804801D46B3F80490D8F8006009EBA4
:1092B8000103089FB34207D8B5F806E0D8F804C000
:1092C80002EB0E03634507D93348344933F0D8FE1F
:1092D8006FF01500BDE8F883046952EA010094F8BC
:1092E800AA3030D14E452ED1F4452CD12889B04230
:1092F80029D10CFB00F138465943FBF75BF8D4F849
:10930800B830BB421DD004F1BC05284606F0CAFEA1
:1093180023680122C4F8B470DA632268536B43F0FF
:10932800010353634FF0FF334FF0FF32284606F036
:1093380093FED4F8EC3023B92268536B23F0010371
:1093480053630020C6E75E434FF000094B4302FB1E
:109358000632D4F8AC601644EA881FFA89F39A42B8
:10936800EFD9AB88394694F8AA2030465A4348F0DA
:1093780075FCA98894F8AA305943304609F10109C7
:10938800FBF718F894F8AA30D8F8002002FB036617
:109398002A8903FB0277DFE738250508FCF405086E
:1093A800F8B5066905460F4606F1D4044FF0FF33B9
:1093B8004FF0FF32204606F04FFED6F8EC30AB42B5
:1093C80009D00C490C4833F05BFE204606F008FE35
:1093D8006FF01500F8BD012F01D00849F2E71C22F3
:1093E800002106F1EC0048F060FC204606F0F8FD8C
:1093F8000020EFE7D7F605083825050804F7050823
:10940800064A11680B6823F004030B60044B50688C
:10941800196883685B6803B1184770471007002410
:109428007C070024094B10B5D3E90040084B1968A4
:1094380083681B6803B19847236843F004032360DB
:10944800236843F00803236010BD00BF1007002401
:109458007C07002408B5EFF31181102383F31288E9
:10946800BFF36F8F094B012093F8482083F8480019
:1094780081F31188BFF36F8F32B9FFF7D3FF502004
:10948800BDE80840FAF702BE08BD00BF1007002477
:10949800F8B58378C678EFF3118E102484F3128818
:1094A800BFF36F8F057890F801C05B1B2C463340E3
:1094B8009A4288BF9AB2AF18374007708EF3118866
:1094C800BFF36F8F8F188F421BD165450CD1EFF317
:1094D8001181102484F31288BFF36F8F04784470CD
:1094E80081F31188BFF36F8F01799B1A94B2994267
:1094F80005D336F011FC68B1084806F013FF204682
:10950800F8BD00EB040E01349EF805E0344001F884
:1095180001EBD8E7FFF79EFFF1E700BF48070024FB
:1095280070B50D4614460CB9204670BD4FF0FF3299
:109538004FF0FF330B4806F08FFD224629460A48B4
:10954800FFF7A6FF064630B94FF0FF324FF0FF3362
:10955800064806F081FDA41B0248354406F040FD8C
:10956800A4B2E0E7180700246E070024300700249F
:1095780010B54368046932486060196883681B68DD
:1095880003B19847012204F10800114636F034FB74
:109598000122002104F1200036F02EFB04F13800EE
:1095A800284936F081FB07230022502084F86130D7
:1095B8000423114684F85E2084F862300F2384F86F
:1095C8005F2084F84C300C2384F8602084F849200C
:1095D80084F84A2084F84B2084F84D3031F065FE39
:1095E800194B1A481B681A491A68196122F07C42FB
:1095F8001C6922F0FF02824203D147F2AC20844268
:1096080012D0186820EA0200124A02431A6047F290
:10961800AC221961196119611A611A6822F0804235
:109628001A601A685200FCD41A6842F004021A60E0
:109638001A6842F008021A60FFF70CFF002010BDFC
:109648004C2005085FD1030810070024000DF00026
:10965800BC0A5917000DF0401D4B014610B51B6898
:10966800EFF31184102282F31288BFF36F8F5A68C8
:10967800500605D45A68D2071DD46FF00A0015E0C9
:109688001A6842F080421A601A6822F080421A6012
:109698000A221868400005D45868400602D4586861
:1096A8004007E7D5013AF4D16FF0040084F311883C
:1096B800BFF36F8F10BD5A689207F5D4586810F041
:1096C8004000F1D19B680B60002BEFD1D5E700BFBC
:1096D800100700242DE9F743D8078846144605D417
:1096E8003148FFF7D5FE03B0BDE8F083002A37D034
:1096F800EFF31185102383F31288BFF36F8F502087
:10970800FAF7E6FC06465020FAF7CEFC85F31188F6
:10971800BFF36F8F0EB9FFF785FEDFF89090D9F889
:1097280000305A68510713D45B685A0610D4204F8A
:109738004FF480332546C7F88831D9F800305B6884
:10974800DB070FD4BFF34F8F20BF40BF20BFF4E724
:10975800002401A8FFF780FF16B35020FAF796FC03
:109768002046C0E701A8FFF777FF4FF48032034691
:10977800C7F8882188B9291F019A89B2002DEBD032
:10978800A94203D1002BD8D00192D6E7013D01238D
:10979800ADB208F80520120AF0E7002DCDD1DBE7BD
:1097A800FFF72EFEDCE700BF59070024100700244E
:1097B80000E100E02DE9F74301A8FFF74DFF00287D
:1097C80043D1284C0427019A804694F84B3001462F
:1097D80094F84CC094F84AE0A3EB0E055FFA82F9BE
:1097E8003CEA05051ED194F8601094F85F6094F87F
:1097F80061508E1B35EA06062AD108B184F84B3031
:10980800B8F1000F00D001925020FAF74DFCFFF795
:10981800F7FD002384F84830134803B0BDE8F0434F
:1098280006F0DEBBE018013380F84E900CEA030323
:109838000120013F4FEA12224FF00108CCD108B1B4
:1098480084F84B3001920029E6D103B0BDE8F083DB
:10985800661801310D4086F86390012184F8605044
:10986800E7E700BF1007002430070024C3780F2B58
:1098780014D9C96B0B480B0E00EA911013708B02B8
:10988800090603F47C0301F0FE41034300200B4367
:1098980011686FF31E210B43136070476FF085004A
:1098A800704700BF00FF0300F8B50D4616460021BB
:1098B8005022044648F0F9F9A5F10803A91E5842B8
:1098C800C9B25841022E11BF002308234FF0006689
:1098D8004FF400670FBF4FF000521E461F461A464E
:1098E80006294FEA001016D80E4DDFF83CE015F8AF
:1098F80001C00E4D35F811505EF8211063614FF428
:109908004053E561A1632664A264C4E903C0C4E9C5
:1099180008372046F8BD4FF080714FF480754FF03E
:10992800010CEBE735400608DC2A050888D605084F
:10993800004870475C2B0508002370B5C0F8AC30B0
:109948000446154634F04BFE38B1104A0121104840
:1099580033F04AFD6FF0040070BD0A2304F1740669
:10996800A5FB0323304606F077FB58B1094A0121CD
:10997800074833F039FD204634F0A2FE304606F0A1
:1099880091FBE7E7D4F8AC00E6E700BF73F70508FA
:109998005025050888F7050870B59AB00E46144694
:1099A80005461422002101A848F07FF906A822469E
:1099B8003146FFF779FF082E41F2883206A90DBF1C
:1099C80040F2F96306200123089318BFCDE9080384
:1099D800002328460D931493179334F0BAFC0346DA
:1099E80040B1214A2148012133F0FEFC6FF0040008
:1099F8001AB070BD082E19D140F2FA53022C4FF458
:109A080080604FF0806108931CD0042301241793D1
:109A180000230D9041F288321491284606A9159426
:109A28000C9334F096FC78B1114ADBE7052101224A
:109A3800022C4FF48070CDE908124FF08071E6D007
:109A48001446E4E70523E2E702231022039001A964
:109A58002846CDE901334FF48003CDE9043241F2C1
:109A68008832FFF769FFC3E7A2F705085025050804
:109A7800C5F7050870B59AB00E46144600211422A1
:109A8800054601A848F011F92246314606A8FFF715
:109A98000BFF082E21D140F2FA53022C08932AD04A
:109AA8000423012417930023102215940C934FF4D8
:109AB8008003012406A928460294CDE9043241F224
:109AC800883234F046FCC0B10F4821460F4A33F0C3
:109AD8008BFC6FF004001AB070BD052301224FF013
:109AE8008071022CCDE908324FF0000314910D93D8
:109AF800D8D01446D6E70523D4E741F2883201A925
:109B08002846FFF719FFE6E750250508E9F7050895
:109B18002DE9F041D0F8048094B004690F46154649
:109B280098F81C1098F8202068461E46FFF7BCFEDF
:109B3800D8F81C30082B1AD145F6A5231422029315
:109B48004FF440531192694641F2883220460893F7
:109B580006970F9634F0FDFB0246B0B11149124842
:109B680033F052FC6FF0150014B0BDE8F0815A22B2
:109B78000123CDE902234FF0807308220E934FF49E
:109B8800807307934FF40053DCE741F2883229468B
:109B9800204634F075FC024608B10449DFE7C4F8F2
:109BA800AC00E1E706F80508502505082AF805087D
:109BB800002208B5C0F8AC2041F2883234F0C9FB65
:109BC800024628B103490448BDE8084033F01CBCEC
:109BD80008BD00BF06F80508502505082DE9F04F17
:109BE8008046B3B00F461446002A3BD046687269D7
:109BF800A242154628BF254600292ADBCB1749195A
:109C080043F100038A424FF00001994121D3C5F383
:109C18000B035BBBD8F81090484633F0FAFB502290
:109C280000210AA848F041F896F82020317F4846DC
:109C3800FFF720FF044618B36FF00F04864A01218E
:109C4800864833F0D1FBD8F810005C3033F0CAFBFB
:109C580008E06FF015043B46814A01217F480095D2
:109C680031F088F9204633B0BDE8F08FA242D1D94F
:109C78007C492A4679486FF0850433F0C5FBF1E743
:109C8800F369082BA3F1080A14BF012204220D92DC
:109C9800326AA2F1020EDEF1000242EB0E02DAF1A4
:109CA800000343EB0A03D2001B010F920E93002D11
:109CB800C9D0002CC7D196F820204846317FFFF73D
:109CC8006BFE044628B1684A0121644833F08CFBD6
:109CD800B9E77269F369AA4263D1082B46F29F0378
:109CE8000AA9109018BF60231190D8F810000C939F
:109CF800FFF75EFF73692146D8F81020ED1AD8F8EF
:109D080004300392142293F81CB093F820A00DEBB2
:109D1800020047F0CAFF594652461EA8FFF7C4FD85
:109D2800BBF1080F22D140F2FA52BAF1020F209289
:109D38002AD0042401232D9300232F941024249344
:109D4800022341F288321EA906934FF48003039838
:109D5800CDE9083434F0FDFAD0B16FF00404434A79
:109D680001213E4833F040FB414AADE74FF0050C76
:109D780001224FF08071BAF1020F25942C91CDE9A0
:109D880020C203D15346D6E70524FBE71346D2E7A2
:109D9800384A05A90398FFF7CFFD0446002886D066
:109DA800E2E7082BD8F8100009F19C0E109714BFB1
:109DB8004FF480734FF480631193336A9A1E5342B1
:109DC8005341DB02139390F89E30042B09F194035E
:109DD8000CBF4FF4405C4FF4005CCDF848C05A7893
:109DE80072B14FF0FF31914037EA010108D10121EA
:109DF8009140A94204D8ECB16178914238BF1C4621
:109E080002339E45EBD1F369B4B1082B1CD02378FB
:109E18000AA90C93FFF7CCFECCB1627801239340DA
:109E28001F44ED1A96F820204846317FFFF722FE9E
:109E380004463CE71C46E3E7082B05D0BCF5405F29
:109E480014BF20232123E3E742F2DE13E0E707F5FE
:109E58008057A5F58055E5E7A5F8050850250508BC
:109E680042F8050887F80508BFF80508DBF8050873
:109E7800FEF80508E004070038B5CB630023154653
:109E880041F28832C0F8AC30044634F062FA024637
:109E980030B10D490D4833F0B7FA6FF0040038BD02
:109EA8002946204634F066FB024608B10849F1E726
:109EB8004FF0FF324FF0FF3304F1740006F0CCF896
:109EC800D4F8AC00EBE700BF06F8050850250508F4
:109ED8002AF80508F7B50D1E1C460FDB476815EB79
:109EE800030C4FEAE5767F6946F1000667454FF0B7
:109EF8000007B74102D363B9184608E007482B4664
:109F0800074A0121009431F035F86FF0150003B0CD
:109F1800F0BD03B0BDE8F04033F0A0BA5025050805
:109F280042F8050838B5154604694268CB63002332
:109F3800C4F8AC30D369082B0BD10B6AB3F5405F7A
:109F480007D0134A0121134833F04EFA6FF004008A
:109F580038BD41F28832204634F0FBF9024620B180
:109F68000D490C4833F050FAF0E72946204634F002
:109F7800E0FA024608B10949F3E74FF0FF324FF023
:109F8800FF3304F1740006F067F8D4F8AC00DFE79B
:109F980010F905085025050806F8050842F90508CE
:109FA8002DE9F04F0D1E97B0804692461E462FDBD6
:109FB8004768AA194FEAE573796943F100039142AA
:109FC8004FF000029A4123D3002E00F0AC80D0F865
:109FD8001090484633F01DFA97F82020397F02A8E0
:109FE800FFF762FCD9F8A430382B049356D041D837
:109FF800322B4BD019D823F01003022B17D1012391
:10A0080005934FF4807309934FF0807310930EE01B
:10A018006FF015042B46454A01214548009630F05B
:10A02800A9FF204617B0BDE8F08F342B2ED0D8F802
:10A0380010304846089593F89E30042B0CBF4FF417
:10A0480040534FF400530A930023139397F82020AA
:10A05800397FFFF70FFD002851D0D8F810005C3089
:10A0680033F0C0F9334A012131486FF0040433F06A
:10A07800BBF9D6E73E2B11D0A22BD8D101230593EB
:10A088004FF4807309934FF00073BFE701230593E2
:10A098004FF4807309934FF04073B7E7012305939A
:10A0A8004FF44073F6E7B6F5807FB3464FEA1522C2
:10A0B80002A928BF4FF4807B404608950BEB0503A7
:10A0C800013BB2EB132F52461CBF5FFA85FBCBF561
:10A0D800807B5B46FFF726FF044608B1164A18E066
:10A0E80097F820204846397FA6EB0B06FFF7C2FCFD
:10A0F800DA445D44044608B1104A0AE06EB197F8A4
:10A1080020204846397FFFF747FC04460028CAD07C
:10A118000B4A0121064833F067F9D8F810005C3083
:10A1280033F060F97DE734467BE700BF42F8050865
:10A13800502505085BF9050889F90508A0F90508FF
:10A1480071F905082DE9F04FD0F80480C3B0044632
:10A158000569D8F81C30082B0ED0D8F82030022B0F
:10A168000AD16FF0850BA94A0121A94833F03CF9BF
:10A17800584643B0BDE8F08F2EAA0021D8F8240035
:10A1880033F013FDB0F1000B08DB2E9B0022197988
:10A19800186833F01CFDB0F1000B05DA9D495A46EA
:10A1A8009B4833F031F9E3E79B4EB7683B683BB90E
:10A1B8009A4A0121964833F017F96FF0040BD7E754
:10A1C80041463046984702460028F1D1BB6908F15C
:10A1D80008090BB9924AECE74946304698470028E7
:10A1E800F8D1FB680BB98F4AE3E70AAA494630461B
:10A1F80098470028F7DB0A990123D8F8180040F29D
:10A208000112B1FBF3F6B04202D201339342F8D106
:10A2180004226B6228466A60D8F81420002A92FA51
:10A22800A2F34FF00202B3FA83F308BF4FF0FF33F3
:10A238002B610023AB60C5E90523C5E90733D8F8CE
:10A248002020022A0ABF4FF080731A464FF080522E
:10A25800EB600023EA62EB63C5E90C3303F022F8F4
:10A26800014608B1704AA4E718220EA847F01DFD60
:10A278002B686E4A934215D10123CDE90E33109312
:10A288004FF00113119303F57F031293012641F256
:10A2980088320EA92846139603F030F9814658B142
:10A2A800634A86E7634A9342F0D10223CDE90E332D
:10A2B800109303F58033E5E73246314605F15C003B
:10A2C80035F09AFC3246494605F1740035F094FCA5
:10A2D800D8F81030204698472769502249462EA8BA
:10A2E80047F0E3FC662341F288322EA93846CDE9CF
:10A2F800303634F02EF830B14F4A3146444833F006
:10A3080073F84E4A55E7992341F288322EA9384608
:10A31800309334F01EF808B1494AEEE7042346F2B8
:10A32800996A339041F28832319310232EA9384626
:10A33800CDF8C0A0329334F00CF808B1414ADCE7FC
:10A3480049F6661941F288322EA93846CDF8C090F0
:10A3580033F0FFFF08B13C4ACFE7082341F28832C7
:10A368002EA938463393CDF8C0A033F0F2FF08B1D8
:10A37800364AC2E741F288322EA93846CDF8C09055
:10A3880033F0E7FF039008B1314AB6E7314835F0BA
:10A398000EFA324631462846FFF76CFB08B12E4AC2
:10A3A80007E7D4F804902769D9F81C30082B16D091
:10A3B800D9F82030012B12D1182314AA00212046E5
:10A3C800FFF7A6FB8346002800F0FA806FF015021D
:10A3D80022490F486FF0150B33F016F8C8E6012232
:10A3E80038461146FFF7D8FA064600283CD01C4AE2
:10A3F8000121074832F0F8FFD8E90732012100921D
:10A408000348184A30F0B6FDD7E600BFB9F9050889
:10A4180050250508E2F905084C20050801FA050849
:10A428001DFA050840FA05086FFA050800500052A1
:10A4380080FA050800A0005295FA050867FB050890
:10A44800B8FA0508DBFA0508FEFA050821FB050835
:10A4580044FB0508A086010079FB05089FFC050858
:10A468008FFB05087BFC0508012207232EA84FF067
:10A47800720A11468DF86830FFF716FA4FF44073E8
:10A488003F96012641F288322EA93846CDF8C0A061
:10A4980034933D9633F05DFF30B1A54A3146A54867
:10A4A80032F0A2FFA44AA3E741F288321AA938463B
:10A4B80033F0A0FF0028F0D1324631463846FFF786
:10A4C800D9FA08B19D4A93E7324631463846FFF734
:10A4D80063FA834608B19A4A8AE7D9F820303246A7
:10A4E80031462EA8022B14BF012302238DF86830B1
:10A4F800FFF7DAF941F288322EA93846CDF8C0A024
:10A50800CDF8D0B0CDF8FCB03D9633F022FF08B1BD
:10A518008C4AC3E741F288321AA9384633F06AFFF9
:10A528000028F5D149F6404035F041F94FF08073E5
:10A538003846FB604FF08053FB6202F0B3FE08B16F
:10A54800814A55E7D9F820A0BAF1010F2BD152461C
:10A5580008213846FFF78EFA064608B17B4A47E7D6
:10A56800012208212EA8FFF79FF947F28E1341F226
:10A5780088322EA930930423384634963F93CDF879
:10A58800F4A033F0E6FE30B16E4A0121694832F09A
:10A598002BFF6F4A2CE741F288321AA9384633F06C
:10A5A8006FFF0028F0D1D9F82020022A7FF404AFE9
:10A5B80008213846FFF75EFA00283FF4FDAECDE7E4
:10A5C800149A644B9A4201D0634902E79DF85630C9
:10A5D80016AE012B96BF01331023DB00F318069348
:10A5E800069BB3426ED0F279337843EA0223B3F57F
:10A5F8007F4F40F0CF81F37871799B00B2790902DF
:10A608003079502B41EA02411AAA28BF502301434E
:10A618002046FFF77DFA002840F0B98127694FF0FE
:10A6280001084E4B07F1940AD4F804900B93ADF847
:10A6380024008DF82600C7F89400C7F898005FFA40
:10A6480088F108F1010852461AA832F009FEB8F15B
:10A65800050F0AF1020AF2D11A9BC3F34148236994
:10A6680008F1FF32012A50D80422B8F1010F83F80B
:10A678009E204DD10DAA1AA93046FFF7F7F80028F9
:10A6880046D19DF83430980742D0414642462EA81C
:10A698000493D4F810A0FFF707F9049B990763D532
:10A6A800424641465046FFF777F900285CDA2C4AC3
:10A6B8000121204832F098FE6FF0040229491D4814
:10A6C80032F0A2FE22696368B2F89C0002F1080524
:10A6D8005969134693F8944034B1039E93F8954012
:10A6E8000EB1B44200D2039402339D42F2D1039CCE
:10A6F8000123A3405C1E044208BF0346C2F8903001
:10A70800B1FBF3F3C2F88C3032E5032283F89E20C4
:10A71800D7F8A430FF2B47D1D9F81C30042B00F010
:10A728009780082B3CD0022B00F09480022339E05C
:10A73800A8FB050850250508B7FB0508CFFB050849
:10A74800E7FB050802FC050828FC050846FC050887
:10A758005DFC050853464450B4FC0508030604078D
:10A76800CCFC05084BFD0508B72201232EA950464D
:10A77800CDE93023002341F2883235933C933F934F
:10A7880033F0E7FD002892D10CAA0321204632F0CD
:10A7980047FE00288BD19DF83030DB0787D5B7E717
:10A7A80041F2ED23C7F8A430D9F81C30082B00F08B
:10A7B800DF8002234FF0000887F8A830032387F8CA
:10A7C8009F80C7F8A030D9F81C30012B00F0D0804A
:10A7D800022B14BF4FF0040A4FF0020A0BAB1AA960
:10A7E800304613F8082009AB049232F0C5FC002863
:10A7F8000DDB049A9DF8243087F8A820C7F8A0300C
:10A808009DF825209DF82630134487F89F3008F1DD
:10A818000108D045E2D1D9F81C30042B40F0A880BB
:10A828000CAA1AA9304632F02FFD002814DA704A13
:10A838000221704832F0D8FD2369049393F8A930B7
:10A84800062B72D8DFE803F094730F7873737300E4
:10A858003823A7E7A223A5E79DF83030C3F34203C6
:10A8680087F8A930E8E74FF040094FF001080DF1EB
:10A8780023024146204632F0D3FD002855DB9DF8DF
:10A88800233019EA0303059372D101220498114673
:10A89800FFF782F8002848DB9DF823A0502223699F
:10A8A8002EA849EA0A0A059907938DF823A047F0CC
:10A8B800FCF94FF0807201233C929845059A0D925D
:10A8C800079ACDE9303392F8A92038D19A428DF809
:10A8D80034A047D10DF135020221204632F0A0FD07
:10A8E800002822DB0DAA02232EA92046FFF71AFB17
:10A8F80000281ADB012204981146FFF7BBF800284C
:10A9080013DB0DF123024146204632F089FD002871
:10A918000BDB9DF8233019EA030F29D1364A0121B0
:10A9280000934346334830F025FB344AC0E64FF0E5
:10A9380002094FF002089AE74FF08009F9E7312140
:10A94800012A8DF835A0309102D0043A012A0CD89A
:10A958000DAA0121204632F063FD0028E5DB012322
:10A968003093BFE70DAA4346BEE70DF13502BBE7BA
:10A97800F3780A2B89BF249B4FF48073C3F3031227
:10A98800012388BF9340A7F89C30083628E66FF06B
:10A99800150293E64FF684729342F6D195F89E30ED
:10A9A800042BF2D1F37871799B00B27909023079DE
:10A9B800082B41EA02412EAA28BF0823014320465A
:10A9C800FFF7A6F800287FF47DAE0DF1BB012B46FA
:10A9D80005F1080711F8012F0233FF2A04BF0022EE
:10A9E80083F8930083F892209F42F3D1CDE700BF0C
:10A9F800E5FC0508502505080CFD050830FD05088F
:10AA080000487047642B0508044BB3F80C389B02C8
:10AA18000B60002318464B60704700BF00F0FF082A
:10AA2800064B186828B94FF4807C4FF40050C3E9EE
:10AA380000C0012010600B60704700BF103900246F
:10AA480007B503461022012104480092044A30F059
:10AA580091FA002003B05DF804FB00BF58250508F3
:10AA680081FD05080B4A5369DB0312D5002910DD67
:10AA780000F1006300F01F000144BFF34F8F20393D
:10AA8800C2F85C3220330029F9DCBFF34F8FBFF3E3
:10AA98006F8F704700ED00E037B50468256915F041
:10AAA800C06F09D0236E9BB21D4A02211D481B01AD
:10AAB8000093012330F05EFA1B4B63611B4B1D4270
:10AAC80009D00123009517480121194A30F052FA9C
:10AAD8006FF004001EE0D4F8105115F0C06F0AD0D2
:10AAE800D4F860319BB20E4A0E481B010093022332
:10AAF800194630F03FFA0F4BC4F814310B4B1D4286
:10AB080007D00D4A154207D0D4F814311343C4F8BE
:10AB18001431002003B030BD02230095D3E700BFF5
:10AB2800D3FD0508582505080F00AF1F0000AE1516
:10AB3800EEFD05080F00AF9F0000088070B50546C0
:10AB480010461A46EFF31186102383F31288BFF3D9
:10AB58006F8F012383F31388104C636943F4807368
:10AB68006361BFF34F8FBFF36F8F01F1006147F04F
:10AB780075F8002383F31388636923F48073636192
:10AB8800BFF34F8FBFF36F8F86F31188BFF36F8FBB
:10AB98002869BDE87040FFF77FBF00BF00ED00E007
:10ABA800F7B517461A4606460D461C4632F0E1FC34
:10ABB80050B90B482B460B4A0121009430F0DAF9C2
:10ABC8006FF0150003B0F0BD44B123463A4629465C
:10ABD800304603B0BDE8F040FFF7B0BF2046F1E7CC
:10ABE8005825050804FE0508F7B505463C2200234C
:10ABF800684635F040FA2869DDE90067FFF74CFF41
:10AC0800044680B902462B691B681969490703D4B1
:10AC1800D3F810315B0708D552B106230A4A01213F
:10AC28000A4830F09DF96FF00404204603B0F0BDE7
:10AC380032463B46684635F043FADDE900321343B5
:10AC48000CBF01220022DEE72EFE05085825050864
:10AC580010B503691C6829B1FFF7C6FF88B16FF00A
:10AC6800040019E0E368DA0717D4D4F80C31DB07DD
:10AC780011D50D4BC4F8043103F18833C4F80431FD
:10AC880009E0E36843F00103E360D4F80C3143F0D2
:10AC98000103C4F80C31002010BD034B636003F1BD
:10ACA80088336360E1E700BF230167452DE9F84F6A
:10ACB8000369B1F5801F9146314A1E688046926942
:10ACC80001F1006A35BF06F10C0706F586771036E4
:10ACD80006F588763C6814F0010403D06FF0040090
:10ACE800BDE8F88FFFF780FF0028F7D1DAE90023E5
:10ACF800B3F1FF3F08BFB2F1FF3FEFD1DAE902231A
:10AD0800B3F1FF3F08BFB2F1FF3FE7D13B6843F023
:10AD180002033B60BFF34F8F09EB040159F804208D
:10AD28004B680AEB0401C1E90023BFF34F8F35F0EC
:10AD3800A0F90A220023F6F791FA10F1640541F10F
:10AD4800000B33685B070FD535F093F90A2200230F
:10AD5800F6F784FA85427BEB0101F2DA6423094AAB
:10AD68000121094830F0FCF8082C07D14046FFF7CC
:10AD78003BFF3B6823F002033B60B1E70824CBE7C5
:10AD88000020005242FE050858250508013A2DE921
:10AD9800F04781468A465718DFF878801E4E574597
:10ADA80001D2002012E0D9F81030BAF5801F4FEA1E
:10ADB8005A351C68D8F818302ABF803D0C3404F581
:10ADC80086742368DB0703D56FF00400BDE8F087BD
:10ADD8004846FFF709FF0028F6D12368AD0123F4A0
:10ADE800FE5305F4FE55236023681D4345F0040512
:10ADF8002560236843F020032360BFF34F8F484644
:10AE0800FFF7F2FE2368334023600028DCD10AF5FF
:10AE1800005AC4E7002000523BE0FFFF2DE9F7434A
:10AE2800012307460C46154632F0B8FB60B9009579
:10AE38006FF0150523461D4A01211D4830F09AF888
:10AE4800284603B0BDE8F083002DF9D0386932F008
:10AE580089FB00213846FFF7FBFE18BB154E21463B
:10AE68002A46384604EA060904F5FF54FFF78EFF20
:10AE780080461E3448462C4404EA0601A1EB090129
:10AE8800FFF7F0FD01213846FFF7E2FEB8F1000FA9
:10AE980008BF0546386918BF6FF00405043005F08F
:10AEA8009FF8CDE76FF00408ECE700BF53FE0508F4
:10AEB8005825050800E0FFFFF7B51C461746012393
:10AEC800054622460E4632F069FB58B96FF0150761
:10AED8003346184A01211848009430F04BF8384698
:10AEE80003B0F0BD24B3286932F03CFB00212846AA
:10AEF800FFF7AEFEC8B93A4623463146284632F037
:10AF08005AFB074601212846FFF7A2FE002F2146DB
:10AF180008BF0746304618BF6FF00407FFF7A2FDC9
:10AF28002869043005F05CF8D9E76FF00407E9E711
:10AF38002746D4E77EFE0508582505082DE9F8437D
:10AF4800D0F80490904607460D46D9F808001E46EA
:10AF580031F01FFAB8F5001F044616D1D9F8084099
:10AF68002846FCF70DFD84420CD1294631F011FA30
:10AF7800044631F013FA2046FCF7F0FC0021204685
:10AF880031F015FA0020BDE8F883B8F5800F20D01D
:10AF9800B6F1806F19D0B6F1C06F18D0B6F1007F46
:10AFA8001AD102263A460F492046FCF7B7FCB0B939
:10AFB800D9F80810284631F023FA2046314631F0F6
:10AFC800F6F92046FCF792FCDCE70126EAE70326BF
:10AFD800E8E76FF08500D6E76FF01500D3E76FF06C
:10AFE8000F00D0E74FD703081FB50C4B0C29D3F837
:10AFF800082828BF0C2112BA0C460192D3F804285D
:10B0080012BA02920A46D3F8003801A91BBA039370
:10B0180046F024FE204604B010BD00BF00F0FF0833
:10B0280080B500AF8AB06A46094B0791CDE9053073
:10B038004FF40073ADF82030064B42F8103F002360
:10B048004FF411510448F8F71BF9BD4680BD00BF05
:10B05800D5FE0508040000017825050808B5044A4E
:10B06800012104482FF073FF6FF0040008BD00BFF2
:10B07800E9FE050878250508F7B50446436806691A
:10B088000F461C480022DD68596883680192DB6816
:10B098004BB96FF00404184A012118482FF057FFE4
:10B0A800204603B0F0BD01AA98470028F1DB3763BA
:10B0B80006F118074FF0FF324FF0FF33384604F01F
:10B0C800CBFF2B68204623F001032B6096F8621013
:10B0D80032F0B7FB2046019900F0A0F896F86130ED
:10B0E80004461BB12B6843F001032B60384604F07B
:10B0F80077FFD5E74C20050807FF050878250508E0
:10B1080070B50446466805694FF0FF3200212846AD
:10B1180034F072FD336820469847002385F8603084
:10B1280085F86230012205F11800114634F064FDFB
:10B13800204600F03FF83169184B994222D015D8C3
:10B14800174B994220D0174BCB1A594259418900C5
:10B15800204641F01001FFF78FFF041E18DA124A4B
:10B16800012112482FF0F3FE204670BD104B994282
:10B178000CD003F5C31303F5206399420CBF0A21D1
:10B188000021E5E70621E3E70221E1E70821DFE7FF
:10B198000123002485F86030E6E700BF40420F0035
:10B1A800A0860100801A060035FF050878250508E5
:10B1B80040E1330037B5456801AA0021686932F0DB
:10B1C800F4FC041E07DB019B00221979186832F091
:10B1D800FEFC041E08DA0D4A234601210C482FF014
:10B1E800BFFE204603B030BD0A48696883681B6803
:10B1F8003BB9094A012106486FF004042FF0A7FE65
:10B20800EFE7984704460028EBD0F2E766FF050809
:10B21800682505084C20050884FF05082DE9F74F27
:10B22800446803690020E5680193DFF81481E36945
:10B23800DFF81091DFF810A1DFF810B10093009B40
:10B248008342019B1A6B0DD1C2F34202012A3AD004
:10B25800022A67D03E4A3F4801212FF078FE6FF05E
:10B2680015001EE00C23D4F818C0DFF8ECE003FB4F
:10B2780000F70CEB0706736873451CD014D85345C8
:10B288001BD05B4514BF002301239B00534013F0E0
:10B298000E0F16D15CF807308B4212D1B36800202C
:10B2A8002B6103B0BDE8F08F434508D04B450CBF78
:10B2B8000A230023EAE70623E8E70223E6E7082350
:10B2C800E4E70130BBE741F25C2E4FF47A6C40F2C0
:10B2D800E2474FF4FA760220204B421EB1FBF2F20D
:10B2E800B3FBF2F2BCFBF2F4013CFF2C23D8BEFB0B
:10B2F800F2F808F1FF38B8F1FF0F1CD8B6FBF2F9E5
:10B30800B9F10F0F17D8B7FBF2F2013A0F2A12D88A
:10B31800023848EA094343EA007343EA025343EA1E
:10B328000423BCE740F2145E4FF4167C4FF4FA771E
:10B3380040F27716CFE701301128CED1084A8AE7C4
:10B3480040E13300404B4C00A0860100801A060003
:10B35800B4FF05087025050840420F0000CA9A3B53
:10B368002F00060837B5456801AA0021E86832F0C1
:10B378001CFC041E07DB019B00221979186832F0B7
:10B3880026FC041E08DA0C4A234601210B482FF03C
:10B39800E7FD204603B030BD0948696883681B682B
:10B3A8002BB19847041E05DA064A2346EDE76FF0ED
:10B3B8005704F9E70024ECE7620006089825050819
:10B3C8004C2005088000060843681B6803F1080242
:10B3D80052E8002F42F0010203F1080040E8002182
:10B3E8000029F3D1194A934223D0A2F54C42934243
:10B3F8001FD002F5806293421BD002F5806293420F
:10B4080017D002F58062934213D002F5444293426A
:10B418000FD0A2F51C4293420BD002F580629342F2
:10B4280007D002F51C42934203D002F58062934292
:10B4380003D15A6842F040025A6053E8002F42F4A0
:10B44800807243E800210029F7D1704700100140BD
:10B4580043681B6803F1080252E8002F22F001023A
:10B4680003F1080040E800210029F3D1194A93426A
:10B4780023D0A2F54C4293421FD002F5806293423A
:10B488001BD002F58062934217D002F58062934286
:10B4980013D002F5444293420FD0A2F51C429342C6
:10B4A8000BD002F58062934207D002F51C4293420A
:10B4B80003D002F58062934203D15A6822F0400219
:10B4C8005A6053E8002F22F4807243E800210029D3
:10B4D800F7D17047001001402DE9F04182B0804655
:10B4E8000D46436800AF1E68002937D058681969AF
:10B4F8008368DB686BB13A1D9847041E0CDA1B4A57
:10B5080001211B482FF023FD20460837BD46BDE822
:10B51800F0816FF05704F2E7336823F40043336097
:10B528007B6803EB5503B3FBF5F30F2B19D86C4677
:10B538008AB0D8F800306A460E490795CDE9051358
:10B548004FF40073ADF820300B4B42F8103F002346
:10B558004FF411510648F7F793FEA5466FF015040E
:10B56800D2E79BB20024F360CEE700BF07FF0508CF
:10B5780000260508EC00060804000001F8B50C4692
:10B58800036941681D682379012B18D0A3F1020EC5
:10B59800DEF1000646EB0E06B6026279022A96BF75
:10B5A800464F4FF4005737F81270A279022A09D093
:10B5B800042A2FD0003B18BF01231B0306E04FF4D9
:10B5C800C066EAE7B3FA83F35B091B07E279096807
:10B5D800012A0CBF4FF4407C4FF0000CA5421CD14F
:10B5E8000A6822F0805222F4B05232431A430A60A9
:10B5F8004B6823F440533B434B6043681A68936895
:10B6080023F4407343EA0C0393602968BDE8F840CB
:10B61800FFF762BF4FF48053D8E7D1F800E00EF48B
:10B62800C06E764506D0D1F800E02EF4C06E4EEA22
:10B6380006060E6041680E68716801F440518F4239
:10B6480004D0716821F440513943716041680E6833
:10B65800316801F010218B4204D0316821F01021AB
:10B668000B433360436819688B6803F440739C4547
:10B6780005D08B6823F4407343EA0C038B6043685E
:10B68800D71E1B687E4299687E41C1F380318E4285
:10B6980007D0032A9A680CBF42F4804222F4804201
:10B6A8009A6021682B68994205D0FFF715FF08B901
:10B6B80023682B60F8BD0020FCE700BF96D605087C
:10B6C8002DE9F04383B08046D0F8049000AFD9F854
:10B6D8000400D9F8101083681B687BB198470546A9
:10B6E80070B93A1D0021D9F8240032F05EFA051E1F
:10B6F8000EDA28460C37BD46BDE8F0836FF05705D3
:10B70800644A012164482FF022FC002DF1DBE8E7B0
:10B718007B6800221979186832F059FA051EE8DBAF
:10B72800D8F80460D8F8103034681D68236823F00E
:10B7380001032360B06834F061F838B9574A012131
:10B7480055486FF012052FF002FCD2E7D6E9020146
:10B758008368DB6803B1984754E8003F43F00C0363
:10B7680044E80032002AF7D129464046FFF706FF91
:10B77800054610B16FF01505BBE7337E1BB1A36812
:10B7880043F00803A360737E1BB1636843F400436E
:10B798006360B37E1BB1636843F480336360F37EF8
:10B7A8001BB1636843F400336360337F002B5BD0C5
:10B7B8003B4B9C423DD0A3F54C439C4239D003F50A
:10B7C80080639C4235D003F580639C4231D003F5F9
:10B7D80080639C422DD003F544439C4229D0A3F5B5
:10B7E8001C439C4225D003F580639C4221D003F57D
:10B7F8001C439C421DD003F580639C4219D0294B01
:10B808009C4216D06C4688B0D8F800306A46264963
:10B81800CDE905134FF40073ADF81C30234B42F803
:10B82800103F00234FF4E2511B48F7F729FDA546C6
:10B83800A0E7D8F804301A68936843F4804393600B
:10B848002368727F23F0787343EA425323602368A6
:10B85800B27F23F4F81343EA02432360F37F1BB15A
:10B86800A36843F40043A36096F820301BB1236813
:10B8780043F000532360236843F001032360E36926
:10B888009A02FCD5E3695B02FCD5D9F8283040461A
:10B8980098472EE703010608002605082301060835
:10B8A80000100140000C00583E010608030000018A
:10B8B8002DE9F041436802460D461C6803691E687D
:10B8C8000B79012B17D0981E41424141890295F806
:10B8D80005E0AF79BEF1020F96BF40484FF4005C17
:10B8E80030F81EC0022F09D0042F01D0002B6BD0D6
:10B8F8004FF4805005E04FF4C061E8E7002B60D0BA
:10B908000020A3F10308B8F1010F04D86FF08503F4
:10B918001846BDE8F0810BB1042FF7D0BCF5805F65
:10B9280054D0BCF5405F53D0BCF1000F0CBF0123CD
:10B9380003239E45EAD132F09EF98742E6D1EB799E
:10B948005BB3012B46D1264B9C4226D0A3F54C4332
:10B958009C4222D003F580639C421ED003F580638D
:10B968009C421AD003F580639C4216D003F54443E9
:10B978009C4212D0A3F51C439C420ED003F5806371
:10B988009C420AD003F51C439C4206D003F5806311
:10B998009C4202D0134B9C42B8D1236829461046DA
:10B9A80023F001032360FFF7E9FD03460028ADD12A
:10B9B800226842F00102226095E8030086E803004D
:10B9C800A6E74FF08050A9E71846A7E70023B0E79D
:10B9D8000223AEE7032BB6D098E700BF96D605083A
:10B9E80000100140000C005838B50B6805460C469D
:10B9F800988832F0E2FA04280346D1E9192014D0D5
:10BA0800022B91F874100BD1012902D9216F012959
:10BA18000BD8298E89B20AB100B11180022509E03C
:10BA2800032913D9216F032912D9296B0AB100B14F
:10BA380011600425B5FBF3F5A26E2AB1954213D91E
:10BA48001649174832F0FFFA284638BD012902D9AD
:10BA5800216F0129DDD895F83010C9B202B108B9B3
:10BA68000125E9E71170FBE7521BA2667AB9226D3E
:10BA780004F1540104F1500008322265626D013A64
:10BA8800626504F1680232F082FA6066DCE7626E91
:10BA9800002AD9D005FB03226266D5E78B01060888
:10BAA800D025050838B50B6805460C46988832F04D
:10BAB80084FA04280346CA6D15D0022891F8741038
:10BAC8000CD1012902D9E16E01290CD86AB3216E83
:10BAD80001B1118889B2298402250AE0032916D9FF
:10BAE800E16E032915D982B1216E01B1116829626D
:10BAF8000425B5FBF3F5226E2AB1954219D91A49E6
:10BB08001A4832F0A0FA284638BD1146EFE7012955
:10BB180002D9E16E0129D9D84AB1216E01B1117853
:10BB2800C9B285F820100125E5E71146D2E711468C
:10BB3800F6E7521B22667AB9A26C04F14C0104F1B3
:10BB480048000832A264E26C013AE26404F160023F
:10BB580032F01DFAE065D6E7E26D002AD3D005FB86
:10BB68000322E265CFE700BF8B010608D025050850
:10BB780070B5436805460669DA68012A12D91E4875
:10BB88009968836808319B694BB100229847041E65
:10BB980008DA1A491A4832F056FA204670BD6FF092
:10BBA8005704F6E7336923B9736006F1080004F017
:10BBB80017FA0121686832F072FA041E02DA14F1E9
:10BBC800860FEAD16D680021284632F068FA041E13
:10BBD8000BDB0948A96883681B684BB19847044682
:10BBE80018B10849064832F02EFA04EAE474D4E79A
:10BBF8006FF05704F5E700BF4C200508A9010608B7
:10BC0800D0250508CB0106082DE9F04F87B08146FD
:10BC18000E469B46924600AF046932B92BB90026FE
:10BC280030461C37BD46BDE8F08FB3889A0400F152
:10BC3800CA804FF0FF324FF0FF3304F1080004F0E0
:10BC48000BFA6660002384F84430C4E90F33D9F84E
:10BC58001030D9F80480FB601B68D8F800509E4269
:10BC6800B28840F0BC80130508D5BAF1000F00F087
:10BC7800B3804FF4C121284632F07AF9B08832F007
:10BC88009CF90346BAF1000F40F02B81C4F848A094
:10BC98000022E26404F14C0104F1600204F148005E
:10BCA800FB6032F074F9FB68E065BBF1000F40F00F
:10BCB8002181C4F850B00022626504F1540104F1F6
:10BCC800680204F1500032F062F9002360661A46F7
:10BCD800E06CA363824240F016810022D4F854C07D
:10BCE8001146614540F0168193422CBFA365A265B9
:10BCF8002A68EB6802F4006203F4C0231343FB6074
:10BD080098F82130D80728D5B388D90725D4D9F889
:10BD18000430D9F81020BB601B681968D86801F492
:10BD2800006100F4C020014340F0FD80116E966E62
:10BD380029B1002E00F0F5808E4228BF0E46002E55
:10BD48005FDBB968C969B142C0F0FB80C2E91B6614
:10BD58005A686FF30F0232435A60D9F804301B68EF
:10BD68001A6842F001021A60DA68520200F1F080A3
:10BD7800012033F01CFD236E1BB9A66E002E00F0C7
:10BD8800BA812268D8F80060928812F0010F00F09A
:10BD9800E8807269920740F11882002B00F0158242
:10BDA80021463046FFF77EFE7369D80740F1FC80D4
:10BDB800636E002B00F0F880A36E002B00F0F48077
:10BDC80021463046F2E12369002B7FF432AF6368E5
:10BDD8009E427FF42EAF35E74FF4C0214BE7D8F8E9
:10BDE8001010C2F34513022918D0032919D00129CC
:10BDF80035D1043B1C2B8CBF00230123ABB96FF05A
:10BE0800850694F8443013B1002E3FF408AF0023A0
:10BE1800636004F1080004F0E3F801E7043B0C2B2D
:10BE2800E9E7082B01D0102BE9D1100405D5EB6800
:10BE380023F4601343F40023EB609148D8F80C20F6
:10BE48008368012AD8F80810DB6833D908315BB950
:10BE58008C498D486FF0040632F0F5F8D1E78B492C
:10BE6800894832F0F0F8CAE707F114029847002829
:10BE7800EEDB7B69002230681146013223FA02FCAE
:10BE8800844540F23382082AF6D16D468AB06A4664
:10BE98007F49CDE9051059081B0A07910893052326
:10BEA80042F8103F00234FF421517748F7F7E8F99B
:10BEB800AD464AE00BB97749CBE707F1140298473A
:10BEC8000028D6DAF7E74FF4C02141E21BB1EB684E
:10BED80023F0105364E2EB6823F0105343F000534F
:10BEE8005EE2DAF80020A264002A3FF4D1AEDAF864
:10BEF8000420CEE6DBF800202265002A3FF4DBAE02
:10BF0800DBF80420D8E6A16C01EBC20101324968D4
:10BF18000B44DFE6206D00EBC100013140680244AC
:10BF2800DFE60E460BE7B1F5C12F30460CBF514690
:10BF38005946C7E9003232F064F80646D7E90032BC
:10BF4800FDE65549504832F07EF86FF0150658E77F
:10BF58001A6842F400721A601A6896053FF508AF2D
:10BF6800FAE798F8213013F0010F3368F26800F00F
:10BF78000E8103F4006302F4C022134366D1726990
:10BF8800500766D5E26E002A63D0226F002A60D07F
:10BF98002146304632F06FF82146304632F057F8E5
:10BFA80073691B0700F18180D8F80060736913F486
:10BFB800787340F00F81FB68B3F5C12F7FF4DBAED7
:10BFC800236E002B36D1A36E002B33D0304632F0CF
:10BFD80009F803460028F9D1326822F001023260DC
:10BFE80022689088C20715D4D4F854C01A4662450E
:10BFF80040F0108131F0E1FF93FBF0F200FB1232C8
:10C00800002A40F01B817268B3FBF0F36FF30F0254
:10C01800134373604FF4C021304631F0A9FF3368F1
:10C0280043F001033360F368590200F1FA800120FC
:10C0380033F0BDFB00212A68EB68002959D102F4CE
:10C04800006203F4C0231343FB6094E6B3F5C12FE9
:10C0580008D07269D10702D5226F002A9CD1B3F5A6
:10C06800C02F9DD073699A079AD5E36E002B97D09D
:10C07800226F934294D12146304631F0FCFF8FE77E
:10C088004C2005080E020608D0250508E60106081A
:10C098009D0206083A02060866020608214630464E
:10C0A800FFF7A2FC236F1B1A2367236F002BF5D120
:10C0B800226EA36E22B1002B56D0934228BF13469E
:10C0C800C4E91B33002B3FF46FAFB369304643F02C
:10C0D8001003B361B36943F00803B36131F0F4FFAF
:10C0E800E26ED8F81C309A4240D97A497A4831F041
:10C0F800AAFF6FF01506D9F80480D9F81050D8F8BF
:10C1080000104B69D80700F19C80CB685A0240F1B7
:10C118009B80DFF8C8A1084631F064FF002800F0D2
:10C1280093800B68D80740F18F8098F82130DA07A0
:10C138000CD42B689B88C3F34513192B06D82AFA0D
:10C1480003F3DB0702D5084631F0BEFF0B68CA6867
:10C1580003F4006302F4C0221343B3F5C02FDAD10D
:10C16800084631F0B1FFD6E71346A9E773682146C0
:10C178006FF30F0313437360336843F001033360B5
:10C18800336843F40073336031F075FF0CE703F450
:10C19800006A02F4C0234AEA030ABAF5C02F08D19C
:10C1A800D8F800004369D907FCD52146FFF71CFCE5
:10C1B800FAE673699807FCD521463046FFF772FC0A
:10C1C800BAF5C12F3FF4F0AEEAE7336923F0020372
:10C1D8003361E9E56D468AB06A46414905914149AE
:10C1E800CDE906134FF40073ADF820303E4B42F80A
:10C1F800103F00234FF411513748F7F741F873699E
:10C20800AD46590603D5B36943F04003B3616FF0F7
:10C21800040670E7216D01EBC201013249680B4445
:10C22800E5E6336843F40073336033689A053FF5F5
:10C23800FEAE73691B073FF5FAAEF6E76FF015011E
:10C24800F9E691F830305CE74B699B0503D58B69BB
:10C2580043F400738B6198F821000B68C007CA6823
:10C2680010D58B6943F010038B618B6943F0400351
:10C278008B618B6943F008038B614B686FF30F0385
:10C288004B6007E003F4006302F4C0221343B3F5E4
:10C29800C02FF2D02B689B88DA0402D4084631F00C
:10C2A80013FF95F844302BB9AE6305F1200003F075
:10C2B80097FEA6E5EB6B1BB12A6C314648469847BA
:10C2C8002B689B8813F400537FF49BAD6B6005F1DA
:10C2D8000800ECE766020608D025050800020202FD
:10C2E800920206083C400608040000012B684F4AE9
:10C2F80023F0010352F821202B60AB6823F0E043C0
:10C308001343AB6098F821309B0703D5EB6843F4DF
:10C318000043EB60B38813F0020FEB6814BF43F0DF
:10C32800007323F00073EB60B38813F0040FEB681D
:10C3380014BF43F0807323F08073EB60B18811F46D
:10C34800006105D0BAF1000F3FF4BDAD4FF4C12133
:10C35800284631F00DFEB38813F0100FEB6814BFB8
:10C3680043F4000323F40003EB60AB6823F4800379
:10C37800AB60B388327D03F0010322B998F821201D
:10C3880051077FF5A3AD33B9EB68DA0003D42B6806
:10C3980043F480532B60EB6823F0105343F0806321
:10C3A800EB60B388224913F0010FEB6814BF23F444
:10C3B800800343F48003EB60B288AB68C2F3451294
:10C3C80023F01F03043A51F822201A491343AB60A3
:10C3D800EB68D8F8182023F00F031343EB60EB68E1
:10C3E800D8F8142023F0F00343EA0213EB6098F81E
:10C3F8002130DB0749BFB388012398F82020C3F315
:10C40800451341BF0733DB085B00B2FBF3F3FA685F
:10C4180082F87430013BAA6851F8233022F4F07294
:10C428001343AB60FB681E6028E400BF642D050859
:10C43800182E0508D82D05084FF0E0230D4A9969F4
:10C44800126818699B69002908BF1146002B08BFAC
:10C45800134610F4803F084801D1994205D201687B
:10C46800114401604FF0E021096900681044C01AC6
:10C47800704700BF903900248C390024094B1022E2
:10C48800002083F8232046F66052074B1A6046F6D0
:10C498005F52064B18604FF0E0235A6107229861FB
:10C4A8001A61704700ED00E0903900248C390024AF
:10C4B800684620F007018D4619B5FFF7BDFF1449FE
:10C4C800144B0868D3E90042001942F10002C3E99D
:10C4D8000002114A00230B6046F66053D2E900417E
:10C4E800001BB0FBF3F043431B1941F10001C2E903
:10C4F8000031EFF31181102383F31288BFF36F8F9C
:10C5080004F028FDF7F774FEBDE81940854670472A
:10C518008C390024882F0024802F00242DE9F04135
:10C52800374E89B1421C0AD14FF0E022136923F03B
:10C53800010313614FF07F433360BDE8F081356834
:10C54800012806DC00240AE0431C3568F8D140F2D3
:10C55800562040F257239842A8BF1846441EEFF3CE
:10C568001187102383F31288BFF36F8FFFF764FFDF
:10C578004FF0E0232349D3F818C0D1E900238018ED
:10C588004FF0000243F10003C1E900031E4B1A609B
:10C598001E4B1A68831A2DD446F6605E46F65F581D
:10C5A80014FB0E841C44131A40F2D662B4FBFEF44A
:10C5B8000EFB0433934238BF1346154A934228BFF3
:10C5C80013464FF0E0223360013B94695361002326
:10C5D800A445ACEB04009361D1E900320DD20544C7
:10C5E800EB1842F10002C1E9003287F31188BFF36A
:10C5F8006F8FA2E740F2D663E3E7C318F1E700BF05
:10C6080090390024882F00248C390024802F00249E
:10C61800407EFF0038B5EFF31185102383F31288AD
:10C62800BFF36F8F084B1C68084B1B68E41AFFF7B1
:10C6380003FF85F31188BFF36F8F46F660532044DC
:10C64800B0FBF3F038BD00BF882F0024802F0024F2
:10C6580038B5EFF31185102383F31288BFF36F8F7A
:10C66800044B1C68FFF7E8FE85F31188BFF36F8F52
:10C67800204438BD882F002410B5EFF3118410230F
:10C6880083F31288BFF36F8FFFF7D6FE054AD2E90E
:10C698000031C01841F1000184F31188BFF36F8F96
:10C6A80010BD00BF882F00242DE9F0414D4C2369AF
:10C6B80003F03803102B00F09080182B0DD0002BBE
:10C6C80040F08D802368484813F0200F03D023687A
:10C6D800C3F3C103D840BDE8F081A76AA36AD4F8C0
:10C6E8002C8013F47C7FC3F30510666BF3D0F4F74A
:10C6F800EBFAC6F3CC06054608F0010007F003077D
:10C708007043F4F7E1FA4FF06451F4F735FB012F69
:10C71800064652D0022F40D0002F4ED123689B06E8
:10C7280029D523683048C3F3C103276BD840F4F7F1
:10C73800CBFA2946F4F7D4FB0446C7F30800F4F70C
:10C74800C3FA3146F4F710FA4FF07E51F4F70CFAB9
:10C7580001462046F4F710FB224B0446186BC0F341
:10C7680046200130F4F7B0FA01462046F4F7B8FB4A
:10C77800F4F704FDAFE7206BC0F30800F4F7A4FA60
:10C788003146F4F7F1F94FF07E51F4F7EDF9294607
:10C7980004461648F4F7A4FBDAE7206BC0F3080058
:10C7A800F4F792FA3146F4F7DFF94FF07E51F4F7D7
:10C7B800DBF9294604460E48ECE7206BC0F3080075
:10C7C800F4F782FA3146F4F7CFF94FF07E51F4F7D7
:10C7D800CBF9294604460748DCE707487BE70748C2
:10C7E80079E700BF004402580090D0030024744C3D
:10C7F800001BB74B0024744A00366E0100093D0047
:10C8080008B5FFF751FF0B4A0B4993699269C3F3C7
:10C81800032302F00F02CB5C03F01F0320FA03F39B
:10C82800885C064A00F01F0023FA00F01060044AF2
:10C83800136008BD004402584E400608F40800245E
:10C84800F808002408B5FFF7DBFF054B054ADB694C
:10C85800C3F30213D35C03F01F03D84008BD00BF25
:10C86800004402584E40060808B5FFF7C9FF054BBB
:10C87800054A1B6AC3F30213D35C03F01F03D840B5
:10C8880008BD00BF004402584E4006082DE9F84391
:10C89800564C0546D4F82880A36AD4F82C9013F493
:10C8A8007C3FC3F30530E76B00F09C80F4F70CFA8B
:10C8B800C7F3CC070646C9F300107843F4F704FA27
:10C8C8004FF06451F4F758FA08F003030746012BB8
:10C8D80078D0022B66D0002B74D123689B064FD5E5
:10C8E80023684348C3F3C103D4F83880D840F4F729
:10C8F800EBF93146F4F7F4FA0446C8F30800F4F704
:10C90800E3F93946F4F730F94FF07E51F4F72CF992
:10C91800364E01462046F4F72FFA0446B06BC0F3B2
:10C928004620F4F7D1F94FF07E51F4F71DF901468E
:10C938002046F4F7D5FAF4F721FC2860B06BC0F371
:10C948000640F4F7C1F94FF07E51F4F70DF90146AE
:10C958002046F4F7C5FAF4F711FC6860B06BC0F331
:10C968000660F4F7B1F94FF07E51F4F7FDF801468F
:10C978002046F4F7B5FAF4F701FCA860BDE8F8839F
:10C98800A06BC0F30800F4F79FF93946F4F7ECF808
:10C998004FF07E51F4F7E8F8314604461548F4F7AD
:10C9A8009FFAB5E7A06BC0F30800F4F78DF9394694
:10C9B800F4F7DAF84FF07E51F4F7D6F8314604462A
:10C9C8000D48ECE7A06BC0F30800F4F77DF9394691
:10C9D800F4F7CAF84FF07E51F4F7C6F8314604462A
:10C9E8000648DCE7C5E90000C7E700BF0044025875
:10C9F8000090D0030024744C001BB74B0024744AE9
:10CA08002DE9F843564C0546D4F82880A36AD4F893
:10CA18002C9013F07C7FC3F30550676C00F09C806A
:10CA2800F4F752F9C7F3CC070646C9F30020784358
:10CA3800F4F74AF94FF06451F4F79EF908F003034C
:10CA48000746012B78D0022B66D0002B74D12368BF
:10CA58009B064FD523684348C3F3C103D4F84080ED
:10CA6800D840F4F731F93146F4F73AFA0446C8F3F6
:10CA78000800F4F729F93946F4F776F84FF07E51B3
:10CA8800F4F772F8364E01462046F4F775F9044675
:10CA9800306CC0F34620F4F717F94FF07E51F4F7E5
:10CAA80063F801462046F4F71BFAF4F767FB2860A1
:10CAB800306CC0F30640F4F707F94FF07E51F4F7F5
:10CAC80053F801462046F4F70BFAF4F757FB686071
:10CAD800306CC0F30660F4F7F7F84FF07E51F4F7C6
:10CAE80043F801462046F4F7FBF9F4F747FBA86042
:10CAF800BDE8F883206CC0F30800F4F7E5F8394680
:10CB0800F4F732F84FF07E51F4F72EF83146044628
:10CB18001548F4F7E5F9B5E7206CC0F30800F4F719
:10CB2800D3F83946F4F720F84FF07E51F4F71CF8A3
:10CB3800314604460D48ECE7206CC0F30800F4F7D2
:10CB4800C3F83946F4F710F84FF07E51F4F70CF8B3
:10CB5800314604460648DCE7C5E90000C7E700BFE0
:10CB6800004402580090D0030024744C001BB74BBB
:10CB78000024744A2DE9F843564C0546D4F8288019
:10CB8800A36AD4F82C9013F47C7FC3F30510676B69
:10CB980000F09C80F4F798F8C7F3CC07064609F034
:10CBA80001007843F4F790F84FF06451F4F7E4F893
:10CBB80008F003030746012B56D0022B66D0002B42
:10CBC80074D123689B0671D523684348C3F3C10316
:10CBD800D4F83080D840F4F777F83146F4F780F984
:10CBE8000446C8F30800F4F76FF83946F3F7BCFFBA
:10CBF8004FF07E51F3F7B8FF364E01462046F4F762
:10CC0800BBF80446306BC0F34620F4F75DF84FF0EC
:10CC18007E51F3F7A9FF01462046F4F761F9F4F7CE
:10CC2800ADFA2860306BC0F30640F4F74DF84FF0CA
:10CC38007E51F3F799FF01462046F4F751F9F4F7CE
:10CC48009DFA6860306BC0F30660F4F73DF84FF06A
:10CC58007E51F3F789FF01462046F4F741F9F4F7CE
:10CC68008DFAA860BDE8F883206BC0F30800F4F7DC
:10CC78002BF83946F3F778FF4FF07E51F3F774FF3E
:10CC8800314604461548F4F72BF9B5E7206BC0F395
:10CC98000800F4F719F83946F3F766FF4FF07E51AC
:10CCA800F3F762FF314604460D48ECE7206BC0F30A
:10CCB8000800F4F709F83946F3F756FF4FF07E51AC
:10CCC800F3F752FF314604460648DCE7C5E90000A1
:10CCD800C7E700BF004402580090D0030024744AFC
:10CCE800001BB74B0024744C1FB5A0F580730B4391
:10CCF80019D19F4B1A6D02F00702042A31D8DFE8D8
:10CD080012F02000BF0005004E014500186810F021
:10CD1800005005D0002301A80193FFF771FE019888
:10CD280005B05DF804FBA0F500730B431BD1904BD5
:10CD38001A6D02F4E072802AE8D00CD8002A40F07C
:10CD48009F80186810F00070EAD0002301A80293B1
:10CD5800FFF710FFF0E0C02A00F02181B2F5807FD4
:10CD680014D00020DCE7A0F580630B432DD1804B65
:10CD78001A6D02F46062B2F5806FC7D0DED9B2F5E1
:10CD8800C06F00F00C81B2F5006FE9E7DA6C196842
:10CD980002F04052480706D52AB91B68C3F3C103FD
:10CDA8007448D840BCE7724B1968C90503D5B2F17D
:10CDB800805F00F0F280186810F40030B0D0B2F153
:10CDC800005F6D4818BF0020AAE7A0F580530B4309
:10CDD8001FD1674B1A6D02F4E042B2F5005F95D09F
:10CDE800ACD9B2F5405F00F0DA80B2F5804FB8D127
:10CDF800DA6C196802F040521B68480701D5002A0E
:10CE0800CCD0D90503D5B2F1805F00F0C680584B6D
:10CE1800D1E7A0F500530B4321D1554A136D03F414
:10CE2800E023B3F5403F00F089800DD8B3F5803F8B
:10CE380000F0A880B3F5003F74D0002B91D105B065
:10CE48005DF804EBFFF7FEBCB3F5802F63D0B3F5B4
:10CE5800A02F86D11068484B10F400305FE0A0F591
:10CE680000230B4321D1424B9A6D02F44032B2F5B4
:10CE7800803F10D0B2F5003FBAD0002A7FF471AFDE
:10CE8800186810F000603FF44BAF002301A801932D
:10CE9800FFF7FCFC43E7186810F000503FF440AF80
:10CEA80001A8FFF7ADFD03983AE7A0F580330B43DF
:10CEB8000DD12F4BDA6C1868D3037FF543AF10F010
:10CEC80000603FF42DAF01A8FFF7E0FCEBE7A0F509
:10CED80080430B4339D1264A936D03F0E043B3F105
:10CEE800405F2BD00DD8B3F1805F4BD0B3F1005F1A
:10CEF80018D0002B7FF435AF05B05DF804EBFFF7D1
:10CF0800B3BCB3F1A04FA5D0B3F1C04F47D0B3F134
:10CF1800804F7FF426AF1068184B10F4807018BF4C
:10CF28001846FDE6106810F000503FF4F9AE0023F3
:10CF380001A80293FFF764FD0298F1E6106810F06B
:10CF480004003FF4EDAE136828E7A0F5004008435D
:10CF58007FF407AF064A136D03F04053B3F1805FC7
:10CF68000ED0B3F1005F0DD0002B7FF4FAAE71E75D
:10CF7800004402580090D00300366E0100093D00BD
:10CF88001068DFE6106810F000603FF4C9AE0023B7
:10CF980001A80293FFF77AFCCEE70248C0E60248F0
:10CFA800BEE600BF00093D000080BB0070B5056803
:10CFB8004B68EC68C4F30B441C44D30184331D4410
:10CFC8006A6802F470426A6005680E68EA681D447F
:10CFD8000136C2F30B42324442EA04426A600268F4
:10CFE800CD68D4681A44C4F30A042C44956805F43F
:10CFF8007045956005688A68EE681D440132C6F37D
:10D008000A06324442EA0442AA6002681A441469D1
:10D0180024F00704146102680C691A441461026858
:10D028008D69D41891F8302042EA056291F83150A0
:10D0380042EA052291F8325042EA0542A2610268AA
:10D048001A44546924F0FF04546102684C691A4474
:10D05800546104681C44E26922F4E06222F0070289
:10D06800E2610268D1E907451A442C43D461026899
:10D078004C6A1A4494620A69072A96BF124C012422
:10D08800A45C02681A44D56A05F0E025D5620268F6
:10D09800D518D1E90062921B8E6A62437443073245
:10D0A80042EA0442EA6202681A44146B6FF30A0403
:10D0B80014630268C96A1A4411630168CA5842F0C5
:10D0C8000102CA5070BD00BF5E40060810B590F856
:10D0D800A02003460220012A14D083F8A1000124CD
:10D0E800186883F8A040426B22F0010242630020D6
:10D0F800054A116419684A6B22434A6383F8A140C0
:10D1080083F8A00010BD00BF001000502DE9F041C9
:10D118000268136823F040531360836833B90268C8
:10D128004C68136823F08003234313600A6803687C
:10D13800022A49D103F5C07203F5C47503F5C87412
:10D1480003F5D073D1E912673E431660CE6A5EB12B
:10D158008E6A1E604F6BCB6A16683B430F6B26F4D2
:10D168007C163B43334313602B684E6C23F01F033C
:10D1780033432B608B6B2BB10B681BB9CB6B0568EA
:10D18800013B2B64CD68CE69002D6AD08F6BD1E945
:10D198000483002E42D0354343EA08031668D1E9D8
:10D1A80008CE2FB33B430F6C43EA0E0343EA0C034C
:10D1B8003B432B433A4D35402B4313608B68236028
:10D1C80003688A699A6439E0032A03BF03F5A072E9
:10D1D80003F5A47503F5A87403F580721BBF03F566
:10D1E800847503F5887403F5B07303F59073A9E7A4
:10D1F80043EA0E0343EA0C032B4326F47C5525F03F
:10D208003F052B431360C36AB3F1805FD6D14B69E6
:10D21800082BD3D1136843F00063CEE71D4313688E
:10D2280045EA08056FB1086C3D4323F07063054378
:10D2380023F03F031D4315608B6823600020BDE881
:10D24800F08123F03F031D431560C36AB3F1805F8B
:10D25800F2D14B69082BEFD1136843F000631360D8
:10D26800EAE7C6B18B6BD1E9087463B1334315683B
:10D2780023430C6C3B43234325F0706424F47C5413
:10D28800234313609CE71368344323F47C533C43E3
:10D298001C43146094E7082343650120CFE700BFCF
:10D2A800C0C0FFF073B504462DF035FD054614B92E
:10D2B800012002B070BD00236365266D002E69D180
:10D2C800204631F045F841F28833E168A365636B85
:10D2D80022681943E369906819432F4B034020469D
:10D2E80019432369013B41EA03416369013B41EA70
:10D2F800032191602268216AD36823F4E0230B4359
:10D30800D360216BA36B226843EA0143136123684E
:10D31800E26B5A61226863681168013B21F4F85195
:10D3280041EA032111603246A36D202100932B4668
:10D3380030F0E6FF0028BBD12168636ACA68013B68
:10D3480022F0FF021343CB602268A168136823F020
:10D3580040030B4313602168D4E90A30D1F808214F
:10D36800034322F0A0421343C1F80831226813682E
:10D3780043F001031360A369022B04D12268936868
:10D3880043F002039360E368B3F1806F0CBF01239D
:10D398000223236500208CE7F4F8E0F838B5036829
:10D3A80004461A6A18685507216D1FD545031DD50F
:10D3B800182914D1226C127883F85020236C013379
:10D3C8002364A36C013BA364A36C23B9226813688C
:10D3D80023F480231360204631F071F938BD2829E1
:10D3E800F2D1226C93F850301370E7E7950740D5D7
:10D3F80085033ED528291ED1A16C69B112F47C5F42
:10D408000AD093F85030226C1370236C01332364D4
:10D41800A36C013BA364E1E7A26C002ADED10222DF
:10D4280020465A6221680B6823F4E0230B602265CA
:10D4380030F084F8D2E7022218295A62206803687B
:10D4480023F4E0230360226503D1204630F079F805
:10D45800C4E7082903D1204630F06DF8BEE7B1F5DE
:10D46800807FBBD1636D2046002B35D131F002F9A6
:10D47800B4E7110711D505030FD508225A622368AE
:10D488001A68500205D51A6822F410221A6002237D
:10D498002365204630F058F8A0E7D1071FD5C5030B
:10D4A8001DD5012202255A622268136823F4F81355
:10D4B8001360236865651A6850070BD51A6822F04F
:10D4C80004021A600C4AE36C9A65E06C30F005FFC0
:10D4D800002883D02046256530F027F87EE7D1065E
:10D4E8007FF57CAFC2027FF579AF102220465A62E1
:10D4F80030F02DF872E700BF7FE603082DE9F04110
:10D508009C4B8CB002684FF0010E0027DFF8688250
:10D518009A426B4607BF0125002200250122BEF171
:10D52800020F1F61C3E90077C3E9027740F01D814C
:10D538009148924E006810F0010F18BF4FF4007622
:10D548004FF0000C08EB8C000CF10104406810F05F
:10D55800010F05D080EA060C1CF0020F08BF1C6002
:10D5680010F0100F05D080EA060C1CF0200F08BF41
:10D578005C6010F4807F05D080EA060C1CF4007F04
:10D5880008BF9C6010F4803F0DD080EA060C1CF4A4
:10D59800802F08D110F4003F0CBF44F4803C44F0C5
:10D5A800807CC3F80CC010F0807F0BD080EA060C9A
:10D5B8001CF0806F06D1800154BF44F4803044F0E1
:10D5C80080701861022C4FF0010CBBD1BEF1020F24
:10D5D80003F1180340F0C780664B186810EA0C0086
:10D5E80004D0186820F0010018606046644B1C687D
:10D5F800E70740F1BC801C6824F001041C6040F07F
:10D6080002040CAB182707FB02375B4B57F8286C52
:10D61800013E03EB8606D6F804C02CF4807CC6F8DD
:10D6280004C01E68F60740F1AF801E6826F00106A8
:10D638001E6065B3069E013E03EB8606776847F0D9
:10D6480002077760079E36B1013E03EB86035E68EA
:10D6580046F020065E60099B5BB1013B03F00103C5
:10D668009B0003F1A44303F534435E6846F4802627
:10D678005E600A9B5BB1013B03F001039B0003F171
:10D68800A44303F534435E6846F080665E600CAEE2
:10D69800182303FB05630E6853F830CC664500F089
:10D6A800B3808F6853F8286CB74214D04E6853F88B
:10D6B8002C3C9E4200D176B90CAB1827CE6807FBEC
:10D6C800053757F8243C9E4205D00B6957F8206C63
:10D6D800B34240F0B0800CF1FF33274E06EB8303D2
:10D6E8005F6827F001075F6018230CAF03FB057321
:10D6F80053F82C3C33B1013B06EB83035E6826F0FC
:10D7080010065E600CAE182303FB056353F8286C03
:10D71800B7001C4E3E44776827F48077776053F84B
:10D72800243C5BB1013B03F001039B0003F1A443DC
:10D7380003F534435E6826F480365E6018230CAE29
:10D7480003FB056555F8203C002B74D0013B03F022
:10D7580001039B0003F1A44303F534435D6825F0FE
:10D7680080755D6067E0A646D9E60026E8E60446CF
:10D7780047E700BF0050005200B4005222020404E0
:10D7880000A00052FCB3005257F8306C002E3FF452
:10D798007EAF013E03EB8606D6F804C02CF0010CE0
:10D7A800C6F804C057F82C6C36B1013E03EB86036B
:10D7B8005E6826F010065E6018230CAE03FB026359
:10D7C80053F8243C5BB1013B03F001039B0003F1D8
:10D7D800A44303F534435E6826F480365E6018235C
:10D7E8000CAE03FB026353F8203C002B3FF44FAF11
:10D7F800013B03F001039B0003F1A44303F5344309
:10D808005E6826F0807641E74F6853F82C6CB74283
:10D818007FF461AFCF6853F8246CB7427FF45BAFF5
:10D828000E6953F8203C9E427FF455AF734D2B6828
:10D8380043F001032B608E68704B013E03EB8606B4
:10D84800756825F4407545EA422545F4807575608C
:10D858004E691D68013EC5F30745AE4205D91D68EE
:10D8680025F47F0545EA06451D600D681E68013DE3
:10D8780016F0010F4FEA85051D4463D06A6822F04F
:10D88800030242F001026A604A6842B1013A03EBBE
:10D8980082035A6822F0300242F010025A60CB68C4
:10D8A800DF032FD5013B03F001039B0003F1A443E1
:10D8B80003F534435A6822F4E02242F480325A6075
:10D8C8000B69DE032ED5013B03F001039B0003F136
:10D8D800A44303F534435A6822F4E02242F4403268
:10D8E8005A6020B1464A136843F001031360A30746
:10D8F80004D5444A136843F00103136000200CB0B8
:10D90800BDE8F081002BDBD0013B03F001039B0055
:10D9180003F1A44303F534435A6822F0E06242F06D
:10D928008072CCE7002BDCD0013B03F001039B00A5
:10D9380003F1A44303F534435A6822F0E06242F04D
:10D948004072CDE76E6826F0030646EA420646F0C6
:10D9580001066E604D6855B1013D03EB85035D68B6
:10D9680025F0300545EA421545F010055D60CB68A5
:10D97800DD0320D5013B03F001039B0003F1A44321
:10D9880003F534435D6825F4E02545EA824545F40E
:10D9980080355D600B69D9031FD5013B03F0010396
:10D9A8009B0003F1A44303F53443596821F4E021B3
:10D9B80041EA824292E7002BECD0013B03F00103DD
:10D9C8009B0003F1A44303F534435D6825F0E0654B
:10D9D80045EA826545F08075DBE7002B81D0013B85
:10D9E80003F001039B0003F1A44303F53443596892
:10D9F80021F0E06141EA8262A1E700BF00B4005271
:10DA08000050005200A000522DE9F04F066889B07E
:10DA18000446304631F09DFE0390002840F06D81A9
:10DA2800206831F068FE002800F06781D6F80838D1
:10DA380006F500652068C3F30D23C4F8D43431F02B
:10DA48005AFE870704D52268536903F0020353611D
:10DA5800206831F050FEC0062DD52268936923F066
:10DA680010039361D6F8208008F4F01308F00F072C
:10DA7800B3F5802F40F0448147F6F07318EA030F9E
:10DA880014D02423C8F30A19304603FB07474A4633
:10DA9800D7F8601231F06CFDD7F860324B44C7F804
:10DAA8006032D7F868324B44C7F868322268936905
:10DAB80043F010039361206831F01DFE010300F16B
:10DAC8003281206831F017FE42030CD5274606F54F
:10DAD800106B4FF0000A206831F019FE0490049B87
:10DAE800002B40F0EA81206831F005FE002813DAA7
:10DAF8006B6823F001036B6094F8CC34012B40F081
:10DB080084820021204684F8CC1431F05FF8226822
:10DB1800536903F000435361206831F0ECFD0105BF
:10DB28000AD5AB68DA0702D520462FF0D2F822686A
:10DB3800536903F400635361206831F0DCFD03018D
:10DB480015D52268536903F00063536194F8CC3407
:10DB5800002B40F05E8201212368204684F8CC1413
:10DB68005B6DC3F38303C4F8D03431F02FF8206819
:10DB780031F0C1FDC70433D56B68102123F00103D0
:10DB88006B60206831F004FC06F510634FF67F31B6
:10DB980022790398824200F24082EB6943F0011334
:10DBA800EB61E37B002B00F05782D5F8843043F01B
:10DBB8000B03C5F884306B6C43F00B036B64D6F829
:10DBC800003804F29C4223F4FE63C6F80038A179B9
:10DBD800206801F045FD2268536903F480535361BE
:10DBE800206831F088FD800416D5206831F0B5FD35
:10DBF800206831F018FC2768E071FEF701FEE27931
:10DC08000146384601F0BEFA20462FF02AF822686D
:10DC1800536903F400535361206831F06CFD010728
:10DC280007D520462FF073F82268536903F00803DC
:10DC38005361206831F05FFD020600F11882206808
:10DC480031F059FDC3020CD5A04606F5126901272B
:10DC58002379BB4200F224822268536903F48013BB
:10DC68005361206831F047FD870229D5234606F520
:10DC780032610122207990421DD993F87C7208689C
:10DC8800012F40F02382002880F22082D4F8D4C4E7
:10DC98008CEA1040C00700F1198283F87B72B069E2
:10DCA80040F08000B0617069000600F10F826B6877
:10DCB80043F400736B602268536903F400135361E3
:10DCC800206831F018FD410007D520462EF0F5FFF9
:10DCD8002268536903F080435361206831F00BFDDB
:10DCE80042070AD523685D686B0702D520462EF0E7
:10DCF800EAFF226853682B43536009B0BDE8F08FF0
:10DD0800B3F5402F7FF4D2AE082204F29C4130468E
:10DD1800C8F30A1831F02CFC242303FB0747D7F873
:10DD280068324344C0E606F53068A24600272068FA
:10DD380031F0E5FC0490049B002B3FF4C2AE049B39
:10DD4800DB0779D55FFA87FB2068594631F0E7FC95
:10DD580010F0010F81461FD00123C8F80830206851
:10DD680094F806C000F53063016CBCF1010F03EBB9
:10DD780047139A6840F08B8012F0080F07D0B44818
:10DD8800814209D9120407D54FF4004203E012F08A
:10DD9800200F5AD020229A6019F0080F21D00823AA
:10DDA800AB49C8F8083023681A6C03F530638A4217
:10DDB80003EB4713986804D9010402D54FF40040D7
:10DDC800986020460592FAF7F1FB059AA0498A4225
:10DDD80007D9A179012904D104F29C42206801F0F5
:10DDE8003FFC19F0100F02D01023C8F8083019F0C2
:10DDF800020F14D073691B0603D56B6843F4806364
:10DE08006B609AF85732012B06D1002359462046F9
:10DE18008AF8573230F05DFD0223C8F8083019F04F
:10DE2800200F02D02023C8F8083019F4005F03D06F
:10DE38004FF40053C8F80830049B013708F1200854
:10DE48000AF1240A5B08049375E7DFF804C2614508
:10DE580001D9120498D41A69DAF87432C2F312029A
:10DE68009B1ACAF868326FB9D4F864222AB904F246
:10DE78009C42012101F0F4FB04E0D4F860221A442A
:10DE8800C4F8602259462046FAF756FB84E7DFF8C3
:10DE9800C4C1614507D111043FF576AF9006F1D5AD
:10DEA80020229A60EEE7002FECD1D4F86432002BE0
:10DEB800E8D104F29C423946DCE7049BD80740F1DC
:10DEC8009B805FFA8AF320681946079331F030FC8B
:10DED80010F0010F804620D001210AF00F026B6B71
:10DEE80001FA02F223EA02036B63CBF80810A17966
:10DEF80001290DD1D7E9072313443B62BAF1000F7A
:10DF080006D1636A23B904F29C42206801F0A8FB99
:10DF18005FFA8AF12046FAF72DFB18F0080F02D0B5
:10DF28000823CBF8083018F0100F02D01023CBF8D4
:10DF3800083018F0400F02D04023CBF8083018F012
:10DF4800020F10D05146304631F022FAFB7D012BEA
:10DF580006D100235FFA8AF12046FB7530F0BAFC3F
:10DF68000223CBF8083018F0800F45D0D7E90932E2
:10DF78009A4241D8A3EB0208FB69216898450591AC
:10DF880028BF984601F5106308F1030803EB4A130C
:10DF98004FEA98080693069B996989B24145D7E9E3
:10DFA800093227D393420BD8059B0AF00F000121B1
:10DFB800D3F83428814022EA0102C3F834281BE050
:10DFC800A3EB0209FB69079A9945059828BF99466A
:10DFD800A37900931FFA89F3396A09F1030831F02C
:10DFE800B4FA3B6A4FEA98084B443B62BB6A4B441D
:10DFF800BB62D0E79342D7D9049B0AF1010A2437C0
:10E008000BF1200B5B08049369E520462EF070FEA7
:10E018007DE520462EF05DFEA9E59960203353F892
:10E02800202C22F4001243F8202CC3F8E811D3F86E
:10E03800E02122F40012C3F8E021D3F8E02142F0F5
:10E048000062C3F8E021039A01320392A0E500BF01
:10E058000A30544F0A31544F6B6943F4005343F06C
:10E068002B036B612B6943F00B032B61A7E5B369A5
:10E07800012704F257284FF0240923F08003B361E5
:10E088002379BB427FF6DBAD09FB07F318F80330B1
:10E09800012B03D1F9B2204630F035FD0137EFE707
:10E0A80098F83C30D9F80020012B09D1002A07DA6A
:10E0B80067F07F01204688F83B30C9B230F023FD75
:10E0C800013708F1240809F12009C1E50132243398
:10E0D8002031CFE52DE9F047054686B088462CF07B
:10E0E8001AFE08218146286830F0C3FE044648BB62
:10E0F800696C2868090430F0A6FF044610BB4FF08D
:10E10800FF300823302669460494CDE90003022332
:10E118002868CDE902630123059330F097FE28684B
:10E1280030F0C5FF044668B90746064640F22A5A49
:10E138002868436B13EA0A0F436B07D01A0719D5EF
:10E1480008248463204606B0BDE8F087190308D484
:10E158003CB930F060FE06462868012430F05BFECA
:10E1680007462CF0D8FDA0EB09000130E0D14FF0B4
:10E178000044E7E7436B9B0701D50224E1E7446BC2
:10E1880014F0200401D02024DBE7044B3FBA36BA50
:10E198008363C8F80070C8F80460D3E73A0F001822
:10E1A80070B5044686B015461E4631B9436B43F038
:10E1B80000636363012006B070BD90F83030012B16
:10E1C8004BD10022AB194263006D834203D9636BC4
:10E1D80043F00073EDE7032384F830302368DA62F4
:10E1E8007302A26BA362012A4FF0FF326162694693
:10E1F800206818BF6D02CDE9002390220223CDE9E3
:10E2080002230023CDE9043330F020FE2268012EDA
:10E21800D36843F04003D360206811D90A23294604
:10E22800E36230F05AFE226880B10D4B9363636B52
:10E2380003436363012384F830300023E362B9E7C2
:10E2480009232946E36230F02EFEECE7D36B43F452
:10E25800014343F02A03D363ADE70220ABE700BFD5
:10E26800FF0FE01F70B5044686B015461E4631B94B
:10E27800436B43F000636363012006B070BD90F800
:10E288003030012B4AD10022AB194263006D834222
:10E2980003D9636B43F00073EDE7032384F8303050
:10E2A8002368DA627302A26B2362012A4FF0FF32FD
:10E2B800E1616946206818BF6D02CDE9002300239B
:10E2C8009022CDE90433CDE9022330F0BFFD226866
:10E2D800012ED36843F04003D360206811D9282366
:10E2E8002946E36230F02DFE226880B10C4B93631F
:10E2F800636B03436363012384F830300023E362D4
:10E30800BAE718232946E36230F001FEECE7D36B45
:10E3180043F4824343F01A03D363AEE70220ACE729
:10E32800FF0FE01FF8B590F8303004460E4615464A
:10E33800012BDFB257D100219642416305D9436BC7
:10E3480043F0006363633846F8BD036D934203D21C
:10E35800436B43F00073F5E7032380F83030236CF8
:10E3680000689B0608D4214B8363636B43F080638A
:10E37800636384F83070E6E730F065FD8201236856
:10E3880005D51A4A9A63636B43F40063F0E7A26BFE
:10E39800012A03D0032A1BD076026D0218463146A3
:10E3A80030F0E9FD0346206843B1104A8263626B8E
:10E3B80013436363012384F83030C4E7294630F0FF
:10E3C800F4FD28B12368094A9A63636B0343F0E7B5
:10E3D8000021206830F003FE0028F3D1012307460E
:10E3E80084F83030AFE70227ADE700BFFF0FE01F2A
:10E3F80010B5C26D0346920F0A70C26DC2F38362F4
:10E408004A7090F85F2002F003028A7090F85E204C
:10E41800CA7090F85D200A7190F85C204A71026E0B
:10E42800120DCA80B0F8622002F00F020A72026E62
:10E43800C2F3C0324A72026EC2F380328A72026E2E
:10E44800C2F34032CA72026EC2F300320A7300226B
:10E458004A73826B002A40F08380006E40F6FC729B
:10E4680002EA8002586E42EA90720A615A6EC2F35A
:10E47800C2620A7593F8672002F007024A755A6E5D
:10E48800C2F342528A755A6EC2F38242CA755A6EF4
:10E49800C2F3C2320A760869013098640A7E02F033
:10E4A800070202329040012298640C7A04F00F04AB
:10E4B800A240DA64520A42431A654FF400720020FF
:10E4C8005A655A6EC2F380324A765A6EC2F3C61241
:10E4D8008A765A6E02F07F02CA769A6ED20F0A774F
:10E4E8009A6EC2F341724A779A6EC2F382628A7751
:10E4F8009A6EC2F38352CA779A6EC2F3405281F879
:10E50800202081F82100B3F86A2002F0010281F886
:10E5180022209A6EC2F3C03281F823209A6EC2F389
:10E52800803281F824209A6EC2F3403281F8252087
:10E538009A6EC2F3003281F826209A6EC2F38122C5
:10E5480081F827209A6EC2F3012281F828209B6E59
:10E55800C3F3460381F82930012381F82A301CE0EF
:10E56800012A10D1026EB0F86600120402F47C127F
:10E5780002430A610A69013292029A641A654FF4E9
:10E588000072DA6499E7026804499163426B42F0C9
:10E5980080524263012083F8300010BDFF0FE01F56
:10E5A80070B5002394B0044600214FF48030CDE9C3
:10E5B8000433CDE90633FEF797FB054648B9012336
:10E5C80084F830304FF0006363630125284614B0A7
:10E5D80070BD7A4E04ABB0FBF6F607983146089644
:10E5E8008DE803000ECB206800F002FC206830F0B4
:10E5F8001AFC734B73489D4284BF7600B5FBF6F551
:10E60800B0FBF5F001302CF08EFB0023206803935B
:10E6180000F01CFC0546A8B9206830F0F5FDB0F103
:10E62800004F06D12068E56300F010FC80B1054674
:10E6380008E00123E3630021206830F004FD50B1B5
:10E648004FF08055012384F83030636B2B43BBE7D0
:10E65800E36B012BEFD000214FF6FE7614E0206823
:10E6680030F0F1FC05460028ECD15749206830F01D
:10E678009AFD0028E4D12946206830F0E4FB039B8A
:10E688000546C10F01330393039BB34201D8002908
:10E69800E5D0039BB34214D8C5F380750023A56366
:10E6A800ADF80A302CF037FB0546206830F0C7FB80
:10E6B80050B94FF08061012384F83030636B0B430D
:10E6C80082E74FF08075BDE7A36B032B3ED020682F
:10E6D80030F03BFD01460028EDD1206830F0B3FB57
:10E6E8000421E066206830F0AEFB0821206720682E
:10E6F80030F0A9FB0C216067206830F0A4FBA36B05
:10E70800A067032B22D041F28736BDF80A10206893
:10E7180059B3A36B032B19D06164090430F02CFDA5
:10E7280001460028C7D1206830F08DFB0421E06540
:10E73800206830F088FB08212066206830F083FBD1
:10E748000C216066206830F07EFBA06604212068FA
:10E7580030F079FB09A9000D20642046FFF748FE38
:10E76800054688B14FF08051A5E70DF10A0130F058
:10E7780031FD014600289ED12CF0CDFA401BB04255
:10E78800C3D94FF0004196E7616C2068090430F066
:10E7980040FC014600288ED14FF40071206830F00B
:10E7A80068FB00283FF412AF2368084A9A63636B3A
:10E7B80003436363012384F8303006E700350C0017
:10E7C800FF340C0010210100000010C1FF0FE01FF2
:10E7D8002DE9F04190F8303096B004460D46032BF1
:10E7E80000F0AB802CF097FA00210646206830F044
:10E7F8002AFB830100F1A6804021206830F039FB14
:10E8080058B1636B636323680125524A9A63636B4B
:10E818000343636384F8305082E0616C2068090424
:10E8280030F011FC0028ECD140234FF0FF374FF0B7
:10E83800600C049069462068CDE900730223CDE995
:10E8480002C30123059330F001FB206830F063FC1C
:10E858000028D6D106AF23685A6B12F4957F0AD0E8
:10E868005A6B110771D45A6B920770D45B6B9B0675
:10E878001ED52020C7E75B6B180408D507F12008D0
:10E88800206830F0C8FA47F8040B4745F8D12CF057
:10E8980042FA801B0130DED14FF00040B3E730F080
:10E8A800BAFA47F8040B2CF036FA801B0130F3D083
:10E8B8002068426B12F48052F1D10699264B83638B
:10E8C800C1F381132B70C1F340136B700B0A23F053
:10E8D800FF0343EA11639BB26B80079B1BBA6B6013
:10E8E800089BD9B22972C3F307216972C3F3035194
:10E8F8001B0CA972099923F0FF03C8B20343AB812B
:10E90800C1F38523AB73C1F30123EB73C1F3031385
:10E9180001F00F012B749DF82B306974AB74154608
:10E928004FF40071206830F0A4FA38B12368094A1E
:10E938009A630123606384F830300125284616B0B5
:10E94800BDE8F0814FF400605DE708205BE7022036
:10E9580059E700BFFF0FE01F3A0F0018032330B537
:10E9680089B080F83030836B04460D46032B02D003
:10E97800B1F5004F03D1636B43F080531FE0B1F54D
:10E98800804F24D100210068039130F05CFA10F028
:10E99800007036D1049003A92046FFF79BFB60B9AD
:10E9A800049B590330D5616C2068090430F04BFB97
:10E9B80018B90221206830F060FB636B034363637E
:10E9C800636B43B323683E4A9A63012550E0F1B96B
:10E9D8000068039130F037FA820112D403A9204667
:10E9E8000495FFF777FB0028E7D1049BDB030BD5E1
:10E9F800616C2068090430F026FB0028DDD101464F
:10EA0800D8E74FF40060D8E74FF08060D5E7436B54
:10EA180043F00063D3E74FF480300021FEF764F938
:10EA2800002847D0636827490393A368B0FBF1F235
:10EA3800CDE9043523690693636993420CD2A56D29
:10EA4800B5F5007F08D0B5F5807F29D11BBB88427A
:10EA580002D91D4BB0FBF3F3079308AB002513E96C
:10EA6800030003AB8DE803000ECB206800F0C0F96B
:10EA78004FF40071206830F0FCF930B123680125AB
:10EA88000F4A9A63636B034363630123284684F840
:10EA9800303009B030BD5A00B0FBF2F28A42D7E7F5
:10EAA8000A491BB9884288BF1346D5E75D00B0FB09
:10EAB800F5F0F7E7636B43F00063636385E700BF36
:10EAC800FF0FE01F80F0FA0200E1F50540787D01B4
:10EAD800F7B503680446C56A5A6B170420D52E0794
:10EAE8001ED5836A1F2B19D9466A351D06F12407DE
:10EAF8002068043530F08FF905F8080C030A05F88A
:10EB0800073C030C000E05F8063C05F8050CBD4251
:10EB1800EED1A36A2036203B6662A36203B0F0BD43
:10EB28005A6BD0055BD54FF480729A632268D36B19
:10EB380023F4414323F03A03D3632268D36B23F0D1
:10EB48008053D3632268D36823F04003D36015F061
:10EB5800080320D015F0220F09D0206800F030FA01
:10EB680028B1636B0343204663632EF004FA2368DD
:10EB7800A907704A9A634FF0010384F830304FF0C8
:10EB88000003E36203D020462EF0F3F9C6E72046DF
:10EB98002EF0EAF9C2E72A06C0D5226815F0220F3E
:10EBA80093622268D3622268136509D0206800F056
:10EBB80007FA28B1636B0343204663632EF0DBF941
:10EBC800012315F0300F84F830304FF00003E36272
:10EBD80002D020462EF0C8F9AF079FD0D3E75A6B72
:10EBE800560427D5280725D5236A1F2B96D9E66909
:10EBF800351D06F1240715F8043C043501A92068E1
:10EC0800019315F8072C43EA0223019315F8062C03
:10EC180043EA0243019315F8052C43EA0263019382
:10EC280030F0FCF8BD42E6D1236A2036203BE6618D
:10EC3800236273E75A6B12F03A0F5A6B5ED0910752
:10EC480003D5626B42F0020262635A6B120703D566
:10EC5800626B42F0080262635A6B970603D5626BD7
:10EC680042F0200262635A6BD60603D5626B42F00B
:10EC7800100262632F4A9A632268D36B23F49D7350
:10EC8800D3632268D36823F04003D3602268D36A31
:10EC980043F40053D3622268D36843F08003D360FF
:10ECA800206800F08DF9636B226815F0080143EACB
:10ECB80000036363D36823F08003D3604FF40062DA
:10ECC80023689A6308D0012384F830300023E36274
:10ECD80020462EF050F921E728067FF51FAF636B19
:10ECE800002B3FF41BAF2268D36B23F08053D36310
:10ECF80023681965012384F83030E9E7D2007FF5ED
:10ED08000DAF4FF0805205F0200520469A63236826
:10ED18001B6D5B0706D415B12FF0E8FFFEE62FF058
:10ED2800E3FFFBE615B12FF0E0FFF7E62FF0DBFF7E
:10ED3800F4E600BF3A0F001838B50D460446F0B1A6
:10ED480090F82C3003F0FF021BB980F82D202FF02B
:10ED5800CEFF0223211D206884F82C3000F014F81F
:10ED68006268294620682FF0FAFF064A00201368D7
:10ED780043F000431360012384F82C3038BD012090
:10ED8800FCE700BF00400052D1E9073230B50C68FB
:10ED980013434D6A154A94B904682B432240134320
:10EDA8004A6813438A681343CA6813430A691343BA
:10EDB8004A6913438A6913430360002030BD04681D
:10EDC8002B4324F4F84423430360436813404A6800
:10EDD80013438A681343CA6813430A6913434A6989
:10EDE80013438A6913434360E7E700BF0080FFFFCE
:10EDF80084B010B503AC84E80E00039B416813434C
:10EE0800059A1343069A1343079A1343044A0A4080
:10EE1800134343600020BDE8104004B0704700BFB2
:10EE2800002CC0FF0B6810B58360C468D1E90132BB
:10EE38001343CA6813430A691343034A224013431E
:10EE4800C360002010BD00BFC0E0FEFF10B5002366
:10EE580086B0044601A9CDE90133CDE903334FF467
:10EE680080530593FFF7DEFF0A4B4FF4FA521B68F5
:10EE7800B3FBF2F341F28832534343B1626B013B77
:10EE88001206FAD5044B0020A36306B010BD4FF05C
:10EE98000040FAE7F8080024C5002000034644486B
:10EEA80010B54FF4FA540068B0FBF4F0414C4243FB
:10EEB800002A48D0586B204207D0800405D45A6BEA
:10EEC800540704D50420986310BD013AF0E75A6B43
:10EED800D00703D501229A630120F5E7364A9A63E1
:10EEE8001A69D2B29142F7D15B69344818400028B8
:10EEF800EAD0002B2ADB5A002BD49C002BD4D90053
:10EF08002BD41A012CD45C012DD4D9012ED41A0289
:10EF18002FD45C0230D4990231D4DA0232D45C03A3
:10EF280033D4990334D4DA0335D41C0436D45904C1
:10EF380037D49A0438D413F0080F0CBF4FF480303C
:10EF48004FF40000C0E74FF00040BDE74FF00070FD
:10EF5800BAE74020B8E78020B6E74FF48070B3E7FF
:10EF68004FF40070B0E74FF48060ADE74FF40060F5
:10EF7800AAE74FF48050A7E74FF40050A4E74FF4F6
:10EF88008040A1E74FF400409EE74FF400309BE734
:10EF98004FF4802098E74FF4002095E74FF4801055
:10EFA80092E74FF400108FE74FF480008CE700BF22
:10EFB800F808002445002000C500200008E0FFFDF7
:10EFC80030B5002387B00C254FF48072044601A9A0
:10EFD800CDE90323CDE901354FF480530593C36888
:10EFE80043F08003C360C36823F04003C360FFF7A6
:10EFF80019FF074A29462046FFF750FFE368B0F19A
:10F00800007F23F0800308BF0020E36007B030BD15
:10F0180000E1F505114B4FF4FA5102461B68B3FBAA
:10F02800F1F341F288314B43ABB1516B11F0450F0D
:10F0380007D0890405D4536B5B0704D5042090637B
:10F048007047013BF0E7506B10F0010014BF01233B
:10F05800034B936370474FF000407047F808002453
:10F06800C50020000F4B4FF4FA5102461B68B3FB52
:10F07800F1F341F288314B438BB1516B11F0450FDD
:10F0880008D0890406D4506B10F0040004D0042082
:10F0980090637047013BEFE7034B936370474FF072
:10F0A80000407047F8080024C500200003461E48A9
:10F0B80010B54FF4FA540068B0FBF4F041F288340C
:10F0C800604358B35C6B14F0450F07D0A40405D413
:10F0D800586B440704D50420986310BD0138F0E745
:10F0E800586BC00703D501229A630120F5E7186918
:10F0F800C0B28142F9D10D4999635B6913F460404C
:10F1080002D11B0C1380E8E75A040AD413F4004F09
:10F118000CBF4FF480304FF48050DEE74FF00040D2
:10F12800DBE74FF40050D8E7F8080024C5002000BA
:10F13800134B4FF4FA5102461B68B3FBF1F341F24B
:10F1480088314B43CBB1516B11F0450F07D0880480
:10F1580005D4536B590704D5042090637047013BCD
:10F16800F0E7506B10F0010002D001239363704761
:10F17800536B5B0603D54023F8E74FF00040704718
:10F18800F8080024022A4AD1274B284A0B44934204
:10F1980039D9274B274A0B44934236D9A1F5740332
:10F1A800254AA3F51053934231D9A1F18373234A19
:10F1B800A3F5E74393422CD3214B224A0B449342B5
:10F1C80029D9214B214A0B44934226D3204B214A6B
:10F1D8000B44934223D3A1F1B7731F4AA3F55853A5
:10F1E80093421ED31D4B1E4A0B4493422CBF062349
:10F1F8000723C26822F47052C260C26842EA8323BD
:10F20800C360002070470F23F3E70E23F1E70D23B7
:10F21800EFE70C23EDE70B23EBE70A23E9E70923E4
:10F22800E7E70823E5E700BF405327FFFF340C005A
:10F23800401E1BFF3F420F007F4F120020D61300D5
:10F2480060B6E5FE5FE3160000D3CEFE40771B00F4
:10F25800C05BB3FEC091210020753800E05459FE10
:10F26800E09C410084B02DE9F843044609A880E8F1
:10F278000E0000239DF824609DF82E50194603F1D6
:10F288004002013304EB82020F2B5160F7D104F5E1
:10F298000067002D6CD17B6843F002037B60A36B91
:10F2A80023F40013A363236843F040032360236817
:10F2B80043F0800323600023C4F8003E9DF8293002
:10F2C800012B5CD19DF82710002956D120464FF616
:10F2D8007F3830F0A1F81021204630F059F8014667
:10F2E800204630F078F80843002304F51062C0B2D5
:10F2F8004FF0904C19464FF0006E00383B617B612F
:10F3080018BF0120FB619E423BD8002204F5306300
:10F318004FF0904C4FF0006E11464FF67F389642F2
:10F3280042D83B6923F480733B610023A3616FF0EB
:10F33800804363619DF826301BB9A36943F010032D
:10F34800A361A269224B1343A3619DF82A301BB124
:10F35800A36943F00803A361012D05D1A36943F014
:10F36800804343F00403A361BDE8F84304B0704749
:10F37800A36B43F40013A3639DE71946A6E7032193
:10F38800A4E7D2F80090B9F1000F0BDA3BB9C2F844
:10F3980000E011610133C2F808802032B3E7C2F8F7
:10F3A80000C0F6E71160F4E7D3F80090B9F1000F58
:10F3B8000BDA3AB9C3F800E019610132C3F80880E2
:10F3C8002033ACE7C3F800C0F6E71960F4E700BFE4
:10F3D80000383C8030B54A780B78012A00EB43139B
:10F3E80000F5006029D1D3F80029002A0BDAD3F8F8
:10F3F800002942F00062C3F80029D3F8002942F03E
:10F408008042C3F800290A780124C56B02F00F0274
:10F4180004FA02F225EA0202C2630978C26901F01D
:10F428000F018C4022EA0402C261184AD3F800197D
:10F438000A40C3F80029002030BDD3F8002B002A69
:10F448000BDAD3F8002B42F00062C3F8002BD3F894
:10F45800002B42F08042C3F8002B0A780124C56BC8
:10F4680002F00F0204FA02F225EA0242C2630978A6
:10F47800C26901F00F018C4022EA0442C261044AC9
:10F48800D3F8001B0A40C3F8002BD4E7007833EC0C
:10F498000078F3EFF7B54B7891F800C0012B6D4D6C
:10F4A80000EB4C146C4E40F089800F6904F5106332
:10F4B8003FBB1F693D401D611D6945F400251D6165
:10F4C8001D693540012A1D614DD1CA6902B15A61D1
:10F4D8000B79012B0CD1D0F8083813F4807FD4F8BD
:10F4E80000390CBF43F0005343F08053C4F800398F
:10F4F800D4F8003943F00443C4F80039002003B0BD
:10F50800F0BD1F693E401E611E6935401D610D69D1
:10F518008E68BCF1000F0CD1B54288BF0E611D6921
:10F5280045F400251D610D691E69C5F312053543B3
:10F53800C8E73544494FD3F810C0013DB5FBF6F58F
:10F54800AEB207EAC54545EA0C051D610D79012DE6
:10F55800E9D11D6925F0C0451D6175071F6905F0D2
:10F56800C0453D43DEE7D4F8003943F00443C4F80E
:10F5780000390B79012B0DD00B69002BBED00A780E
:10F588000123D0F8344802F00F0293402343C0F817
:10F598003438B3E7D0F8083813F4807FD4F800394A
:10F5A8000CBF43F0005343F08053C4F80039009275
:10F5B8000B8A0A78C9682FF0C8FF9FE7D4F8107B38
:10F5C80004F530633E401E611E6935401D610E69B9
:10F5D8008D68BCF1000F27D106B10D610D621E695F
:10F5E800C5F3120535431D611D6945F40025012A3F
:10F5F8001D6102D1CA6802B15A610B79012B0CD185
:10F60800D0F8083813F4807FD4F8003B0CBF43F0DF
:10F61800005343F08053C4F8003BD4F8003B43F058
:10F628000443C4F8003B69E7002ED8D02E44013EBD
:10F63800B6FBF5F6B6B275430D62084D1F6905EACB
:10F64800C6453D431D610D6A1E69C5F31205354364
:10F65800CDE700BFFFFF07E00000F8FF0000F81F3C
:10F6680030B5114C00F53063056CA54203D9D0F8CC
:10F67800004B002C16DB002401291C611C6944F492
:10F6880000241C611C6944F018041C611C6944F0C6
:10F69800C0441C6106D15A61D0F8003B43F0802376
:10F6A800C0F8003B002030BD0A30544F00287FD0FE
:10F6B800414B9A6902F44042B2F5404F1BD13F4B8F
:10F6C8003F4A0344934258D33E4A3F4B02449A422E
:10F6D80066D33E4A02449A4264D33D4A02449A425F
:10F6E80062D33C4A02449A4260D33B4A02449A425B
:10F6F8001ED2012342E09A6902F44042B2F5004F5B
:10F708001AD1364B364A0344934249D3354A364BCD
:10F7180002449A4246D9354A02449A4244D9344A64
:10F7280002449A4242D9334A02449A42E1D9013307
:10F7380098423DD8002321E09B6903F44043B3F588
:10F74800804F0FD12C4B2D4A034493422AD32C4A85
:10F758002C4B02449A4227D92B4A02449A4225D973
:10F768002A4AE1E72A4A2B4B02449A421CD31A4AF6
:10F7780002449A421AD3284AB8E7062327490A6856
:10F7880022F00F021A430A600A6802F00F0293423D
:10F7980010D0086800F00F00C01A18BF0120704789
:10F7A8000523EBE70423E9E70323E7E70223E5E77B
:10F7B800012070470020704700480258FFAD43F011
:10F7C8000024F400FF10E3F200639F02FF7382F548
:10F7D800FFD621F8FF39C1FAFF9C60FD7FA77BF3B4
:10F7E800C0E1E400FF85FCF57FDE80027F647DF8E0
:10F7F800FF42FEFA7F217FFDFFCDE4F700366E0160
:10F808007F9AEBF97FCC0602FF66F2FB7F33F9FDA6
:10F818007FEB10FC80B14F017F4EB0FE00200052FC
:10F8280070B50546C8B1047874B10D4C0D4EB4429C
:10F8380001D3002408E02168A94207D120462FF00F
:10F84800DDFF002808BF0024204670BD2846F1F7D8
:10F858005FFD0028F2D01C34E9E70446F4E700BF56
:10F868004C2005085C23050810B50446F3F73AFC5C
:10F8780003480121034A2BF06AFB20462FF0C9FFF9
:10F88800C0250508E30206082DE9F843044600AF41
:10F898000D46EFF31188102383F31288BFF36F8F9F
:10F8A80004282A4AE9468AB098BF294B9668117CF1
:10F8B8006A4694BF53F82030264BCDE9073140F211
:10F8C80001332548ADF82430244BCDE9050442F82E
:10F8D800103F00234FF431512148F3F7D1FCCD46B6
:10F8E80045B1EB69C3F3080323B11E4A01211C4843
:10F8F8002BF02DFB2EB1304630F017FA08B1037803
:10F9080003B91948E9468AB06A46184B0790CDE909
:10F91800053640F20133ADF82030154B42F8103F60
:10F9280000234FF411510E48F3F7AAFC294620464C
:10F93800CD46FFF799FF88F31188BFF36F8F3046E4
:10F94800F4F766FCBD46BDE8F88300BF943900248F
:10F958008C2E0508F20206080803060805000001B7
:10F96800C0250508300306080003060851030608E9
:10F978000400000138B50A4B53F82040013053F811
:10F988002050A54200D838BD606830B1037EDB073F
:10F9980001D42FF01BFF0834F3E723689847FAE7F0
:10F9A800A02E0508284B0122032070B5274C86B0ED
:10F9B800274D1A70FFF7DEFF0420FFF7DBFF26460E
:10F9C8003034AE420FD3214C01F0FAF8AC4226D3C2
:10F9D80001F00AF92AF05BFC1E4A938923F001031F
:10F9E800938106B070BD54F80C3C059354F8103C54
:10F9F800049354F8143C039354F8183C029354F8B5
:10FA08001C3C019354F8203C009354E90A2354E920
:10FA18000C0100F031FD54F8303C5E65CFE7D4E9C5
:10FA28000A23B3F1FF3F08BFB2F1FF3F05D052EA06
:10FA38000301206803D100F0A9FD3034C6E7064968
:10FA4800183001F0A9F9F8E70A44002460230508F2
:10FA5800902305083030002459FE030870B5A02310
:10FA6800154E86B0012203FB00660023134D0446A1
:10FA780001931349CDE904230F22CDE9023214235F
:10FA88004FF4A07203FB00554FF4C0700D4B00FB00
:10FA980004113046009500F0EFFC337C0A4A23F04D
:10FAA8000403EE602C7433744FF4046304FB0333D3
:10FAB80013446B6006B070BD902F00249439002465
:10FAC80040600024ABF90308005800247FB50020EB
:10FAD800FFF750FF274B83F30888274D0024F023B6
:10FAE80085F82230EC772C766C76AC7685F8204059
:10FAF8006B6A43F4E0236B62F4F760FAF4F772FB85
:10FB08004FF0FF33AB62EB62F4F752FD1B4DF4F795
:10FB180097FCF3F747FA1A4800F014FDF3F7F0F8EA
:10FB28000120FFF727FF0220FFF724FF01F040F82C
:10FB3800144B4FF4BE4214495D612846134B0094A0
:10FB480005930123CDE90144CDE90343104B00F0AF
:10FB580093FC2B7C0646284623F004032B7430F0D4
:10FB68003FF92046FFF77AFF094A31462846F4F75D
:10FB780019FB00BF4060002400ED00E03030002495
:10FB8800D030002494390024C0610024D9DE05084F
:10FB9800ADF9000838B5064C064DAC4201D300203B
:10FBA80038BDD4E90112204614342FF07CFEF4E766
:10FBB800A0110024B411002430B585B0044BDDE950
:10FBC80008450293CDE900452FF02BFE05B030BD66
:10FBD80097A4030838B5074C074DAC4201D3002061
:10FBE80038BD20462FF083FE08B91C34F5E76FF0C6
:10FBF8001500F5E784110024A011002473B50C4604
:10FC0800EFF31181102585F31288BFF36F8FC56854
:10FC18005DB125602B68C36083690133836100206F
:10FC280081F31188BFF36F8F11E052EA030603D105
:10FC38006FF00B002560F3E7CDE90023024608309A
:10FC480000F0C0FE18B9034B9B685B69236002B0E3
:10FC580070BD00BF94390024F7B50E4604469DF8E0
:10FC68002010EFF31187102080F31288BFF36F8FF5
:10FC7800256AE068854245D22568AC4219D0C5B1ED
:10FC880028462FF099FE05F1180001F01BF9A2682B
:10FC98003146686941F0E2FF00232846C5F89830EC
:10FCA80030F09EF804F10800394630F015F90020CC
:10FCB80036E0A268D9B13146E06941F0CFFFE36987
:10FCC800A268134462699342E36101D12369E36145
:10FCD800236A102104F124000133236230F060FA12
:10FCE8000028DFD187F31188BFF36F8F18E0A06970
:10FCF80031462369984208BF6069801AA06141F0C3
:10FD0800ADFFE5E752EA03010CD0084904F1080009
:10FD180089684E613946CDE90023224600F052FE3B
:10FD280003B0F0BD6FF02200DCE700BF9439002477
:10FD3800F7B504460846EFF31186102181F31288BF
:10FD4800BFF36F8F216A00293BD0A268A16941F0F7
:10FD580085FFA369A2682568134462699342A36179
:10FD680004BF2369A361AC42236A03F1FF33236212
:10FD780036D02846002D34D02FF01EFE05F118008D
:10FD880001F0A0F86969A2680027E06941F066FF00
:10FD9800E369A2682846134462699342E36104BF99
:10FDA8002369E361236A01332362C5F8987030F050
:10FDB80017F804F10800314630F08EF8384603B0E1
:10FDC800F0BD52EA030111D00A49896848613146F9
:10FDD80004F10800CDE90023224600F0F3FDEEE728
:10FDE800002086F31188BFF36F8FE8E76FF02200D9
:10FDF800F7E700BF943900242DE9F341044617467C
:10FE08001E46EFF31188102383F31288BFF36F8F18
:10FE1800304BC2689B6872B18068984217D057EA25
:10FE2800060216D188F31188BFF36F8F6FF00F00A9
:10FE380002B0BDE8F08193F90E1001322161C4E9E6
:10FE4800023288F31188BFF36F8F0020F0E7216931
:10FE5800F3E793F90E1090F90E30994230DA99428F
:10FE6800A8BF19462FF00AFE0546224641461A4801
:10FE7800CDE9007600F0A6FD0028E6D0EFF3118664
:10FE8800102383F31288BFF36F8FA068D0B1236863
:10FE980021699C420AD04BB193F90E309942A8BF10
:10FEA80019466FF07F039942B8BF19462FF0E6FD57
:10FEB80040B13146084830F00FF86FF00A00B7E754
:10FEC8000025D2E7002DF4D186F31188BFF36F8F98
:10FED800F3E700BF943900240B440024F8B5836885
:10FEE8000546002B40D0234A926893423FD1C3680D
:10FEF800012B03D9013BC3600020F8BDEFF3118744
:10FF0800102383F31288BFF36F8F016980682FF085
:10FF1800B5FD2C68A54207D10023C5E9023387F354
:10FF28001188BFF36F8FE7E7002CF5D0002604F1A6
:10FF38001800D4E9003213605A60237CA66023F0CD
:10FF48000203C4E90066237400F0BCFFAC6094F9B6
:10FF58000E3020462B61C4F898602FF041FF3946D7
:10FF680005482FF0B9FFC7E76FF01500C5E74FF058
:10FF7800FF30C2E7943900240B44002437B51146FA
:10FF8800EFF31185102282F31288BFF36F8F046894
:10FF98009CB123680121426823F003039442036063
:10FFA80008BF436020462FF0F6FD044685F311880C
:10FFB800BFF36F8F204603B030BD51EA0302F5D07E
:10FFC80000F10802CDE900131046294600F0FAFCBA
:10FFD8000028EFD1014B9B685C69EBE7943900245A
:10FFE80070B5EFF31186102383F31288BFF36F8F78
:08FFF8000468A0421BD0D4B143
:020000040801F1
:10000000002504F11800D4E9003213605A60237C03
:10001000A56023F00203C4E90055237400F056FFE5
:100020002046C4F898502FF0DFFE31460B48BDE85B
:1000300070402FF055BFD0E90232022110309A42B1
:1000400018BF013340F8083C30F0AEF80028ECD17E
:1000500086F31188BFF36F8F70BD00BF0B4400247F
:1000600013B5EFF31181102484F31288BFF36F8F5F
:10007000846844B1013C846081F31188BFF36F8FC1
:10008000002002B010BD52EA030406D181F31188AA
:10009000BFF36F8F6FF00F00F3E7CDE90023024647
:1000A000014800F093FCECE70B440024F8B505464A
:1000B000EFF31186102383F31288BFF36F8F0027AD
:1000C0002C68A54219D0C4B104F118000127D4E965
:1000D000003213605A600023227CA36022F00202E7
:1000E000C4E90033227400F0F1FE6FF00A032046E9
:1000F000C4F898302FF078FEE2E70023022105F1E2
:100100001000AB6030F050F828B927B986F3118899
:10011000BFF36F8FF8BD31460248BDE8F8402FF0BD
:10012000DFBE00BF0B4400242DE9FF410446102729
:10013000534EEFF3118887F31288BFF36F8FD4F813
:10014000A450F5B9022104F1BC002FF069FD00288C
:1001500070D004F1B4050022012128462FF046FF9B
:100160000028F8D100234FF0FF3241464548029362
:100170004FF0FF33CDE9002304F1AC0200F04EFD57
:10018000D7E7D4F8A8202B689542C4F8A43008BF5C
:10019000C4F8A830D4F8BC3043F00203C4F8BC3033
:1001A000EB6823F0040343F00103EB606B6888F312
:1001B0001188BFF36F8F28469847EFF3118887F3B4
:1001C0001288BFF36F8FEB68D80623F001023ED48C
:1001D000EA60EB689A0717D523F002033068EB60FA
:1001E00090B10368002178B1426895423DD103681F
:1001F000002934D172683360904200D173600023CB
:1002000040F8083BFFF7F0FED4F8BC3023F00203BF
:10021000C4F8BC30DB0530D4D4F8A430003B18BFA0
:10022000012388F31188BFF36F8F002B81D02FF04B
:10023000A1FD7EE7D4F8BC30D90693D5C4F8BC0044
:1002400088F31188BFF36F8F04B0BDE8F08123F00D
:100250001103EB6005F11000FFF7C6FEB9E70B6074
:100260007368984208BF7160C9E701461BB11A68FC
:1002700018461346B7E71A46FAE70023D1E700BF4E
:10028000B83900240B440024F8B5C36804460E4670
:100290009A07C3F3400541D45F0741D40B680BB9FB
:1002A00083680B60E368D80745BFA3680225012572
:1002B0003360376857B31C4B9A68D7F8A0309A421E
:1002C0001ED12FF02DFD80F00100C0B2D7F8BC3058
:1002D000D907C3F380021CD5F2B1F8B10023236023
:1002E000D7F8A83073B9C7E9294438462FF0B2FCD3
:1002F000E36843F00403E3603368A3602846F8BD75
:100300000020E3E71C60C7F8A840EEE76FF0150592
:1003100006E06FF0120503E01B07DFD56FF00F0555
:1003200000233360EAE700BF943900240146014806
:100330002FF0DABC90310024F0B50446002089B0DB
:10034000C4E9290004F1AC000E9DC4E92B0004F1BE
:10035000B400C4E92D0055B32879002840F20110FB
:1003600008BF0120C4F8BC0000204FF0FF364FF05A
:10037000FF370094CDE90330CDE901000D4B204655
:10038000CDE9066700F02AF955B1296811B1204678
:100390002FF0CCFC6B791BB1A38943F00103A3813F
:1003A000204600F0F7F8C4F8A04009B0F0BD0120E5
:1003B000D8E700BF2901010837B501900846EFF3DF
:1003C0001184102181F31288BFF36F8FC16811F07F
:1003D0001E0F17D153EA020508D101A9FFF754FFF8
:1003E00084F31188BFF36F8F03B030BD41F0080173
:1003F000103040F8041C01998161034900F0D0FCE1
:100400000120EDE70020EBE763FC0308014601480B
:10041000FFF7D2BF90310024F7B50C4616461D46B3
:100420000190EFF31187102383F31288BFF36F8FCE
:1004300008462FF000FC55EA060309D101A9204621
:10044000FFF722FF87F31188BFF36F8F03B0F0BD72
:10045000E3683246064904F1100043F00803E36004
:10046000019BA3622B4600F09BFC0120EAE700BF42
:1004700063FC030801460148FFF7CEBF903100241A
:10048000073222F007022DE9F04F7F3285B01F4678
:1004900000F15803044622F03F020E4604213F2A91
:1004A000A2F1400B06F14008C0E91633129B4FF051
:1004B00000002174A381119BA060A373E073DDE9A8
:1004C0000EA9C4E9060005D880F31188BFF36F8F29
:1004D000084602DFB51820462946F3F727FB073008
:1004E000109B314620F007002D1AC4F888002046E2
:1004F0002A46C4E9208BCDE90193CDF800A03B4604
:10050000F3F724FE0023C4F874906365109BC4E9DC
:100510001B7AA367EFF31182102383F31288BFF3D2
:100520006F8F094B196A1C62E16782F31188BFF370
:100530006F8F9B680BB1D3F88C302846C4F88C3091
:1005400005B0BDE8F08F00BF943900240123037487
:1005500083810023C0E92033C0F88C30014B9860C0
:10056000704700BF9439002408B500F05BFA70B101
:10057000074B9B68DB7B53B9EFF31180102383F3A8
:100580001288BFF36F8FBDE8084000F0B7BA08BD0E
:100590009439002438B50446EFF31185102383F312
:1005A0001288BFF36F8F037C5B070FD5183000F004
:1005B0008DFC237C204623F0040323742FF023FCBE
:1005C00029460548BDE838402FF08ABC85F31188DC
:1005D000BFF36F8F38BD00BF0B440024F0B500257A
:1005E00087B004460595109D04950F9D03950E9DBB
:1005F00002950D9D01950C9DDDE912760095FFF7A2
:100600003FFFB6F1FF3F08BFB7F1FF3F05D056EA05
:10061000070305D12046FFF7BDFF204607B0F0BD18
:100620003A46334604F11800014900F0B9FBF4E7FB
:1006300059FE03080A4A6FF00A019368C3F898103C
:100640000849C3F894004B6843F080534B60002383
:1006500083F31188BFF36F8F9368D3F898007047C6
:100660009439002400ED00E038B590F910200146DF
:10067000037C002A04DA03F07F0303742FF07CFB71
:100680000D4D2A46AB6852F8184F944200D004B979
:10069000EC688B4207D01A7CD20604D1DA897F2A13
:1006A00001D9A2692AB1A34202D0204600F0F8FA8B
:1006B00023466B6138BD00BF9439002470B590F9B2
:1006C0001020037C002A2FDBD9062DD11A4C63F0B1
:1006D0007F0322460374E16952F8183F934207D121
:1006E000C0E900210860E0610FE09942F8D01B6882
:1006F000002BF5D093F90E6090F90E50AE42F4DD68
:100700005968C0E9003108605860A569954200D079
:1007100005B9E568A3681A7CD20606D1DA897F2A72
:1007200003D9AA690AB9636170BDAB4202D02846F9
:1007300000F0B6FA6561F7E794390024034648B93A
:10074000EFF3058232B9064A51699268914201D0AD
:10075000FFF770BF83F31188BFF36F8F704700BF3F
:100760009439002438B5184CA168E0690B688142BF
:1007700014BF1A46002249680B605960A368E169FA
:100780002AB9124AC3E900210B60E3610AE092F939
:100790000E5093F90E00854212DD5168C3E9002125
:1007A0000B605360A569094B9D4200D005B9E5680F
:1007B000A3689D4202D0284600F072FA656138BDF8
:1007C0008A42DED01268DBE794390024AC39002479
:1007D000002A2DE9F0470CBF4FF010094FF008092F
:1007E000027C04460E460F4619EA020F2BD149EA55
:1007F0000203D20949D10374B9F1080F4BD04FF06D
:100800000008DFF8F8A0534653F8185F9D4200D067
:100810000DB9DAF80C50DAF80830AB4202D02846AD
:1008200000F03EFAB9F1100FCAF814500BD0204670
:100830002AF047FD204600F083FAB8F1000F02D0FD
:100840002F48FFF783FE2D4B9B68A3424FD1EFF358
:100850000583002B4BD1A289D20711D586F31188CD
:10086000BFF36F8F83F31188BFF36F8F0423184694
:1008700002DFEFF31187102383F31288BFF36F8F2A
:100880003846BDE8F047FFF7D5BE03F07F03037499
:100890002FF072FAB0E7A36813B120462FF074FA74
:1008A00004F1180004F1580800F010FBA56DA845EC
:1008B00011D04FF0000A75B128462FF065FA05F106
:1008C000180000F003FB2846C5F898A0FFF7F6FED5
:1008D000A56DA845EFD1094B9B689C428FD1EFF3E2
:1008E0000588B8F1000818BF4FF0010889E786F3C2
:1008F0001188BFF36F8FBDE8F08700BF94390024E3
:10090000D030002470B50F4D06462B4653F8184FD3
:100910009C4200D004B9EC68AB681A7CD20604D1C2
:10092000DA897F2A01D9A2692AB1A34202D02046DE
:1009300000F0B6F9234630466B61BDE87040FFF722
:10094000FDBE00BF9439002470B5EFF3118610236B
:1009500083F31288BFF36F8F1A4CA168E0690B68AC
:10096000814214BF1A46002249680B605960A3688F
:10097000E1692AB9144AC3E900210B60E3610AE086
:1009800092F90E5093F90E00854216DD5168C3E9C5
:1009900000210B605360A5690B4B9D4200D005B947
:1009A000E568A3689D4202D0284600F079F93046F8
:1009B0006561BDE87040FFF73DBE8A42DAD012683B
:1009C000D7E700BF94390024AC390024F8B5124BA6
:1009D0000C461146114A9868DDE906761060EFF37F
:1009E0001182102282F31288BFF36F8F9D68284610
:1009F0002FF0D4F9B6F1FF3F08BFB7F1FF3F06D0A3
:100A00003A463346064905F1180000F0C9F9204678
:100A1000BDE8F840FFF70EBE94390024C039002429
:100A200059FE0308F8B50446EFF31187102383F34A
:100A30001288BFF36F8F037C49B203F01F02002AB4
:100A40000CBF0126002635D103F07F032A4D037425
:100A50002FF092F9037C2A46817363F07F030374BD
:100A600052F8183FE869934207D1C4E900200460B6
:100A7000EC610DE09842F8D01B68002BF5D093F99B
:100A80000EC08C45F6DD5968C4E900310C605C602D
:100A9000AC69944200D004B9EC68AB689C4202D0C7
:100AA000204600F0FDF86C6187F31188BFF36F8F6B
:100AB0003046F8BD9B071CD585682FF05DF9817322
:100AC0002B689D4209D16B68C4E900531C606C60BF
:100AD000EAE76A689A42F6D01B68002BF3D093F9D4
:100AE0000E208A42F5DD5A68C4E9003214605C6069
:100AF000DAE78173D8E700BF94390024034648B988
:100B0000EFF3058232B9064A51699268914201D0E9
:100B1000FFF790BD83F31188BFF36F8F704700BF5D
:100B200094390024F8B550EA010306460C4603D177
:100B30002FF020F90020F8BDEFF31187102383F385
:100B40001288BFF36F8F184D184BA86818602FF0EC
:100B50005CF9A868324623461549183000F020F9A0
:100B6000AB6804461A7CC3F8947042F004021A740D
:100B70006FF00A02C3F898200E4A536843F080537E
:100B80005360002383F31188BFF36F8FAA68D2E903
:100B90000A12B2F1004F08BF9942CBD12FF069FA87
:100BA000201A20EAE070C6E794390024C0390024F6
:100BB00059FE030800ED00E0024B03F11802C3E9FF
:100BC0000622704794390024EFF31181102383F338
:100BD0001288BFF36F8F054B9A68D37B013BD373A9
:100BE00081F31188BFF36F8F704700BF94390024E1
:100BF000EFF31180102383F31288BFF36F8F034B41
:100C00009A68D37B0133D373FFF77CBE94390024F9
:100C1000014B9868704700BF94390024D3B5DDE9D3
:100C20000667089CCDE90067FFF7D0FE1CB1034BB7
:100C30009B685B69236002B0D0BD00BF943900247B
:100C4000027C034612F01F0210D10A4988420DD0DF
:100C50000949086868B1D9897F2909D893F90E2014
:100C6000064B1B689A42B8BF0020704700207047AF
:100C700010467047902F0024FC080024C43900243B
:100C8000044B0122C01A044BC0105843034B1A54A2
:100C9000704700BF70310024ABAAAAAA0B440024FD
:100CA0000C4B70B50C4C1E7CFFF7CAFF1823054691
:100CB00003FB0644204600F009F9084B00229A5530
:100CC0003DB12A46EB1720460549BDE8704000F0CB
:100CD00067B870BD94390024703100240B4400249F
:100CE000810C010838B5EFF31185102383F31288C6
:100CF000BFF36F8F0F4B104A9C681068A04206D15B
:100D0000FFF7CEFF85F31188BFF36F8F38BD002149
:100D10001B7C1160094AD35C002BF3D02046FFF7FF
:100D20008FFF0028EED0237CDB0601D1FFF71AFDF0
:100D30002046E5E794390024C03900240B44002400
:100D4000EFF31181102383F31288BFF36F8F0A4AE8
:100D5000136A834207D1DB6F136281F31188BFF3FB
:100D60006F8F70471346002BF7D0DA6F8242F9D1AC
:100D7000C26FDA67F1E700BF94390024024B1868AC
:100D8000984208BF0020704700090024034B1B68ED
:100D90000BB9FBF743BC0020704700BFC8390024E3
:100DA000B3F1FF3F08BFB2F1FF3F2DE9F84F044612
:100DB0009946154698467FD08160EFF3118710233E
:100DC00083F31288BFF36F8FB9F1000FDFF8F0A043
:100DD00025DBFFF7DBFF3B4B451906461A6849EB5D
:100DE000E079B2FA82F252095219DAE9005149F176
:100DF00000034FF00109551943EB0108C4E904232E
:100E0000FFF7BCFFDFF8C0E00346DEF804A0EBB953
:100E1000C4E900EACAF80040CEF8044028E0DAE964
:100E200000126FF001035B1A4FF0FF3161EB020219
:100E30005B1B62EB0902012B4FF0000972F100010C
:100E4000BCBF01230022C0E90432D9E7D3E9041C66
:100E5000D4E904208A4270EB0C0B24DA891A5A6810
:100E60006CEB0000C3E90410C4E9003214605C605C
:100E7000FFF784FF84420ED1124B1B685BB9B9F1B6
:100E8000000F02D1FFF782FF064630462FF0DAF856
:100E90000021FBF747FB87F31188BFF36F8F2846CC
:100EA0004146BDE8F88F521A60EB0C005345C4E987
:100EB0000420ADD01B68AAE70025A846EFE700BFD5
:100EC00088310024C8390024000900240246F8B5FE
:100ED000EFF31185102383F31288BFF36F8F01683E
:100EE00051B3FFF74BFF1C4B5B689A4208D0D1E926
:100EF0000434D2E90476DB1944EB0604C1E9043476
:100F0000D2E90031002400264FF0004790420B60E8
:100F10005960C2E90044C2E9046705D0002085F3A6
:100F20001188BFF36F8FF8BDFFF730FF2FF08AF8FD
:100F30002146FBF7F7FAF1E7D0E90413B3F1004FCC
:100F400008BF012904D100204FF00041C2E904018B
:100F50006FF01500E3E700BF000900242DE9F84F0A
:100F6000DFF8BC900C462F4D01264FF0004702469B
:100F7000C9F80000FFF702FF4FEAE278D5E900C1A7
:100F800058B1D0E904AE524578EB0E031CDABAEB47
:100F900002036EEB0806C0E9043612EB0C0241EBCB
:100FA0000801C5E9002100252846C9F800502FF0A6
:100FB00049F82946FBF7B6FA84F31188BFF36F8F1F
:100FC000BDE8F84FFFF78EBE1AEB0C034FF0000B95
:100FD0004FF0100841EBEA71C5E90031D0E9011288
:100FE00003680B605960C0E900BBC0E9046784F383
:100FF0001188BFF36F8F9047EFF3118488F3128845
:10100000BFF36F8FFFF7BAFE18B1D0E90423134383
:10101000E4D0D9F80020A2EB0A02C9F80020ABE71F
:10102000C83900248831002410B5EFF3118410234F
:1010300083F31288BFF36F8FFFF7A8FE054A0346BC
:10104000D2E90001181841EBE37184F31188BFF372
:101050006F8F10BD883100242DE9F0410446EFF375
:101060001187102383F31288BFF36F8F4FF0004670
:10107000D0E90423B34208BF012A05D087F31188C1
:10108000BFF36F8FBDE8F081D0E90A586A1C48F1C0
:101090000003022A73F1000324D32EF0EEFF281878
:1010A00048EB0101012871F1000142DB2EF0E5FF60
:1010B0006FF00203281848EB010183426FF00043F0
:1010C0008B413BDB2EF0D9FF6FF001022D184FF062
:1010D000FF3348EB0108521B63EB08031949204614
:1010E000FFF75EFE236B01332363236A63B187F34B
:1010F0001188BFF36F8F20469847EFF311871023B5
:1011000083F31288BFF36F8F54F8185FA542B5D0F0
:10111000002DB3D028462EF07AFE0023C5F8983073
:1011200087F31188BFF36F8F2846BDE8F0412EF09A
:101130005BBE6FF001024FF0FF33CFE70022334672
:10114000CCE700BF59100108F8B5044616461D4605
:10115000EFF31187102383F31288BFF36F8FB5F17C
:10116000FF3F08BFB2F1FF3F04D187F31188BFF3FF
:101170006F8FF8BDFFF7AAFE0023324623632B468C
:10118000DDE90601C4E90A0120460249FFF708FE2D
:10119000EBE700BF5910010870B50546EFF3118465
:1011A000102686F31288BFF36F8FFFF78FFE20B1F2
:1011B00084F31188BFF36F8F70BD6B6A63B184F3E2
:1011C0001188BFF36F8F6B6A28469847EFF311843D
:1011D00086F31288BFF36F8F05F118002EF054FECE
:1011E0000028E5D02EF000FE21460248BDE8704000
:1011F0002EF076BE0C440024034610B5EFF31184A4
:10120000102282F31288BFF36F8FC16001218160C9
:101210000068834205D184F31188BFF36F8F0020EB
:1012200010BDD0E9003213605A600023C0E90033DA
:101230002EF077FF214602482EF052FEEFE700BF66
:101240000C440024F8B507460C4616462EF068FDFF
:1012500008B10020F8BD0E4B9B68D3F88C50002DD0
:10126000F7D0221DF5D2EFF31184102383F31288F7
:10127000BFF36F8F47F004012846B04784F311880D
:10128000BFF36F8F0028E4D040F8045BE2E700BFB3
:10129000943900240146024A0020FFF7D3BF00BF63
:1012A00091A40308074B07B54FF4806200930649E9
:1012B0004FF0FF330548FFF73FF8002003B05DF81B
:1012C00004FB00BFB82E050800C1002490310024A3
:1012D000F0B504468BB02FF07AF9042C2BD0344DA6
:1012E000286818B118F0DEFE00232B601CB3314BC8
:1012F0009C4220D001AB0026214602A802932E4B2F
:101300000196039332F096FC01983146013018F0B3
:10131000A9FE0246286070B106AF0199384633F045
:101320009CFB264B214604A80593049732F082FCCF
:101330002A68019BD654224D03F0C6FB37F01BFDF3
:101340002FF01EF801F048FB1E4B0022D5F8F040AC
:101350001A7084B1204615F05FF930B3A06807F029
:1013600071FBD5F8F040002CF4D1D5F8F0301C46D4
:10137000DB68002BFBD1C5F8EC400025124C02F0D5
:101380000BFA0EF089F815F037FA206818F08AFE8B
:1013900025600E4C206818F085FE25602EF06BFF4E
:1013A0000BB0BDE8F0402EF0ECBFE468DBE700BF17
:1013B000BC3B0024503C002427020408D349040805
:1013C000D83B00240C440024083A0024043A0024AA
:1013D00070B5164B0022044600EB81059A60C3E904
:1013E000002226460434306832F008F9022818D169
:1013F00030680F4C206098B10E482FF05DF82068DF
:101400002EF061FF0C4802F04BFB01F02BFB07496B
:1014100020682EF053FF0023236001F023FB0120FE
:1014200070BDAC42DDD10020E3E700BFD03900241D
:10143000003A0024664006082764060873B506468D
:101440002EF09FFF12F04AF818F00AFD054618F03A
:1014500013FD044612F04AF8641B0025A4F58060D1
:10146000244C12F049F801F0B7FA00F01BFC6B466F
:101470004FF400622049304600952EF0D8FE1F4BF5
:1014800001461860009B19440DF010F84FF400520B
:1014900001AB1B49304601952EF0C9FE194B0146A0
:1014A0001860019B194415F089F80BF08BFC294654
:1014B000D4F8E8000AF0C4FE1621D4F8E80032F0AF
:1014C00079FD6621D4F8E80032F074FD40F6B6519B
:1014D000D4F8E80032F06EFD294604F1D8000AF095
:1014E000AFFE094806F060FA084B01221A7002B0FC
:1014F00070BD00BFD83B0024BC030608043A00249A
:10150000D3030608083A0024B7DF05080C4400247A
:1015100009282DE9F0410546A4B000F0878001F0CC
:1015200075FA044640B1002D40F08380424BD3F859
:10153000F040003C18BF01242846FFF77FFF2FF042
:101540005EF8002C6CD002AC3C4F01F0F1FA4FF485
:1015500000712046002633F065FA3C6001F05EFA27
:101560000121054600F180082EF03BFF344B354A3F
:1015700006AC3549354835F0DFFE06A800F0FCFA28
:101580003349324835F0FDFE013614F8012B31495C
:101590002E4835F0F6FE202EF6D12F492B4835F097
:1015A000CBFE37F0E9FB02212C48FFF711FF0023A7
:1015B0003B6001F0C3FA0123294A0EA9404638F0E6
:1015C00064FBA0B9029835F0A4FF039A04460146D3
:1015D00001AB01320EA838F07AFC40B9039A019BA6
:1015E0009A4204D12146049840F06BFBA0B14FF41D
:1015F0007A702EF0B8FF0A23194A0EA9404638F037
:1016000044FB01AB0EA8DDE9032138F014FD0EA860
:1016100038F07DFE01F0E0F9002128462EF0E1FED1
:10162000104C6068FFF754FE0023636024B0BDE8EF
:10163000F081002480E700BFD83B0024CC3900248F
:10164000ED030608FE0306085D0406086C94050811
:10165000B65B060813640608020C0608F42E05089B
:101660006D040608D03900242DE9F04F814689B079
:10167000AA4E002842D00024202725463368B3F51F
:10168000007F00F0B480B9F1000F40F0B480012673
:101690004FF4405302932EF062FF0390002C40F071
:1016A0003A814FF4C87BA0460BFB06F3012603F5F5
:1016B0009C5A04930AF1080A02F03CF802F0A2F9DD
:1016C00005460190002800F0998047F0100702F0CD
:1016D0004DF9934E306828B103781F4002D118F0BD
:1016E000E1FC3760B8F1000F04D0002002F0EAF806
:1016F00002F0E2F8284609B0BDE8F08F01F06CF97D
:1017000002F09EF905460028B5D1854FFFF796FEF9
:101710002EF077FF3B68002B56D01A7822F020027B
:101720001A703B689A681C78127892B1586808B1B0
:1017300006F03AF93B68012107A89B680793FFF779
:1017400047FE98B93B6898682EF0B6FE754802F0DF
:10175000A7F904217448FFF73BFE38B90821734804
:10176000FFF736FE10B1724802F09AF93368180597
:101770002CD500F0B1FF012828D16E4802F090F975
:101780004FF000086C4B706883F80080FFF7A0FDF5
:101790003A68C6F804802AB11378990644BF43F02A
:1017A0002003137033681A0512D500F095FF441E0C
:1017B0004FF0300718BF0124336803F48073002B07
:1017C0000CBF2546012459E72C46C2E75B48D5E704
:1017D0001BB904F001042427EEE714F002044FF0D3
:1017E00028071CBF83F48063C3F38024E4E7022648
:1017F0004FF440134EE70326514B4BE72EF035FED6
:10180000059080B12EF050FE68B102F019F905463E
:1018100048B92EF037FE04287FF45BAF032000F0B8
:1018200061FF059D55E7F4B92EF01FFEE0B102F00F
:1018300007F9C8B943482EF046FD02F0BFF800286A
:101840003AD0414802F02CF9B9F1000F02D03F48DC
:1018500002F026F9484601F0A5FC3D482EF02CFE8A
:101860003C4802F01DF901242EF0FFFD2040C4B2D7
:101870002EB102F0E5F810B904F03AFF06462EF05A
:101880006EFE039B049A0546C31A9A4223D9B3FB02
:10189000FBF20BFB1235632D10D9B8F1000F04D009
:1018A000002002F00FF802F007F8C5F5C8706EB31B
:1018B000B04228BF304629E02748C3E7B8F1000FFF
:1018C00004D102F019F8029801F0FCFF0123C5F1E0
:1018D00064000193EBE79A4507D22EF040FECDF865
:1018E00004800390DDF80480E6E6B8F1000F04D030
:1018F000002001F0E7FF01F0DFFF039B5344581B7A
:1019000016B1B04228BF30460028EBD018F0D8FA04
:1019100018F020FBE6E74FF00008DAE6D0390024A3
:10192000B83B00242E640608E42E0508C42E0508E2
:10193000E85A0608595A06080C440024735A060847
:1019400000303000664006081B620608C25C0608CC
:101950008E050608425D060849620608114B07B568
:10196000186820B103B05DF804EB2EF0A5BD0E4B56
:101970001A6892050FD59A68002A0CDD596851B192
:1019800009680C330948C9880091094935F0D4FC2D
:1019900003B05DF804FB074803B05DF804EB02F008
:1019A0007FB800BF003A0024D03900246C940508A9
:1019B0007B040608B3600608F7B518F035FA01F0A5
:1019C0003FFB2EF058FC18F0E7FA2EF0B7FF01F0BD
:1019D000CDF850482EF077FC2EF034FD01F0B8F829
:1019E00001F028FBB0FA80F00021400900F026FF4A
:1019F00010B9082001F024FB01F01CFB18B901F01C
:101A000025FB01F01DFB37F0B6F92EF0B9FC00F014
:101A1000BFFE03F0A5F93F482EF055FC002000F072
:101A200061FE01F007FB08B901F0A6FF01200125C6
:101A300000F0E6FF012000F0DDFF4FF4807401F0BC
:101A4000F9FA354EFFF764FD2EF09CFC012000F002
:101A5000FDFF284614F4106754D015B92F4802F042
:101A60001FF83578002D3ED101F0E4FAFFF7FCFDB8
:101A70000028EFD101F0DEFA044600F0ADFF204669
:101A8000FFF7DCFC2EF0BDFD012001F087FF01F027
:101A9000D1FA28B9224B012101A80193FFF798FC44
:101AA00001F02AFF1F4801F00DFF01F005FF337818
:101AB000012B1AD101F03CF800F098FC044601F02B
:101AC0003DF80420FFF704FC01F016FF002001F0B0
:101AD000F9FE01F0F1FE012001F068FF032000F0A3
:101AE00001FE0020B6E70025C4E70F4B0F4F3B6017
:101AF00000F0B8FF00F000FD002304463B6000F05A
:101B0000B1FFDEE7002CB3D032F081FC384603B0E1
:101B1000F0BD00BF664006080D4400248F52060841
:101B200084040608303030008C040608003A002493
:101B300008B514F081FD00F01BFB0421064835F0C8
:101B400093FC2EF05BFD01F05BFE03F043F8BDE873
:101B5000084014F085BD00BFC83C0024014B187834
:101B6000704700BF0C440024004870470076B01056
:101B7000004870473333534038B505462021F9F704
:101B800037FA041E11DA21460024094828F0BEFD68
:101B900021462022074828F0B9FDC4F12002281967
:101BA0000021BDE8384040F084B81F2CF0DD38BD7E
:101BB0001C050608360506080428034607B506D89E
:101BC00001460F4803B05DF804EB01F021B806218F
:101BD0000C4A684626F0F0F9011E0DDD052901D9F1
:101BE00029F097FB01F108034422013168466B4458
:101BF00003F8082C01F00CF803B05DF804FB00BFFB
